:0200000480007A
:1000000097E11300938111FE13850100138601000F
:100010003306A64093050000EF60835017350300B8
:10002000130585606308050017050400130585485E
:10003000EF30435FEF50037003250100930541004B
:1000400013060000EF00D07A6F30C36DB7B704809D
:1000500003C707CA63140704130101FF23248100A7
:1000600013840700B70700002326110093870700B9
:10007000638A070037B504801305C5CB97000000DD
:10008000E7000000930710008320C1002300F4CA9A
:1000900003248100130101016780000067800000D4
:1000A000B707000093870700638E0700B7B5048089
:1000B00037B50480938545CA1305C5CB17030000E7
:1000C0006700000067800000130101FD2326810204
:1000D00013040103232EA4FC232CB4FC232AC4FC08
:1000E0008327C4FD83A707002326F4FE832744FD4E
:1000F0002322F4FE832744FE03C707008327C4FEA0
:100100002380E7008327C4FE93871700032744FE5C
:10011000034717002380E7008327C4FE9387270047
:10012000032744FE034727002380E7008327C4FEFC
:1001300093873700032744FE034737002380E700F7
:100140008327C4FE938747002326F4FE232404FE5E
:10015000032784FE832744FD635CF702832784FE24
:10016000032784FDB307F70003C707008327C4FEF6
:100170002380E7008327C4FE938717002326F4FE1D
:10018000832784FE938717002324F4FE6FF05FFC1F
:100190008327C4FD0327C4FE23A0E700130000004B
:1001A0000324C1021301010367800000130101FD54
:1001B0002326810213040103232EA4FC232CB4FC68
:1001C0008327C4FD83A707002326F4FE832744FE6C
:1001D0002320F4FE8327C4FE03C70700832704FE01
:1001E0002380E700832704FE938717000327C4FEBC
:1001F000034717002380E700832704FE9387270027
:100200000327C4FE034727002380E700832704FE5B
:10021000938737000327C4FE034737002380E70096
:100220008327C4FE938747002326F4FE232404FE7D
:10023000032784FE832744FE635CF702832784FE42
:10024000032784FDB307F7000327C4FE0347070015
:100250002380E7008327C4FE938717002326F4FE3C
:10026000832784FE938717002324F4FE6FF05FFC3E
:100270008327C4FD0327C4FE23A0E700130000006A
:100280000324C1021301010367800000130101FF71
:100290002326810013040101130000000324C10080
:1002A0001301010167800000130101FE232E81006C
:1002B000130401022326A4FE2324B4FE832784FE14
:1002C0003727000023A2E7009307000013850700EB
:1002D0000324C1011301010267800000130101FE24
:1002E000232E8100130401022326A4FE930710008D
:1002F000138507000324C101130101026780000078
:10030000130101FF232681001304010113000000E3
:100310000324C1001301010167800000130101FFE4
:100320002326810013040101130000000324C100EF
:100330001301010167800000130101FD23268102E2
:1003400013040103232EA4FC232CB4FC232AC4FC95
:10035000B70701002324F4FE232604FE0327C4FE6E
:10036000832744FD6356F7028327C4FE032784FDD9
:10037000B307F70003C70700B707010023A0E70092
:100380008327C4FE938717002326F4FE6FF01FFD1A
:10039000832744FD138507000324C10213010103D1
:1003A00067800000130101FD23268102130401036D
:1003B000232EA4FC8327C4FD63D807008327C4FD34
:1003C000B307F040232EF4FC0327C4FDB737000029
:1003D0009387078063D8E700B737000093870780CB
:1003E000232EF4FCB7B7048083A747DA2326F4FE54
:1003F000B7B7048003A747DA8327C4FD3307F700A4
:10040000B7B7048023A2E7DA8327C4FE1385070069
:100410000324C1021301010367800000130101FEE0
:10042000232E1100232C8100130401022326A4FE95
:1004300013050000EF00C00E130000008320C1016F
:10044000032481011301010267800000130101FFF1
:100450002326810013040101130000000324C100BE
:100460001301010167800000130101FF23268100B1
:1004700013040101130000000324C1001301010152
:1004800067800000130101FF23261100232481004F
:1004900013040101EF00400B9307050013850700CB
:1004A0008320C10003248100130101016780000043
:1004B000130101FF23268100130401011300000032
:1004C0000324C1001301010167800000130101FF33
:1004D0002326810013040101B7B7048083A7C7D581
:1004E0009386170037B70480232ED7D413850700CF
:1004F0000324C1001301010167800000130101FF03
:100500002326810013040101130000000324C1000D
:1005100013010101678000006B10B50067800000C7
:100520006B000500678000006B40B500678000002D
:100530006B200500678000006B30000067800000C2
:100540007325100267800000732500026780000099
:10055000130540006B000500F32610029396F60089
:10056000732600029315A6001316260037F1FF6FBD
:100570003301B1403301D1403301C100F3261002F1
:1005800063860600130500006B000500678000000D
:10059000130141FF232011002322B10083450500F0
:1005A00063880500EF00C001130515006FF01FFF01
:1005B00083200100832541001301C10067800000F2
:1005C000B702010023A0B20067800000130101FD03
:1005D000232611022324810213040103232EA4FCE9
:1005E0000327C4FD9307F00063E4E702B7B7048074
:1005F0001387870A8327C4FD93972700B307F70063
:1006000083A7070013850700EFF09FF86F008007AE
:10061000930700022326F4FEA30504FE8327C4FEED
:100620009387C7FF0327C4FDB357F70093F7F7007D
:100630002322F4FE832744FE6386070093071000FD
:10064000A305F4FE8347B4FE63820702B7B70480B4
:100650001387870A832744FE93972700B307F70081
:1006600083A7070013850700EFF09FF28327C4FEDE
:100670009387C7FF2326F4FE8327C4FE6354F0004C
:100680006FF0DFF98320C10203248102130101030B
:1006900067800000130101FE232E1100232C81002E
:1006A000130401022326A4FE2324B4FE0325C4FE62
:1006B000EFF01FEE032584FEEFF05FF1B7B7048083
:1006C00013858712EFF0DFEC130000008320C101D7
:1006D000032481011301010267800000130101FE60
:1006E000232E1100232C810013040102B7B70480CC
:1006F00083A7C71B13850700EFF09FE2B7B70480FD
:1007000003A7471BB7B7048083A7871B1385070080
:10071000E7000700EFF0DFE2930705002326F4FE71
:100720008327C4FE6388070013050000EFF05FDF36
:100730006F00C00013051000EFF09FDE13000000F3
:100740008320C1010324810113010102678000009D
:10075000130101FE232E1100232C8100130401023A
:100760002326A4FE2324B4FE2322C4FE2320D4FE89
:10077000B7B70480032744FE23AAE71AB7B704805B
:10078000032704FE23ACE71AB7B70480032784FECF
:1007900023AEE71AB70700809387C76D93850700DC
:1007A0000325C4FEEFF05FD7EFF05FF31300000006
:1007B0008320C1010324810113010102678000002D
:1007C000130101FE232E1100232C810013040102CA
:1007D000B7B704801385872FEFF09FDB1305400028
:1007E000EFF01FD4EFF05FD6930705002326F4FE49
:1007F0000327C4FEB7B70480938687288327C4FEE7
:1008000093972700B387F60023A0E7001305100095
:10081000EFF01FD1B7B704809387872883A707001D
:1008200013850700EFF09FDAB7B704801385873090
:10083000EFF01FD6B7B704809387872883A74700B8
:1008400013850700EFF09FD8B7B704801385873072
:10085000EFF01FD4B7B704809387872883A787005A
:1008600013850700EFF09FD6B7B704801385873054
:10087000EFF01FD2B7B704809387872883A7C700FC
:1008800013850700EFF09FD4B7B704801385873036
:10089000EFF01FD0130000008320C1010324810169
:1008A0001301010267800000130101FE232E1100D5
:1008B000232C810013040102EFF01FC993070500E8
:1008C0002326F4FE8327C4FE93B72700A305F4FE76
:1008D0008347B4FE13850700EFF09FC58347B4FE3E
:1008E000638407068327C4FE93B71700A304F4FEAE
:1008F000834794FE13850700EFF09FC3834794FE60
:1009000063820702B7B70480138787298327C4FE51
:1009100093972700B307F7001307A00023A0E70071
:100920006F000002B7B70480138787298327C4FEAE
:1009300093972700B307F7001307B00023A0E70041
:10094000EFF09FBF6F0040068327C4FE93B73700C8
:100950002305F4FE8347A4FE13850700EFF05FBD77
:100960008347A4FE63820702B7B7048013878729F1
:100970008327C4FE93972700B307F7001307C0002F
:1009800023A0E7006F000002B7B704801387872910
:100990008327C4FE93972700B307F7001307D000FF
:1009A00023A0E700EFF05FB9EFF01FB9B7B70480FD
:1009B0009387872983A7070013850700EFF01FC1DE
:1009C000B7B7048013858730EFF09FBCB7B70480BA
:1009D0009387872983A7470013850700EFF01FBF80
:1009E000B7B7048013858730EFF09FBAB7B704809C
:1009F0009387872983A7870013850700EFF01FBD22
:100A0000B7B7048013858730EFF09FB8B7B704807D
:100A10009387872983A7C70013850700EFF01FBBC3
:100A2000B7B7048013858730EFF09FB6130000003E
:100A30008320C101032481011301010267800000AA
:100A4000130101FE232E1100232C81001304010247
:100A5000EFF01FAF930705002326F4FEB7B704801D
:100A60001387872A8327C4FE93972700B307F700CD
:100A70000327C4FE23A0E7008327C4FE6386070084
:100A800013050000EFF0DFA9130000008320C1016F
:100A9000032481011301010267800000130101FE9C
:100AA000232E1100232C810013040102B7170080AC
:100AB000938707A42326F4FE8325C4FE1305400074
:100AC000EFF09FA5EFF0DFF7B7B704809387872A91
:100AD00083A7070013850700EFF05FAFB7B7048067
:100AE00013858730EFF0DFAAB7B704809387872A92
:100AF00083A7470013850700EFF05FADB7B7048009
:100B000013858730EFF0DFA8B7B704809387872A73
:100B100083A7870013850700EFF05FABB7B70480AA
:100B200013858730EFF0DFA6B7B704809387872A55
:100B300083A7C70013850700EFF05FA9B7B704804C
:100B400013858730EFF0DFA4130000008320C1017C
:100B5000032481011301010267800000130101FFDA
:100B6000232611002324810013040101EFF05FC547
:100B7000B7B704801385C730EFF09FA1130540007D
:100B8000EFF01F9AEFF05FD213051000EFF05F99BE
:100B9000B7B7048013850732EFF09F9FEFF01FF087
:100BA000130000008320C100032481001301010110
:100BB00067800000130101FC232E1102232C810207
:100BC00013040104232EA4FC232CB4FC232AC4FC0C
:100BD0002328D4FC2326E4FC2324F4FCB7B70480A8
:100BE0001385C74CEF50D32C8325C4FDB7B70480C1
:100BF0001385C74EEF50D32B8325C4FDB7B70480B0
:100C000013854750EF50D32AB7B7048003A707478F
:100C100093071000631CF700B7B704801385875152
:100C2000EF5013299307F0FF6F00C00BB7B7048094
:100C300083A7074793850700B7B7048013854753F9
:100C4000EF501327B7B7048083A707479386170091
:100C500037B704802328D746138707009307070078
:100C600093971700B387E700939737001387070020
:100C7000B7B7048093874747B307F7002326F4FEEE
:100C80008327C4FE0327C4FD23A0E7008327C4FEF7
:100C9000032784FD23A2E7008327C4FE032744FD26
:100CA00023A4E7008327C4FE032704FD23A6E7004F
:100CB0008327C4FE0327C4FC23A8E7008327C4FEC0
:100CC000032784FC23AAE7008327C4FE83A7070029
:100CD00093850700B7B7048013854755EF50531D20
:100CE00093070000138507008320C10303248103B9
:100CF0001301010467800000130101FC232E11027F
:100D0000232C810213040104232EA4FC232CB4FC05
:100D1000232AC4FC2328D4FC2326E4FC2324F4FC4B
:100D2000B7B704801385C756EF5093188325C4FDC9
:100D3000B7B7048013854759EF509317B7B70480AE
:100D400083A7074793850700B7B704801385075A21
:100D5000EF501316232604FEB7B7048083A7074776
:100D60000327C4FE635EF7108325C4FEB7B7048073
:100D70001385475BEF50D3130327C4FE9307070087
:100D800093971700B387E7009397370013870700FF
:100D9000B7B7048093874747B307F7002324F4FECF
:100DA000832784FE83A707008325C4FD13850700DE
:100DB000EF70435093070500B337F00093F7F70F38
:100DC00063820702832784FE83A707000326C4FDEE
:100DD00093850700B7B704801385075DEF50530D67
:100DE0006F000009B7B7048013850760EF50530CFC
:100DF000832784FD638A0700832784FE03A74700B7
:100E0000832784FD23A0E700832744FD638A07002E
:100E1000832784FE03A78700832744FD23A0E700E0
:100E2000832704FD638A0700832784FE03A7C70086
:100E3000832704FD23A0E7008327C4FC638A0700FF
:100E4000832784FE03A707018327C4FC23A0E700B0
:100E5000832784FC638A0700832784FE03A7470156
:100E6000832784FC23A0E700930700006F00800124
:100E70008327C4FE938717002326F4FE6FF0DFED6F
:100E80009307F0FF138507008320C1030324810328
:100E90001301010467800000130101FF23261100E4
:100EA0002324810013040101B7C7048083A7C7C1AD
:100EB000638A0700B7C7048083A7C7C113850700EB
:100EC000EF109014B7C7048083A747C2638A070056
:100ED000B7C7048083A747C213850700EF8010526D
:100EE000B7C7048083A707C2638A0700B7C7048017
:100EF00083A707C213850700EF409005B7C704809A
:100F000083A787C2638A0700B7C7048083A787C205
:100F100013850700EF309024B7C7048083A7C7C2AA
:100F2000638A0700B7C7048083A7C7C21385070079
:100F3000EF30D022B7C7048083A707C3638A0700B6
:100F4000B7C7048083A707C313850700EF301021BC
:100F5000B7C7048083A787C1638A0700B7C7048027
:100F600083A787C113850700EF00D04AB7C7048065
:100F700083A707C4638A0700B7C7048083A707C491
:100F800013850700EF40D324B7C7048083A747C366
:100F9000638A0700B7C7048083A747C31385070088
:100FA000EF401323B7C7048083A787C3638A070072
:100FB000B7C7048083A787C313850700EF40532179
:100FC000B7C7048083A7C7C3638A0700B7C7048075
:100FD00083A7C7C313850700EF40931F13000000CA
:100FE0008320C100032481001301010167800000F8
:100FF000130101F52326110A2324810A1304010B8E
:101000002326A4F62324B4F613051000EFF04FD1E5
:10101000B7B704801385C761EFF08FD7B7B70480E7
:1010200013850763EF50C3689307C4F913060000E4
:101030009385070013051000EFC0806B9307050030
:101040002322F4FE832744FE63840702032644FE22
:10105000B7B704809385C764B7B704801385476723
:10106000EF500365EFF05FE31305F0FFEF20836BB4
:10107000130000008327C4F993850700B7B70480E5
:1010800013858769EF50C3620325C4F9130784F9F8
:10109000930700009306100093051000130600004C
:1010A000EFC01018930705002320F4FE832704FEE9
:1010B00063840702032604FEB7B704809385076B99
:1010C000B7B7048013854767EF50835EEFF0DFDC2E
:1010D0001305F0FFEF20036513000000B7B704808D
:1010E0001385C76FEF50C35C930720FE2326F4F8E7
:1010F0009307C4F8130684F9130700009306000051
:101100009305100013050000EFD080289307050019
:10111000232EF4FC8327C4F8638607028327C4F8D0
:1011200013860700B7B704809385C771B7B70480EB
:1011300013854767EF50C357EFF01FD61305F0FF35
:10114000EF20435EB7C704800327C4FD23ACE7C08C
:10115000B7B7048013854775EF508355930720FE7A
:101160002324F4F8B7C7048003A587C1930784F844
:1011700013070000930600019305400013060000CA
:10118000EF10502593070500232CF4FC832784F8E7
:1011900063860702832784F813860700B7B70480A5
:1011A00093854776B7B7048013854767EF50435060
:1011B000EFF09FCE1305F0FFEF20C356B7C70480B2
:1011C000032784FD23A4E7C2930720FE2322F4F81B
:1011D000B7C7048003A587C1930744F8130700002D
:1011E000930600019305400013060000EF10901EC7
:1011F00093070500232AF4FC832744F8638607023B
:10120000832744F813860700B7B704809385477691
:10121000B7B7048013854767EF508349EFF0DFC706
:101220001305F0FFEF200350B7C70480032744FDE8
:1012300023A6E7C2930720FE2320F4F8B7C7048053
:1012400003A587C1930704F8130700009306000164
:101250009305200013060000EF10D0179307050038
:101260002328F4FC832704F863860702832704F805
:1012700013860700B7B704809385477BB7B7048010
:1012800013854767EF50C342EFF01FC11305F0FF0E
:10129000EF204349B7C70480032704FD23A8E7C212
:1012A000B7C7048013854780EF50834013050001C2
:1012B000EF4003719307050013870700B7C7048049
:1012C00023AAE7C213050001EF40836F93070500CF
:1012D00013870700B7C7048023ACE7C213050001DA
:1012E000EF40036E9307050013870700B7C704801C
:1012F00023AEE7C2B7C7048003A747C3B7C70480BC
:1013000003A687C3B7C7048083A7C7C39386070014
:1013100093050700B7C7048013858781EF504339D1
:10132000232604FE0327C4FE9307300063CCE704A2
:10133000B7C7048003A747C38327C4FE939727003A
:10134000B307F7000327C4FE1317170023A0E70015
:101350008327C4FE13971700B7C7048083A687C3EB
:101360008327C4FE93972700B387F600130717005F
:1013700023A0E7008327C4FE938717002326F4FEEB
:101380006FF05FFAB7C704801385C783EF5043320D
:10139000930720FE232EF4F6B7C7048003A587C168
:1013A0009307C4F7130684F913870700B7C70480AF
:1013B0009386078793051000EF305063930705006D
:1013C0002326F4FC8327C4F7638607028327C4F728
:1013D00013860700B7C7048093858787B7B7048053
:1013E00013854767EF50C32CEFF01FAB1305F0FFD9
:1013F000EF204333B7C704800327C4FC23A0E7C210
:10140000B7C704801385878CEF50832AB7C7048041
:1014100003A507C2130684F9930700001307000011
:101420009306000093051000EF40D02E93070500AF
:101430002324F4FC832784FC63840702032684FCB2
:10144000B7C704809385C78FB7B7048013854767F4
:10145000EF500326EFF05FA41305F0FFEF20832C7D
:1014600013000000930720FE232CF4F6B7C7048076
:1014700003A707C2930784F713860700B7C7048042
:101480009385078713050700EF70504C93070500FD
:101490002322F4FC832784F763860702832784F7DB
:1014A00013860700B7C7048093858793B7B7048076
:1014B00013854767EF50C31FEFF01F9E1305F0FF22
:1014C000EF204326B7C70480032744FC23A2E7C2CA
:1014D000B7C7048003A747C2B7C70480938687C2F3
:1014E000130640009305000013050700EF80D03D70
:1014F000930705002320F4FC832704FC6384070280
:10150000032604FCB7C7048093854796B7B70480C9
:1015100013854767EF50C319EFF01F981305F0FFCD
:10152000EF20432013000000B7C7048003A747C281
:10153000B7C704809386C7C2130640009305100006
:1015400013050700EF80503893070500232EF4FAA7
:101550008327C4FB638407020326C4FBB7C7048048
:101560009385479AB7B7048013854767EF504314B4
:10157000EFF09F921305F0FFEF20C31A1300000055
:10158000B7C7048003A747C2B7C70480938607C3C1
:10159000130640009305200013050700EF80D032AA
:1015A00093070500232CF4FA832784FB6384070246
:1015B000032684FBB7C704809385479EB7B7048092
:1015C00013854767EF50C30EEFF01F8D1305F0FF33
:1015D000EF20431513000000930720FE232AF4F6A2
:1015E000B7C7048083A787C1832584F9130744F70D
:1015F000130600009306000013850700EF00D038A3
:1016000093070500232AF4FA832744F76386070229
:10161000832744F713860700B7C70480938547A242
:10162000B7B7048013854767EF508308EFF0DF8674
:101630001305F0FFEF20030FB7C70480032744FB17
:1016400023AEE7C0B7C7048003A5C7C1B7C70480EE
:1016500083A587C2B7C7048083A747C3232001009F
:101660009308000013080000130700019306000010
:1016700013061000EFD08066930705002328F4FAC4
:10168000832704FB63840702032604FBB7C7048097
:10169000938587A5B7B7048013854767EF5043014B
:1016A000EFF08FFF1305F0FFEF20C30713000000DA
:1016B000B7C7048003A5C7C1B7C7048083A5C7C245
:1016C000B7C7048083A787C32320010093080000C5
:1016D0001308000013070001930600001306100012
:1016E000EFD0C05F930705002326F4FA8327C4FADE
:1016F000638407020326C4FAB7C704809385C7AB87
:10170000B7B7048013854767EF40937AEFF0CFF8BF
:101710001305F0FFEF2003011300000093074000C2
:10172000232AF4F8930720002328F4F8B7C704808D
:1017300003A5C7C1B7C7048083A547C2930704F9AF
:10174000130744F923200100930800001308000048
:101750009306000013061000EF9000789307050031
:101760002324F4FA832784FA63840702032684FA85
:10177000B7C70480938507B2B7B70480138547675E
:10178000EF401373EFF04FF11305F0FFEF10937973
:1017900013000000B7C7048083A7C7C113850700E3
:1017A000EFE04079930705002322F4FA832744FAF7
:1017B00063840702032644FAB7C70480938587B879
:1017C000B7B7048013854767EF40936EEFF0CFEC17
:1017D0001305F0FFEF10137513000000B7C7048066
:1017E00003A5C7C1B7C7048083A507C3B7C70480D3
:1017F00083A7C7C32320010093080000130800003B
:10180000130700019306000013061000EF2050009C
:10181000930705002320F4FA832704FA6384070260
:10182000032604FAB7C70480938507BAB7B70480C4
:1018300013854767EF40D367EFF00FE61305F0FF1E
:10184000EF10536E13000000232404FE232604FE31
:101850000327C4FE9307300063CEE706B7C70480B2
:1018600003A7C7C38327C4FE93972700B307F700D6
:1018700003A70700B7C7048083A647C38327C4FE16
:1018800093972700B387F60083A60700B7C70480A5
:1018900003A687C38327C4FE93972700B307F600E8
:1018A00083A70700B387F600630EF700B7C704806D
:1018B000138507C0EF40D35F930710002324F4FE85
:1018C0006F0040018327C4FE938717002326F4FE90
:1018D0006FF01FF80327C4FE930740006318F7005A
:1018E000B7C704801385C7C0EF40935CEFF0CFDA31
:1018F000832784FE138507008320C10A0324810AFD
:101900001301010B67800000130101FF2326110062
:10191000232481001304010137C50480130595D2E7
:10192000EF004001032481008320C1001301010165
:1019300067800000130101FF23261100232481008A
:1019400013040101232AA4FE37C50480130515D30F
:10195000B7250080938585A837C604801307A6D2D3
:1019600037C60480930706D31306300093060000A1
:10197000EFF04FA4032481008320C1001301010173
:1019800067800000130101FF23261100232481003A
:1019900013040101EFF05FF7032481008320C100ED
:1019A0001301010167800000130101FE232E1100C5
:1019B000232C8100232A9100232821012326310191
:1019C0002324410123225101130401021371C1FF99
:1019D0001389060093090600138A0500930A05007F
:1019E00083A48601138504009305070097900400E3
:1019F000E78040CD8325C9003385A5001315250058
:101A0000B382AA003303AA00B383A9000328090202
:101A1000032EC90193080000930E000013850200F5
:101A200093050300138603009307000003270500B6
:101A300083A60500B386E6002320D60013054500E3
:101A4000938545001306460093871700E3E097FE51
:101A5000938E1E00E3E4CEFD93881800E3EE08FBAE
:101A6000130104FE832A4100032A81008329C10057
:101A70000329010183244101032481018320C10141
:101A80001301010267800000130101FF23261100EA
:101A90002324810023229100232021019384050027
:101AA0001309050003A4850113050400930506002E
:101AB00097900400E78000C183A5C4003385A5008A
:101AC000131525008325890083A5050003264900F9
:101AD000032606008326090083A60600B382A6001B
:101AE0003303A600B383A50003A8040203AEC40118
:101AF000930800009304000013850200930503007F
:101B000013860300930700008326050003A7050042
:101B1000B306D7002320D600130545009385450062
:101B20001306460093871700E3E087FE93841400B2
:101B3000E3E4C4FD93881800E3EE08FB03290100E9
:101B400083244100032481008320C100130101018B
:101B500067800000130101FF232611002324810068
:101B600023229100232021019384050013090500FD
:101B700003A4850113050400930506009790040053
:101B8000E78040B483A5C4003385A5001315250064
:101B9000832589000326490083260900B382A60015
:101BA0003303A600B383A50003A8040203AEC40157
:101BB00093080000930400001385020093050300BE
:101BC00013860300930700008326050003A7050082
:101BD000B306D7002320D6001305450093854500A2
:101BE0001306460093871700E3E087FE93841400F2
:101BF000E3E4C4FD93881800E3EE08FB0329010029
:101C000083244100032481008320C10013010101CA
:101C100067800000130101FD2326110223248102A5
:101C2000232221032320310313040103232EA4FCC8
:101C30008326C4FD83C68601639C06000325C4FD7C
:101C4000EF301359232E04FC930700006F0000307F
:101C500097E6FF019386863B03A6060083A646000F
:101C60001377060493F7060093060700B3E6F60021
:101C70006384060AEF4001189306100017A60400BB
:101C80001306C6179305E00217A504001305C52720
:101C9000EF40D10597E7FF019387C73683A7070079
:101CA000638807029797040083A7C7FE83A70700EE
:101CB00083A7C700938607001306E0009305100072
:101CC00017A5040013054514EF30D30E6F00000272
:101CD0009797040083A707FC83A7070083A7C70083
:101CE0009385070013050002EF20034F9797040028
:101CF00083A747FA83A7070083A7C7009386070037
:101D0000130610019305100017A504001305C51054
:101D1000EF30530AEF40C10F8327C4FD83A747006C
:101D20006342F00297A604009386461017A60400AB
:101D30001306861D9305F00217A50400130505116F
:101D4000EF1093078327C4FD83A747009387F7FF0E
:101D50000327C4FD2322F7002324F4FE8327C4FDB8
:101D600083A7470063D2070297A604009386061054
:101D700017A60400130646199305F00217A50400E0
:101D80001305C50CEF105303832784FE639E071AC7
:101D900097E7FF019387872703A7070083A74700DB
:101DA0001379070493F9070093070900B3E7370194
:101DB0006382070AEF4001049306100017A604008F
:101DC0001306C6039305200317A504001305C513C6
:101DD000EF40C17197E7FF019387C72283A70700F0
:101DE000638807029797040083A7C7EA83A70700C1
:101DF00083A7C700938607001306E0009305100031
:101E000017A5040013054500EF30C37A6F000002E8
:101E10009797040083A707E883A7070083A7C70055
:101E20009385070013050002EF20033B97970400FA
:101E300083A747E683A7070083A7C7000326C4FD3F
:101E400097A504009385850413850700EF20432E92
:101E5000EF30117C232604FE6F0000038327C4FDAE
:101E600003A787008327C4FE93972700B307F700D3
:101E700083A7070013850700EFE080178327C4FEC0
:101E8000938717002326F4FE8327C4FD83A7070149
:101E90000327C4FEE364F7FC8327C4FD83A7870000
:101EA00013850700EF30D3328327C4FD23A4070036
:101EB0008327C4FD83A7C70013850700EF30533184
:101EC0008327C4FD23A60700232604FE6F00800499
:101ED0000327C4FD8327C4FE9387870093972700B9
:101EE000B307F70083A7070013850700EF30532ED1
:101EF0000327C4FD8327C4FE938787009397270099
:101F0000B307F70023A007008327C4FE93871700B9
:101F10002326F4FE0327C4FE93075000E3FAE7FAF2
:101F20000325C4FDEF30D32A232E04FC9797040029
:101F300083A707D683A707001387F7FF97970400A7
:101F400083A707D523A0E7009307000013850700A8
:101F50008320C10203248102032941028329010253
:101F60001301010367800000130101FD2326110204
:101F7000232481022322210323203103232E410124
:101F8000232C5101130401039305000017A504003D
:101F9000130505F1EF305153232EA4FC8327C4FD14
:101FA0006382071C9797040083A787CE83A7070047
:101FB00093B7170093F7F70F232CF4FC832784FDC6
:101FC000638A070C97E7FF019387470403A707007D
:101FD00083A74700137A070493FA070093070A00C0
:101FE000B3E757016384070AEF30D160930610000E
:101FF00017A60400130686E09305D00617A5040073
:102000001305C5F1EF40814E97E7FF01938787FFE6
:1020100083A70700638807029797040083A787C7F1
:1020200083A7070083A7C700938607001306E00075
:102030009305100017A50400130505DDEF30835745
:102040006F0000029797040083A7C7C483A7070007
:1020500083A7C7009385070013050002EF20C3176D
:102060009797040083A707C383A7070083A7C70028
:1020700093860700130600039305100017A50400BC
:10208000130545E3EF300353EF309158EF705120C3
:102090006F00800D97E7FF01938747F703A70700BD
:1020A00083A74700B71600003379D70093F90700DC
:1020B00093070900B3E737016388070AEF309153AC
:1020C0009306300017A60400130606E293052007C6
:1020D00017A50400130585E4EF40414197E7FF0190
:1020E000938747F283A70700638807029797040046
:1020F00083A747BA83A7070083A7C7009386070073
:102100001306E0009305100017A504001305C5CFC2
:10211000EF30434A6F0000029797040083A787B708
:1021200083A7070083A7C700938507001305000254
:10213000EF20830A9797040083A7C7B583A70700FA
:1021400083A7C7009386070013066001930510005C
:1021500017A504001305C5D9EF30C345EF30514B27
:102160006F008000130000008320C102032481025D
:102170000329410283290102032AC101832A810123
:102180001301010367800000130101FB23261104E2
:10219000232481042322910423202105232E3103AB
:1021A000232C4103232A5103130401052326A4FCF5
:1021B0002324B4FC2320C4FC2322D4FC232EE4FAE1
:1021C000232A04FC8327C4FC6394070E97E7FF01CE
:1021D0009387C7E303A7070083A74700B71600004C
:1021E000337ED70093FE070093070E00B3E7D701B5
:1021F000638A070AEF3011409306300017F6040097
:102200001306C63A9305600217F5040013054550FE
:10221000EF40C12D97E7FF019387C7DE83A7070033
:10222000638807029797040083A7C7A683A70700C0
:1022300083A7C700938607001306000293051000CA
:1022400017F5040013050537EF30C3366F00C002E1
:102250009797040083A707A483A7070083A7C70055
:1022600093860700130630019305100017F504004C
:1022700013058536EF3003349797040083A787A1B1
:1022800083A7070083A7C70017F6040013060636C6
:1022900097F504009385C53613850700EF10536941
:1022A000EF3011379307E0FD232CF4FC6F00C05191
:1022B000832784FC6394070E97E7FF01938707D574
:1022C00003A7070083A74700B71600003373D700A2
:1022D00093F3070093070300B3E77700638A070AC5
:1022E000EF3051319306300017F604001306062C28
:1022F0009305800217F5040013058541EF40011F87
:1023000097E7FF01938707D083A707006388070239
:102310009797040083A7079883A7070083A7C700A0
:10232000938607001306F0019305100017F50400CB
:102330001305452DEF3003286F00C0029797040066
:1023400083A7479583A7070083A7C7009386070045
:10235000130620019305100017F504001305852CC2
:10236000EF3043259797040083A7C79283A7070000
:1023700083A7C70017F604001306062C97F5040080
:102380009385052813850700EF10935AEF305128E5
:102390009307F0FD232CF4FC6F00004397E7FF0147
:1023A0009387C7C603A7070083A7470013781700C2
:1023B00093F8070093070800B3E717016386070A3D
:1023C000EF3051239306100017F604001306062879
:1023D0009305A00217F5040013058533EF400111A2
:1023E00097E7FF01938707C283A707006388070267
:1023F0009797040083A7078A83A7070083A7C700CE
:10240000938607001306E0009305100017F50400FB
:1024100013054524EF30031A6F000002979704005C
:1024200083A7478783A7070083A7C7009385070073
:1024300013050002EF10535A9797040083A787856E
:1024400083A7070003A7C700832784FC83A7471A35
:102450001386070097F504009385C5201305070030
:10246000EF10134DEF30D11A832744FC639C070013
:10247000832744FC639A070E032704FC930730006C
:1024800063F4E70E97E7FF01938747B803A70700B8
:1024900083A74700B7160000337AD70093FA0700E6
:1024A00093070A00B3E75701638A070AEF309114D4
:1024B0009306300017F604001306460F9305D0026A
:1024C00017F504001305C524EF40410297E7FF010B
:1024D000938747B383A707006388070297870400A1
:1024E00083A7477B83A7070083A7C70093860700BE
:1024F0001306E0019305100017F504001305C51835
:10250000EF30430B6F00C0029787040083A78778E2
:1025100083A7070083A7C70093860700130610014F
:102520009305100017F5040013050518EF30830814
:102530009787040083A7077683A7070083A7C700B0
:10254000938607001306B0029305100017F50400E8
:102550001305C516EF300306EF30910B930720FEED
:10256000232CF4FC6F00402697E7FF01938707AA0E
:1025700003A6070083A6470093070600B3E7D7002A
:10258000639A07009787040083A7477083A7070013
:10259000638E0700832704FC93E727002320F4FCC5
:1025A000832744FC93E707002322F4FC232E04FC3A
:1025B0006F0000048327C4FC03A787008327C4FDA2
:1025C00093972700B307F70083A40700032584FC33
:1025D000EF10011A930705006396F40093071000AB
:1025E000232AF4FC8327C4FD93871700232EF4FCD1
:1025F0008327C4FC83A707010327C4FDE36CF7FA14
:10260000832744FD6394070E97E7FF01938707A094
:1026100003A7070083A74700B71600003379D70048
:1026200093F9070093070900B3E73701638A070AA4
:10263000EF30417C9306300017F60400130606F7CE
:102640009305900317F504001305850CEF30116A0C
:1026500097E7FF019387079B83A70700638807021B
:102660009787040083A7076383A7070083A7C70092
:10267000938607001306F0019305100017F5040078
:10268000130545F8EF2013736F00C002978704000D
:1026900083A7476083A7070083A7C7009386070027
:1026A000130620019305100017F50400130585F7A4
:1026B000EF2053709787040083A7C75D83A70700A7
:1026C00083A7C700938607001306500293051000E6
:1026D00017F5040013054501EF20D36DEF3041736A
:1026E0009307F0FD232CF4FC6F00000E130500038C
:1026F000EF30032D930705002328F4FC832704FD06
:10270000639807009307A0FF232CF4FC6F00C00B15
:10271000832704FD1307100023A2E700832704FD8D
:102720000327C4FC23A4E700832704FD032784FCBC
:1027300023A6E700832604FD032704FC832744FC2B
:1027400023A8E60023AAF600832704FD23AE070092
:10275000832704FD23AC0700832704FD23A0070281
:10276000832704FD23A20702832704FD23A4070275
:102770000325C4FCEFF0516E032584FCEFD0103E1E
:10278000232C04FC832784FC83A7472583A7C70346
:10279000638E0700832784FC83A7472583A7C7038D
:1027A000032504FDE7800700232CA4FC8327C4FB3A
:1027B000638807008327C4FB032784FD23A0E70069
:1027C000832704FD6F00C0018327C4FB63880700D3
:1027D0008327C4FB032784FD23A0E70093070000A1
:1027E000138507008320C10403248104832441044A
:1027F000032901048329C103032A8103832A410396
:102800001301010567800000130101FC232E110252
:10281000232C8102232A2103232831032326410369
:1028200023245103130401042326A4FC8326C4FC9F
:102830006392060E97D6FF019386467D03A6060097
:1028400083A64600B71500003377B60093F706005D
:1028500093060700B3E6F600638A060AEF30815953
:102860009306300017360500130646B29305E001C3
:1028700017350500130545C6EF30514797D7FF01BF
:102880009387477883A70700638807029787040028
:1028900083A7474083A7070083A7C7009386070045
:1028A000130660029305100017350500130585AE69
:1028B000EF2053506F00C0029787040083A7873D25
:1028C00083A7070083A7C70093860700130690011C
:1028D0009305100017350500130545AEEF20934D05
:1028E0009787040083A7073B83A7070083A7C70038
:1028F00017360500130646AE97350500938545AF9C
:1029000013850700EF10D302EF3081509307C0FD0D
:102910006F00002A8327C4FC83A78700232EF4FCC2
:102920008327C4FC83A7C700232CF4FC0325C4FC25
:10293000EFD0C0658327C4FC83A747006342F00241
:1029400097360500938606AB173605001306C6B802
:102950009305500217350500130505ACEF00D3456C
:102960008327C4FC83A747009387F7FF0327C4FC92
:102970002322F700232AF4FC8327C4FC83A7470003
:1029800063D2070297360500938646AB17360500DB
:10299000130686B493055002173505001305C5A725
:1029A000EF00934197D7FF019387476603A707007E
:1029B00083A74700137A070493FA070093070A00D6
:1029C000B3E757016384070AEF30C1429306100052
:1029D000173605001306C6A89305600217350500D3
:1029E000130585AFEF30913097D7FF01938787614B
:1029F00083A70700638807029787040083A78729B6
:102A000083A7070083A7C700938607001306E0008B
:102A10009305100017350500130545A5EF209339E0
:102A20006F0000029787040083A7C72683A70700CB
:102A300083A7C7009385070013050002EF10C37931
:102A40009787040083A7072583A7070083A7C700EC
:102A5000832644FD0326C4FC97350500938505A213
:102A600013850700EF10C36CEF30813A832744FDD4
:102A7000639E07128327C4FC83A7070263820702B1
:102A800097360500938686A1173605001306C6A45F
:102A90009305A0021735050013050598EF00D33103
:102AA00097D7FF019387875603A7070083A747009F
:102AB0001379070493F9070093070900B3E7370177
:102AC0006382070AEF3001339306100017360500C2
:102AD000130606999305B002173505001305C59F27
:102AE000EF30D12097D7FF019387C75183A7070005
:102AF000638807029787040083A7C71983A7070085
:102B000083A7C700938607001306E0009305100013
:102B10001735050013058595EF20D3296F000002B6
:102B20009787040083A7071783A7070083A7C70019
:102B30009385070013050002EF10036A97870400CE
:102B400083A7471583A7070083A7C7000326C4FCF4
:102B5000973505009385C59613850700EF10435DF3
:102B6000EF30012B8327C4FC83A7C70083A7472529
:102B700083A70704638E07008327C4FC83A7C700CD
:102B800083A7472583A707040325C4FCE780070024
:102B90000325C4FCEF20D363232604FC0325C4FDD6
:102BA000EFF04F87032584FDEFD0804493070000AA
:102BB000138507008320C1030324810303294103F4
:102BC00083290103032AC102832A8102130101041C
:102BD00067800000130101ED2326111223248112C6
:102BE0002322211323203113232E4111232C511191
:102BF000232A611123287111232681112324911185
:102C00002322A1112320B111130401132326A4FAB6
:102C10002320B4FA2322C4FA2324D4FA232EE4F87E
:102C2000232CF4F8232604FC832784FA6394070EEC
:102C300097D7FF019387873D03A7070083A7470026
:102C4000B71600003378D70093F807009307080001
:102C5000B3E71701638A070AEF30C1199306300002
:102C6000176605001306862F9305A0021775050049
:102C700013054584EF30910797D7FF019387873875
:102C800083A70700638807029787040083A787004C
:102C900083A7070083A7C700938607001306400297
:102CA00093051000176505001305C52BEF20931041
:102CB0006F00C0029787040083A7C7FD83A70700A2
:102CC00083A7C700938607001306700193051000C1
:102CD000176505001305852BEF20D30D978704009A
:102CE00083A747FB83A7070083A7C70017660500D4
:102CF0001306462B976505009385852B13850700E2
:102D0000EF100343EF30C110930730FC2324F4FC91
:102D10006F1000288327C4FA6394070E97D7FF012A
:102D20009387C72E03A7070083A74700B7160000A5
:102D30003373D70093F3070093070300B3E77700DB
:102D4000638A070AEF30010B93063000176605000F
:102D50001306C6209305C002176505001305857587
:102D6000EF30C17897D7FF019387C72983A7070062
:102D7000638807029787040083A7C7F183A707002A
:102D800083A7C7009386070013060002930510006F
:102D90001765050013050522EF20D3016F00C0025F
:102DA0009787040083A707EF83A7070083A7C700BF
:102DB0009386070013063001930510001765050080
:102DC00013058521EF20037F9787040083A787ECF5
:102DD00083A7070083A7C70017660500130606210F
:102DE000976505009385C51C13850700EF104334D4
:102DF000EF3001029307E0FD2324F4FC6F1040192B
:102E000013050009EF20D33B930705002326F4FCAC
:102E10008327C4FC639807009307A0FF2324F4FCD6
:102E20006F1000178327C4FC23A60702032704FAA8
:102E3000832744FA3367F700631A0700130710006B
:102E4000930700002320E4FA2322F4FA832744FAAC
:102E5000639C0700832744FA639A070E032704FA4A
:102E60009307F03F63F4E70E97D7FF019387071AA4
:102E700003A7070083A74700B71600003379D700E0
:102E800093F9070093070900B3E73701638A070A3C
:102E9000EF20517693063000176605001306060CE6
:102EA0009305B003176505001305C560EF30016495
:102EB00097D7FF019387071583A707006388070249
:102EC0009787040083A707DD83A7070083A7C700B0
:102ED000938607001306E0019305100017650500AF
:102EE00013050512EF20036D6F00C00297870400E1
:102EF00083A747DA83A7070083A7C7009386070045
:102F00001306100193051000176505001305451100
:102F1000EF20436A9787040083A7C7D783A70700DA
:102F200083A7C700938607001306F00293051000DD
:102F30001765050013050510EF20C367EF20516DDD
:102F4000930720FE2324F4FC6F108004832704FAE7
:102F500013FA1700832744FA93FA070093070A002D
:102F6000B3E7570163800712832704FA13FB270096
:102F7000832744FA93FB070093070B00B3E777011D
:102F800063900702832704FA13FD4700832744FA5E
:102F900093FD070093070D00B3E7B7016384070EA5
:102FA00097D7FF019387870603A7070083A74700EA
:102FB000B7160000337CD70093FC070093070C0082
:102FC000B3E79701638A070AEF20D16293063000C6
:102FD00017660500130686F89305E00317650500DC
:102FE0001305454DEF30815097D7FF019387870137
:102FF00083A70700638807029787040083A787C910
:1030000083A7070083A7C700938607001306E00184
:103010009305100017650500130585FEEF20835901
:103020006F00C0029787040083A7C7C683A7070065
:1030300083A7C700938607001306100193051000AD
:10304000176505001305C5FDEF20C35697870400DB
:1030500083A747C483A7070083A7C70093860700F9
:10306000130640069305100017650500130585FF3C
:10307000EF204354EF20D159930720FE2324F4FC82
:103080006F001071832704FA93F747002328F4F8A0
:10309000832744FA93F70700232AF4F8832604F9D8
:1030A000032744F993870600B3E7E700638207121A
:1030B000832704FA93F727002324F4F8832744FA9C
:1030C00093F707002326F4F8832684F80327C4F82F
:1030D00093870600B3E7E700638C070E97D7FF01DD
:1030E0009387C7F203A7070083A74700B71600001E
:1030F000B376D7002320D4F893F707002322F4F8FF
:10310000832604F8032744F893870600B3E7E70013
:10311000638A070AEF20114E9306300017660500F8
:103120001306C6E3930530041765050013058538BB
:10313000EF30C13B97D7FF019387C7EC83A7070008
:10314000638807029787040083A7C7B483A7070093
:1031500083A7C700938607001306E00193051000BC
:10316000176505001305C5E9EF20C3446F00C002D1
:103170009787040083A707B283A7070083A7C70028
:1031800093860700130610019305100017650500CC
:10319000130505E9EF2003429787040083A787AF53
:1031A00083A7070083A7C700938607001306600460
:1031B0009305100017650500130545F1EF20833FC7
:1031C000EF201145930720FE2324F4FC6F00505C90
:1031D000832704FA93F78700232CF4F6832744FA15
:1031E00093F70700232EF4F6832684F70327C4F70A
:1031F00093870600B3E7E70063880714832704FA80
:1032000093F707012328F4F6832744FA93F707007E
:10321000232AF4F6832604F7032744F7938706004E
:10322000B3E7E70063980702832704FA93F70702DE
:103230002324F4F6832744FA93F707002326F4F6B1
:10324000832684F60327C4F693870600B3E7E700D6
:10325000638C070E97D7FF01938747DB03A707000F
:1032600083A74700B7160000B376D7002320D4F613
:1032700093F707002322F4F6832604F6032744F687
:1032800093870600B3E7E700638A070AEF209136C9
:103290009306300017660500130646CC93057004AC
:1032A0001765050013050521EF30412497D7FF016D
:1032B000938747D583A70700638807029787040091
:1032C00083A7479D83A7070083A7C70093860700AE
:1032D0001306E0019305100017650500130545D29C
:1032E000EF20432D6F00C0029787040083A7879AC1
:1032F00083A7070083A7C700938607001306100162
:103300009305100017650500130585D1EF20832A6A
:103310009787040083A7079883A7070083A7C700A0
:10332000938607001306E006930510001765050055
:10333000130545DEEF200328EF20912D930720FE93
:103340002324F4FC6F00D044832704FA93F7070882
:10335000232CF4F4832744FA93F70700232EF4F484
:10336000832684F50327C4F593870600B3E7E700B7
:1033700063820712832704FA93F707102328F4F4D3
:10338000832744FA93F70700232AF4F4832604F5ED
:10339000032744F593870600B3E7E700638C070E25
:1033A00097D7FF01938787C603A7070083A7470026
:1033B000B7160000B376D7002324D4F493F70700A0
:1033C0002326F4F4832684F40327C4F493870600A9
:1033D000B3E7E700638A070AEF20D12193063000A4
:1033E00017660500130686B79305C0041765050028
:1033F0001305450CEF30810F97D7FF01938787C0E6
:1034000083A70700638807029787040083A787883C
:1034100083A7070083A7C700938607001306E00170
:103420009305100017650500130585BDEF2083186F
:103430006F00C0029787040083A7C78583A7070092
:1034400083A7C70093860700130610019305100099
:10345000176505001305C5BCEF20C3159787040049
:1034600083A7478383A7070083A7C7009386070026
:10347000130600059305100017650500130585D098
:10348000EF204313EF20D118930720FE2324F4FCF0
:103490006F001030832704FA93F707202320F4F4F9
:1034A000832744FA93F707002322F4F4832604F4D5
:1034B000032744F493870600B3E7E7006388071403
:1034C000832704FA93F70710232CF4F2832744FA96
:1034D00093F70700232EF4F2832684F30327C4F323
:1034E00093870600B3E7E70063980702832704FA8F
:1034F00093F707082328F4F2832744FA93F7070089
:10350000232AF4F2832604F3032744F39387060067
:10351000B3E7E700638C070E97D7FF01938707AFE8
:1035200003A7070083A74700B7160000B376D700AC
:103530002324D4F293F707002326F4F2832684F29F
:103540000327C4F293870600B3E7E700638A070AFC
:10355000EF20510A9306300017660500130606A0F7
:1035600093050005176505001305C5F4EF201178D4
:1035700097D7FF01938707A983A7070063880702EE
:103580009777040083A7077183A7070083A7C70065
:10359000938607001306E0019305100017650500E8
:1035A000130505A6EF2003016F00C0029777040002
:1035B00083A7476E83A7070083A7C70093860700EA
:1035C000130610019305100017650500130545A5A6
:1035D000EF10537E9777040083A7C76B83A707007C
:1035E00083A7C700938607001306200793051000E2
:1035F00017650500130545BEEF10D37BEF20510181
:10360000930720FE2324F4FC6F0090188327C4F94D
:1036100063980714832704FA93F787002320F4F2B2
:10362000832744FA93F707002322F4F2832604F257
:10363000032744F293870600B3E7E7006398070285
:10364000832704FA93F70702232CF4F0832744FA24
:1036500093F70700232EF4F0832684F10327C4F1A7
:1036600093870600B3E7E7006382072497D7FF013B
:103670009387C79903A7070083A74700B7160000E1
:10368000B376D7002328D4F093F70700232AF4F069
:10369000832604F1032744F193870600B3E7E7008C
:1036A000638A070AEF20017593063000176605004C
:1036B0001306C68A9305700517650500130585DF97
:1036C000EF20D16297D7FF019387C79383A70700A5
:1036D000638807029777040083A7C75B83A7070067
:1036E00083A7C700938607001306100293051000F6
:1036F00017650500130585B5EF10D36B6F00C00289
:103700009777040083A7075983A7070083A7C700FB
:103710009386070013064001930510001765050006
:10372000130505B5EF1013699777040083A7875633
:1037300083A7070083A7C7009386070013068003AB
:103740009305100017650500130505B4EF10936687
:10375000EF20016C9307B0FD2324F4FC6F005003AD
:10376000832704FA93F787002324F4F0832744FA8D
:1037700093F707002326F4F0832684F00327C4F090
:1037800093870600B3E7E70063920712832704FAE2
:1037900093F707022320F4F0832744FA93F70700F6
:1037A0002322F4F0832604F0032744F093870600D5
:1037B000B3E7E700639C070E97D7FF019387078560
:1037C00003A7070083A74700B7160000B376D7000A
:1037D000232CD4EE93F70700232EF4EE832684EFF8
:1037E0000327C4EF93870600B3E7E700638A070A5D
:1037F000EF20416093063000175605001306067649
:103800009305D005176505001305C5CAEF20114EB5
:1038100097C7FF019387077F83A707006388070285
:103820009777040083A7074783A7070083A7C700EC
:103830009386070013061002930510001765050014
:103840001305C5A0EF1013576F00C002977704004F
:1038500083A7474483A7070083A7C7009386070071
:10386000130640019305100017650500130545A0D8
:10387000EF1053549777040083A7C74183A707002D
:1038800083A7C70093860700130620049305100042
:1038900017650500130505A3EF10D351EF2041571D
:1038A0009307B0FD2324F4FC6F00806E8327C4FAD5
:1038B00083A7C701032784FA63F0E71097C7FF01C6
:1038C0009387C77403A7070083A74700B7160000B4
:1038D000B376D7002328D4EE93F70700232AF4EE1B
:1038E000832604EF032744EF93870600B3E7E7003E
:1038F000638E070AEF20015093063000175605002B
:103900001306C6659305200617650500130585BADD
:10391000EF20D13D97C7FF019387C76E83A70700AC
:10392000638807029777040083A7C73683A7070039
:1039300083A7C70093860700130640029305100073
:103940001755050013050562EF10D3466F00C0023E
:103950009777040083A7073483A7070083A7C700CE
:103960009386070013067001930510001755050094
:103970001305C561EF1013449777040083A78731BF
:1039800083A7070003A7C7008327C4FA83A7C7013B
:1039900093860700032684FA976505009385C596EC
:1039A00013050700EF00C378EF208146930730FC32
:1039B0002324F4FC6F00C05D8327C4FC13071000B0
:1039C00023A2E7008327C4FC23AE07028327C4FC9D
:1039D00023A207028327C4FC23AC07028327C4FC6D
:1039E00023AE07068327C4FC23A007048327C4FC57
:1039F000371700001307070F23A4E7008326C4FC32
:103A0000032704FA832744FA23A8E60023AAF60032
:103A10008327C4FC23A407048327C4FC23AA07022A
:103A20008327C4FC23A007088327C4FC23A207081C
:103A30008327C4FC23A4070897D70C00938787CF5C
:103A400083A707009305000113850700EFF052409C
:103A500093070500138707008327C4FC23A6E7020A
:103A60008327C4FC83A7C702639C070E97C7FF0187
:103A70009387C75903A7070083A74700B71600001D
:103A8000B376D7002324D4EE93F707002326F4EE71
:103A9000832684EE0327C4EE93870600B3E7E7008E
:103AA000638A070AEF200135930630001756050098
:103AB0001306C64A9305C007176505001305859FC1
:103AC000EF20D12297C7FF019387C75383A7070031
:103AD000638807029777040083A7C71B83A70700A3
:103AE00083A7C700938607001306300293051000D2
:103AF0001765050013054586EF10D32B6F00C00234
:103B00009777040083A7071983A7070083A7C70037
:103B100093860700130660019305100017650500E2
:103B20001305C585EF1013299777040083A787161F
:103B300083A7070083A7C7001766050013068685BD
:103B4000975505009385C54613850700EF00435E32
:103B5000EF20012C9307A0FF2324F4FC6F004043C7
:103B6000232204FC6F0000088327C4FA03A7870000
:103B7000832744FC93972700B307F70083A7070028
:103B800083A7471A232CF4FA8327C4FA03A78700D4
:103B9000832744FC93972700B307F70003A7070088
:103BA0008327C4FC83A6C702832784FB939747001F
:103BB000B387F6000327871A23A2E7008327C4FCF4
:103BC00003A7C702832744FC93974700B307F70076
:103BD0001307100023A0E700832744FC93871700F6
:103BE0002322F4FC8327C4FA83A70701032744FC9C
:103BF000E36CF7F68327C4FC032784FA23ACE700C1
:103C00008327C4FC23AE07008327C4FC0327C4FA20
:103C100023A4E7028327C4FC0327C4F923A0E702F7
:103C20008327C4FC23A807028327C4FA83A70705B8
:103C3000638007048327C4FA83A7070583A7472562
:103C400003A747048327C4FA83A707050326C4F9FB
:103C50008325C4FC13850700E700070093070500D0
:103C6000638807009307C0FF2324F4FC6F00C02C77
:103C7000232204FC6F00400B8327C4FA03A7070527
:103C80008327C4FA83A68700832744FC93972700E1
:103C9000B387F60083A707006300F7088327C4FAF9
:103CA00003A78700832744FC93972700B307F700F7
:103CB00083A70700232EF4FA8327C4FB83A7472595
:103CC00083A7470463920702975605009386466EC2
:103CD000175605001306067E9305100A17550500B2
:103CE0001305456FEFF0520D8327C4FB83A74725CB
:103CF00083A747040326C4F98325C4FC0325C4FB1A
:103D0000E780070093070500638A07009307C0FF59
:103D10002324F4FC6F00402213000000832744FC9E
:103D2000938717002322F4FC8327C4FA83A7070193
:103D3000032744FCE362F7F4832704FA93F70701AF
:103D40002320F4EE832744FA93F707002322F4EEAE
:103D5000832604EE032744EE93870600B3E7E700CB
:103D6000638607068327C4FC83A7070263900706C0
:103D70008327C4FC83A707036382070297560500C5
:103D800093860667175605001306C6729305C00A88
:103D90001755050013050564EFF01202832584FA18
:103DA00013050008EFC0D035130705008327C4FCB6
:103DB00023A0E7028327C4FC83A7070263980700B8
:103DC0009307A0FF2324F4FC6F0000178327C4FA95
:103DD00083A747006342F002975605009386066466
:103DE000175605001306066D9305500B1755050071
:103DF0001305455EEFF0427C8327C4FA83A7470092
:103E0000138717008327C4FA23A2E7008327C4FA85
:103E100083A7470063D20702975605009386066280
:103E200017560500130606699305500B1755050034
:103E30001305455AEFF0427897C7FF019387071D96
:103E400003A7070083A7470093762700232CD4EC11
:103E500093F70700232EF4EC832684ED0327C4EDAB
:103E600093870600B3E7E700638C070AEF109178A9
:103E700093061000175605001306465E9305700B57
:103E80001755050013050563EF20416697C7FF012D
:103E90009387471783A70700638807029777040073
:103EA00083A747DF83A7070083A7C7009386070080
:103EB0001306E00093051000175505001305855AF9
:103EC000EF10436F6F0000029777040083A787DC31
:103ED00083A7070083A7C700938507001305000287
:103EE000EF00832F9777040083A7C7DA83A7070023
:103EF00003A5C7008327C4FC83A607028327C4FC4D
:103F000083A7C70203A78700832784FA0326C4FC7C
:103F10009755050093850556EF008321EF10516FEB
:103F2000832784F963860700832784F923A0070089
:103F30008327C4FC6F00000A232004FC6F004004A8
:103F40008327C4FA03A78700832704FC93972700DD
:103F5000B307F70083A70700232EF4FA8327C4FBD7
:103F600083A7472583A787048325C4FC0325C4FBB7
:103F7000E7800700832704FC938717002320F4FCC5
:103F8000032704FC832744FCE36CF7FA13000000CA
:103F90008327C4FC638E07008327C4FC83A7C70262
:103FA00013850700EF10D3228327C4FC23A6070242
:103FB0000325C4FCEF10D321232604FC832784F9B6
:103FC00063880700832784F9032784FC23A0E70084
:103FD00093070000138507008320C1120324811278
:103FE0000329411283290112032AC111832A811155
:103FF000032B4111832B0111032CC110832C811041
:10400000032D4110832D011013010113678000005F
:10401000130101F9232611062324810623222107F7
:1040200023203107232E4105232C5105232A610526
:104030002328710523268105232491052322A10528
:104040002320B10513040107232EA4FA232CB4FA6C
:10405000232AC4FA2328D4FA2326E4FA2324F4FAE0
:10406000232204FB232014FB232004FC8327C4FB0E
:104070006392070E97C7FF01938747F903A70700CD
:1040800083A74700B7160000337DD70093FD0700D4
:1040900093070D00B3E7B701638A070AEF10915544
:1040A0009306300017960500130606579305D002B5
:1040B00017A505001305C589EF20414397C7FF01E8
:1040C000938747F483A70700638807029777040064
:1040D00083A747BC83A7070083A7C7009386070071
:1040E000130660029305100017950500130545534C
:1040F000EF10434C6F00C0029777040083A787B985
:1041000083A7070083A7C7009386070013069001C3
:10411000930510001795050013050553EF1083490B
:104120009777040083A707B783A7070083A7C70073
:1041300017960500130606539795050093850554B9
:1041400013850700EFF0D27EEF10914C9307C0FD6E
:104150006F00007D832784FB6392070E97C7FF01E2
:104160009387C7EA03A7070083A74700B716000095
:10417000337CD70093FC070093070C00B3E797014B
:10418000638A070AEF10114793063000179605005F
:10419000130686489305F002179505001305457B25
:1041A000EF20C13497C7FF019387C7E583A70700B6
:1041B000638807029777040083A7C7AD83A707002A
:1041C00083A7C700938607001306300293051000EB
:1041D000179505001305C54AEF10C33D6F00C002D7
:1041E0009777040083A707AB83A7070083A7C700BF
:1041F00093860700130660019305100017950500CC
:104200001305454AEF10033B9777040083A787A85F
:1042100083A7070083A7C700179605001306064A61
:10422000979505009385854513850700EFF052703B
:10423000EF10113E9307A0FD6F00806E832784FB73
:1042400083A7C70363800710832784FB03A7C701E5
:104250008327C4FB83A7C70083A7C70BB377F702E5
:104260006382070E97C7FF01938747DA03A707000A
:1042700083A74700B7160000337BD70093FB0700E6
:1042800093070B00B3E77701638A070AEF109136B3
:1042900093063000179605001306063893051003A1
:1042A000179505001305C56AEF20412497C7FF0144
:1042B000938747D583A70700638807029777040091
:1042C00083A7479D83A7070083A7C700938607009E
:1042D0001306D00293051000179505001305453FFE
:1042E000EF10432D6F00C0029777040083A7879AD1
:1042F00083A7070083A7C700938607001306000261
:1043000093051000179505001305853FEF10832ACC
:104310009777040083A7079883A7070083A7C700A0
:1043200093860700130610039305100017950500E8
:104330001305453FEF100328EF10912D930730FF31
:104340006F00005E8327C4FB03A78700832784FBDD
:1043500083A787026302F70E97C7FF01938707CBF6
:1043600003A7070083A74700B7160000337AD700DA
:1043700093FA070093070A00B3E75701638A070A15
:10438000EF10512793063000179605001306C62834
:1043900093053003179505001305855BEF20011584
:1043A00097C7FF01938707C683A7070063880702A3
:1043B0009777040083A7078E83A7070083A7C7000A
:1043C0009386070013060002930510001795050059
:1043D00013058538EF10031E6F00C00297770400A5
:1043E00083A7478B83A7070083A7C700938607008F
:1043F00013063001930510001795050013050538C5
:10440000EF10431B9777040083A7C78883A7070093
:1044100083A7C70093860700130670039305100057
:10442000179505001305C536EF10C318EF10511E80
:104430009307E0FD6F00C04E832784FB03A70701AD
:1044400083A74701137F072893FF070093070F00F7
:10445000B3E7F7016382070E97C7FF01938707BB96
:1044600003A7070083A74700B7160000337ED700D5
:1044700093FE070093070E00B3E7D701638A070A8C
:10448000EF10511793063000179605001306C61853
:1044900093056003179505001305854BEF20010573
:1044A00097C7FF01938707B683A7070063880702B2
:1044B0009767040083A7077E83A7070083A7C70029
:1044C0009386070013062002930510001795050038
:1044D0001305852FEF10030E6F00C00297670400CD
:1044E00083A7477B83A7070083A7C700938607009E
:1044F0001306500193051000179505001305052FAD
:10450000EF10430B9767040083A7C77883A70700C2
:1045100083A7C700938607001306D00493051000F5
:10452000179505001305052EEF10C308EF10510E67
:10453000930750FC6F00C03E832784FA6392070EF6
:1045400097C7FF01938787AC03A7070083A747009E
:10455000B71600003373D70093F3070093070300E7
:10456000B3E77700638A070AEF10D108930630009B
:10457000179605001306460A9305C0031795050014
:104580001305053DEF10917697C7FF01938787A725
:1045900083A70700638807029767040083A7876FD4
:1045A00083A7070083A7C700938607001306E001CF
:1045B00093051000179505001305C529EF00937F9B
:1045C0006F00C0029767040083A7C76C83A707002A
:1045D00083A7C700938607001306100193051000F8
:1045E0001795050013050529EF00D37C9767040094
:1045F00083A7476A83A7070083A7C700179605000C
:1046000013068628979505009385450713850700AF
:10461000EFF01232EF10C17F930720FE6F004030A1
:10462000832784FB0326C4FA832504FB1385070034
:10463000EFD0807E9307050063860700930720FE76
:104640006F00002E832784FB83A7C70363820702C2
:10465000832784FB83A7C701032704FBB307F70065
:104660002328F4FA832784FB83A7C703232CF4FAB7
:10467000832784FB83A78701232CF4F8232E04F8D7
:104680008327C4FB83A7C70003A7070883A747089E
:10469000032584F98325C4F9138605009386070052
:1046A00063EEC60013860500938607006318D60ED6
:1046B000930605009307070063F2D70E97C7FF0123
:1046C0009387C79403A7070083A74700B716000086
:1046D0003379D70093F9070093070900B3E737014F
:1046E000638A070AEF1001719306300017960500E0
:1046F000130686F29305300417950500130545252A
:10470000EF10D15E97C7FF019387C78F83A707007C
:10471000638807029767040083A7C75783A707002A
:1047200083A7C700938607001306100293051000A5
:104730001795050013054516EF00D3676F00C002FB
:104740009767040083A7075583A7070083A7C700BF
:104750009386070013064001930510001795050086
:104760001305C515EF0013659767040083A78752EB
:1047700083A7070083A7C7009386070013062003BB
:1047800093051000179505001305C514EF009362FB
:10479000EF1001689307B0FF6F008018032604FA3A
:1047A000832544FA0325C4FBEFF0806C2324A4FC8A
:1047B000832784FC63860700832784FC6F004016F0
:1047C0008327C4FB83A7C70013850700EFE0507A57
:1047D0002322A4FC232604FC6F0040038327C4FB90
:1047E00083A7870003A787008327C4FC939727002C
:1047F000B307F70083A70700032744FC6304F7020D
:104800008327C4FC938717002326F4FC8327C4FB6B
:1048100083A7870083A707010327C4FCE360F7FC95
:104820006F008000130000008327C4FB83A787006C
:1048300083A707010327C4FC6362F702979605006C
:104840009386860C17960500130686109305C00400
:10485000179505001305C50DEFE01256032744FA1E
:10486000930784FB130504FC9388070013081000CA
:10487000832704FA83260400371600001306361F28
:104880008325C4FBEFC0100A2324A4FC832784FCE7
:1048900063860700832784FC6F008008832704FC5D
:1048A000032784FA23A0E700832784FB83A6C7029B
:1048B000832744FC83A7471A13974700832704FCE8
:1048C0003387E60023A2E700832704FC032704FBC9
:1048D00023A4E700832704FC0327C4FA23A6E700E8
:1048E000832784FB13850700EF00406B832784FB3D
:1048F0000327C4FB0327C70023AAE702832704FC7E
:10490000938507000325C4FBEFC0D04D832744FBEC
:10491000638607000325C4FBEFB0C0619307000066
:10492000138507008320C10603248106032941065D
:1049300083290106032AC105832A8105032B41052A
:10494000832B0105032CC104832C8104032D410416
:10495000832D01041301010767800000130101FA90
:10496000232E1104232C8104232A21052328310519
:104970002326410523245105130401062326A4FA06
:10498000232804FC8325C4FA6392050E97B7FF0120
:104990009387C76703A7070083A74700B7150000E1
:1049A0003376B70093F6070093070600B3E7D70006
:1049B000638A070AEF1001449306300017D60500FA
:1049C000130606CB9305500217D50500130585DAAB
:1049D000EF10D13197B7FF019387C76283A7070014
:1049E000638807029767040083A7C72A83A7070085
:1049F00083A7C700938607001306300293051000B3
:104A000017D50500130545C7EF00D33A6F00C00264
:104A10009767040083A7072883A7070083A7C70019
:104A200093860700130660019305100017D5050053
:104A30001305C5C6EF0013389767040083A78725C1
:104A400083A7070083A7C70017D60500130686C6ED
:104A500097D50500938545C713850700EFF0426D94
:104A6000EF10013B9307A0FD6F0000518326C4FAAD
:104A700083A686022326D4FC8326C4FA83A6460096
:104A80006342D00297D60500938646C417D6050028
:104A9000130646CE9305900217D505001305C5C42D
:104AA000EFE092318326C4FA83A646009386F6FF90
:104AB0000326C4FA2322D6002324D4FC8326C4FA76
:104AC00083A6460063D2060297D605009386C6C326
:104AD00017D60500130606CA9305900217D50500E0
:104AE000130585C0EFE0522D97B6FF01938606525D
:104AF00003A6060083A646001377060493F7060074
:104B000093060700B3E6F6006384060AEF10812ED1
:104B10009306100017D60500130606C19305B002D0
:104B200017D50500130505C5EF10511C97B7FF01F8
:104B30009387474D83A707006388070297670400A0
:104B400083A7471583A7070083A7C700938607009D
:104B50001306E0009305100017D50500130585BD69
:104B6000EF0053256F0000029767040083A78712A8
:104B700083A7070083A7C7009385070013050002DA
:104B8000EFF082659767040083A7C71083A707002B
:104B900083A7C700832684FC0326C4FA97D50500A3
:104BA000938545BA13850700EFF08258EF10412630
:104BB000832784FC6390073C8327C4FA83A7870478
:104BC000638607068327C4FA03A78700B717000088
:104BD0009387670F631CF7048327C4FA83A7C7076B
:104BE0002322F4FC832744FC6392070297D6050036
:104BF0009386C6B617D605001306C6B79305A0035D
:104C000017D50500130545AEEFE0121B032544FC44
:104C1000EFF0DFD42320A4FC0325C4FAEF00535B9C
:104C2000232604FA832704FC6F00003597B7FF01A1
:104C30009387C73D03A7070083A74700137A07049C
:104C400093FA070093070A00B3E757016382070A44
:104C5000EF10411A9306100017D605001306C6ACD4
:104C60009305000417D505001305C5B0EF10110812
:104C700097B7FF019387073983A707006388070267
:104C80009767040083A7070183A7070083A7C700CE
:104C9000938607001306E0009305100017D5050062
:104CA000130545A9EF0013116F0000029767040078
:104CB00083A747FE83A7070083A7C7009385070044
:104CC00013050002EFF042519767040083A787FCA9
:104CD00083A7070083A7C7000326C4FA97D505005A
:104CE000938505A813850700EFF08244EF10411269
:104CF0008327C4FA83A7C703639607128327C4FADE
:104D000083A70703232EF4FA232E04FC6F00800EE2
:104D10008327C4FC03A787008327C4FD939727003C
:104D2000B307F70083A707000327C4FB630CF70A48
:104D30008327C4FC03A787008327C4FD939727001C
:104D4000B307F70083A70700232CF4FA8327C4FADC
:104D500083A78704638C0704832784FB83A78708C2
:104D600063860704832784FB83A7472583A7470A15
:104D7000638E0702832784FB83A7472583A6470A00
:104D80008327C4FA03A7C702832784FB83A7471A94
:104D900093974700B307F70083A7C7001386070060
:104DA0008325C4FA032584FBE7800600832784FB60
:104DB00083A7472583A787048325C4FA032584FB9B
:104DC000E78007008327C4FA03A7C702832784FB71
:104DD00083A7471A93974700B307F70023A4070058
:104DE0006F008000130000008327C4FD9387170025
:104DF000232EF4FC8327C4FC83A707010327C4FDEB
:104E0000E368F7F08327C4FB638E07008327C4FBA6
:104E100083A7472583A787048325C4FA0325C4FBFA
:104E2000E78007008327C4FA83A78703232CF4FCB9
:104E30006F008001032584FDEF009339232C04FCCF
:104E4000832704FB232CF4FC832784FD638A07005B
:104E5000832784FD83A707012328F4FA6FF09FFDC1
:104E60008327C4FA23AC07028327C4FA83A7C703A6
:104E70002328F4FC8327C4FA83A7C7036394070499
:104E80008327C4FA03A7070183A747011379070102
:104E900093F9070093070900B3E73701638407021A
:104EA0008327C4FA83A70702638E07008327C4FA07
:104EB00083A7070213850700EF0093318327C4FA05
:104EC00023A007028327C4FA83A7C702138507001C
:104ED000EF0013308327C4FA23A607028327C4FAFE
:104EE00083A70704232AF4FC6F00C003832744FD33
:104EF00003A70700832744FD83A747009385070086
:104F00000325C4FAE7000700832744FD83A7870031
:104F1000232AF4FA032544FDEF00932B832744FB57
:104F2000232AF4FC832744FDE39207FC8327C4FA79
:104F300083A78704638E07008327C4FA83A74704E7
:104F400013850700EF00D3288327C4FA23A20704A0
:104F50000325C4FAEF00D327232604FA832704FD90
:104F600063860700032504FDEFF05F9F0325C4FC63
:104F7000EFC05FCA93070000138507008320C105B7
:104F8000032481050329410583290105032AC1045E
:104F9000832A81041301010667800000130101FECA
:104FA000232E1100232C8100130401022326A4FECA
:104FB0008325C4FE6392050E97B7FF01938707050B
:104FC00003A7070083A74700B71500003376B70093
:104FD00093F6070093070600B3E7D700638A070A32
:104FE000EF00516193063000170606001306865441
:104FF0009305D0011705060013058562EF10014FD8
:1050000097B7FF019387070083A70700638807020C
:105010009767040083A707C883A7070083A7C70073
:10502000938607001306300293051000170506004B
:105030001305C550EF0003586F00C00297670400C6
:1050400083A747C583A7070083A7C70093860700E8
:10505000130660019305100017050600130545505F
:10506000EF0043559767040083A7C7C283A70700D3
:1050700083A7C7001706060013060650970506000B
:105080009385C55013850700EFF0820AEF00515851
:105090009307A0FD6F0040148326C4FE83A646003C
:1050A0006342D002970606009386864E17060600D6
:1050B000130606579305E001170506001305054F73
:1050C000EFE0824F8326C4FE83A6460013861600B7
:1050D0008326C4FE23A2C6008326C4FE83A6460000
:1050E00063D20602970606009386464E1706060010
:1050F000130606539305E001170506001305054B3B
:10510000EFE0824B97B6FF01938646F003A60600B8
:1051100083A646001377060493F70600930607005C
:10512000B3E6F6006388060AEF00D14C9306100040
:10513000170606001306864B9305F00117050600B7
:105140001305054EEF10813A97B7FF01938787EB60
:1051500083A70700638807029767040083A787B3C4
:1051600083A7070083A7C700938607001306E00004
:10517000930510001705060013050548EF0083434B
:105180006F0000029767040083A7C7B083A70700DA
:1051900083A7C7009385070013050002EFF0C20341
:1051A0009767040083A707AF83A7070003A7C7007B
:1051B0008327C4FE83A74700938607000326C4FE07
:1051C000970506009385454413050700EFE05276E6
:1051D000EF00114493070000138507008320C101ED
:1051E000032481011301010267800000130101F90A
:1051F000232611062324810623229106232021073A
:10520000232E3105232C4105232A510513040107C0
:105210002326A4FA2324B4FA2322C4FA2320D4FA9E
:10522000232EE4F8232E04FC232004FC232C04FC6E
:10523000232A04FC832704FA6394070E97B7FF011F
:105240009387C7DC03A7070083A74700B7160000B2
:105250003378D70093F8070093070800B3E71701E6
:10526000638A070AEF0011399306300017460600DB
:10527000130686D29305F002174506001305C5E014
:10528000EF10C12697B7FF019387C7D783A7070001
:10529000638807029767040083A7C79F83A7070057
:1052A00083A7C700938607001306E001930510004B
:1052B000174506001305C5CEEF00C32F6F00C002CF
:1052C0009767040083A7079D83A7070083A7C700EC
:1052D000938607001306100193051000174506007A
:1052E000130505CEEF00032D9767040083A7879A67
:1052F00083A7070083A7C70017460600130686CDBD
:1053000097450600938585CE13850700EFE052622E
:10531000EF001130930720FE232CF4FA6F00C03DFC
:10532000032504FAEF30C31B93070500232EF4FC7A
:10533000930744FB1386070097450600938545CBEA
:105340000325C4FDEF3053782328A4FC6F00001A16
:10535000232604FC232404FC6F004007832784FCDD
:1053600093972700032744FAB307F70083A70700A2
:10537000232EF4FA8327C4FB83A7472583A7870C32
:10538000638E07028327C4FB83A7472503A7870CE7
:105390008327C4FB83A78719832504FD1385070092
:1053A000E700070093070500638C07008327C4FC10
:1053B000938717002326F4FC6F0080001300000081
:1053C000832784FC938717002324F4FC032784FCA1
:1053D000832784FAE364F7F88327C4FC6394070EF9
:1053E00097B7FF01938787C203A7070083A74700EA
:1053F000B7160000337AD70093FA070093070A0024
:10540000B3E75701638A070AEF00D11E9306300005
:1054100017460600130646B89305F0031745060025
:10542000130585C6EF10810C97B7FF01938787BDE1
:1054300083A70700638807029767040083A787850F
:1054400083A7070083A7C700938607001306E00120
:105450009305100017450600130585B4EF0083156A
:105460006F00C0029767040083A7C78283A7070065
:1054700083A7C70093860700130610019305100049
:10548000174506001305C5B3EF00C3129767040064
:1054900083A7478083A7070083A7C70093860700D9
:1054A0001306D0039305100017450600130585B4B5
:1054B000EF004310EF00D115930720FE232CF4FAE0
:1054C0006F008023832744FD93871700232AF4FC71
:1054D000930744FB1386070097450600938545B163
:1054E00013050000EF30535E2328A4FC832704FD3E
:1054F000E39007E60325C4FDEF00834D232E04FC53
:1055000093054000032544FDEFE082149307050056
:10551000232CF4FC832784FD6394070E97B7FF01C7
:105520009387C7AE03A7070083A74700B7160000FD
:105530003379D70093F9070093070900B3E73701E0
:10554000638A070AEF00110B930630001746060026
:10555000130686A493058004174506001305C5B2FB
:10556000EF00D17897B7FF019387C7A983A70700FA
:10557000638807029757040083A7C77183A70700B2
:1055800083A7C70093860700130630029305100017
:1055900017450600130505AAEF00C3016F00C002FE
:1055A0009757040083A7076F83A7070083A7C70047
:1055B0009386070013066001930510001745060047
:1055C000130585A9EFF0127F9757040083A7876C16
:1055D00083A7070083A7C70017460600130646A93E
:1055E00097450600938585A013850700EFE05234A8
:1055F000EF0011029307A0FF232CF4FA6F00C00FF5
:10560000032504FAEF20D36D93070500232EF4FC45
:10561000930744FB13860700974506009385459D35
:105620000325C4FDEF30534A2328A4FC232204FCA5
:105630006F00C004832744FC93972700032784FD51
:10564000B304F700032504FDEF20936993070500D9
:1056500023A0F400930744FB138607009745060038
:105660009385059913050000EF3013462328A4FC09
:10567000832744FC938717002322F4FC832704FD2F
:10568000E39A07FA0325C4FDEF008334232E04FCBC
:10569000930784FB9308100013880700930700000A
:1056A0001307000093060000032644FA832584FABA
:1056B0000325C4FAEFD0C1432320A4FC832704FCB4
:1056C000638A0702832704FC032744FD23A4E7021F
:1056D000832704FC032784FD23A6E7028327C4F95C
:1056E000638607008327C4F923A00700832704FCEF
:1056F0006F008003130000000325C4FDEF00432D5D
:10570000232E04FC032584FDEF00832C232C04FCB2
:105710008327C4F963880700032784FB8327C4F920
:1057200023A0E70093070000138507008320C1062C
:105730000324810683244106032901068329C10528
:10574000032A8105832A41051301010767800000B0
:10575000130101FC232E1102232C8102232A210391
:1057600023283103130401042326A4FC8325C4FC4D
:105770006392050E97B7FF019387478903A7070038
:1057800083A74700B71500003376B70093F60700EC
:1057900093070600B3E7D700638A070AEF00816525
:1057A0009306300017760600130606619305D002B3
:1057B0001775060013050574EF00515397B7FF01E5
:1057C0009387478483A707006388070297570400DD
:1057D00083A7474C83A7070083A7C70093860700CA
:1057E0001306000293051000177506001305455DAA
:1057F000EFF0525C6F00C0029757040083A78749FF
:1058000083A7070083A7C70093860700130630010C
:1058100093051000177506001305C55CEFF092594B
:105820009757040083A7074783A7070083A7C700EC
:10583000177606001306465C977506009385055D8E
:1058400013850700EFE0D20EEF00815C930740FD67
:105850006F00806A8326C4FC83A646006342D002A0
:10586000977606009386C65A177606001306866852
:105870009305F002177506001305855BEFD0D25330
:105880008326C4FC83A646009386F6FF0326C4FC49
:105890002322D6002322D4FE8326C4FC83A64600FE
:1058A00063D20602977606009386865A177606001C
:1058B000130646649305F002177506001305455755
:1058C000EFD0924F97A6FF019386467403A6060079
:1058D00083A646001377060493F706009306070095
:1058E000B3E6F6006388060AEF00C1509306100085
:1058F000177606001306C6579305000317750600B2
:105900001305455FEF00913E97A7FF019387876FCF
:1059100083A70700638807029757040083A7873788
:1059200083A7070083A7C700938607001306E0003C
:10593000930510001775060013054554EFF09247C4
:105940006F0000029757040083A7C73483A707009E
:1059500083A7C7009385070013050002EFE0D20775
:105960009757040083A7073383A7070003A5C70041
:105970008327C4FC83A7870313870700832644FE7D
:105980000326C4FC9775060093854550EFE0427AE4
:10599000EF000148832744FE639E07548327C4FC1D
:1059A00083A787002320F4FE97A7FF01938707664C
:1059B00003A7070083A747001379070493F907009B
:1059C00093070900B3E737016382070AEF008142BA
:1059D00093061000177606001306864993055003B8
:1059E0001775060013050551EF00513097A7FF0109
:1059F0009387476183A707006388070297570400CE
:105A000083A7472983A7070083A7C70093860700BA
:105A10001306E000930510001775060013050546F0
:105A2000EFF052396F0000029757040083A78726D2
:105A300083A7070083A7C70093850700130500020B
:105A4000EFE082799757040083A7C72483A7070054
:105A500083A7C7000326C4FC977506009385854677
:105A600013850700EFE0C26CEF00813A8327C4FC86
:105A700083A7070463820702977606009386C645CC
:105A80001776060013060647930580031775060070
:105A90001305053AEFD052328327C4FC03A7470110
:105AA0008327C4FC83A7870083A78700630EF700C2
:105AB0008327C4FC83A7470113850700EFF05271C9
:105AC0008327C4FC23AA07008327C4FC83A787017C
:105AD00013850700EFF0D26F8327C4FC23AC0700C7
:105AE0008327C4FC83A7872D13850700EFF0526E30
:105AF0008327C4FC23AC072C8327C4FC83A707029D
:105B000013850700EFF0D26C8327C4FC23A00702A3
:105B10008327C4FC83A7470263800706232604FE6D
:105B20006F0080048327C4FC03A747028327C4FEB9
:105B300093972700B307F70083A707001385070093
:105B4000EFF012698327C4FC03A747028327C4FE32
:105B500093972700B307F70023A007008327C4FE0D
:105B6000938717002326F4FE8327C4FC83A7C7006E
:105B70000327C4FEE368F7FA8327C4FC83A7470220
:105B800013850700EFF0D2648327C4FC23A2070229
:105B90008327C4FC83A7070313850700EFF0526334
:105BA0008327C4FC23A807028327C4FC83A74703D9
:105BB00063800706232604FE6F0080048327C4FC4D
:105BC00003A747038327C4FE93972700B307F70073
:105BD00083A7070013850700EFF0925F8327C4FCBB
:105BE00003A747038327C4FE93972700B307F70053
:105BF00023A007008327C4FE938717002326F4FE03
:105C00008327C4FC83A7C7000327C4FEE368F7FA11
:105C10008327C4FC83A7470313850700EFF0525B7B
:105C20008327C4FC23AA07020325C4FCEF30111804
:105C30008327C4FC83A7870463800706232604FE0A
:105C40006F0080048327C4FC03A787048327C4FE56
:105C500093972700B307F70083A707001385070072
:105C6000EFF012578327C4FC03A787048327C4FEE1
:105C700093972700B307F70023A007008327C4FEEC
:105C8000938717002326F4FE8327C4FC83A7C7004D
:105C90000327C4FEE368F7FA8327C4FC83A78704BD
:105CA00013850700EFF0D2528327C4FC23A4070416
:105CB0008327C4FC83A787036380071E232604FE73
:105CC0006F00001B8327C4FC03A7C7038327C4FE00
:105CD00093976700B307F700232EF4FC8327C4FDD6
:105CE00083A7070113850700EFF0924E8327C4FDB9
:105CF00023A807008327C4FD83A7C70013850700D7
:105D0000EFF0124D8327C4FD23A60700232404FED1
:105D10006F0000088327C4FD03A74701832784FE83
:105D200093975700B307F70083A747001385070031
:105D3000EFF0124A8327C4FD03A74701832784FE9F
:105D400093975700B307F70023A207008327C4FDEA
:105D500003A74701832784FE93975700B307F700F3
:105D600083A7070013850700EFF092468327C4FD41
:105D700003A74701832784FE93975700B307F700D3
:105D800023A00700832784FE938717002324F4FEB3
:105D90008327C4FD83A70700032784FEE36CF7F67F
:105DA0008327C4FD83A7470113850700EFF0524204
:105DB0008327C4FD23AA07008327C4FD83A7870385
:105DC000638E0704232404FE6F0040048327C4FD70
:105DD00003A78703832784FE93972700B307F70061
:105DE00083A70700638E07008327C4FD03A78703EB
:105DF000832784FE93972700B307F70023A00700AB
:105E0000832784FE938717002324F4FE8327C4FC92
:105E100083A7C700032784FEE36AF7FA8327C4FD3C
:105E200083A7870313850700EFF0923A8327C4FD09
:105E300023AC07028327C4FD83A7870013850700CF
:105E4000EFF012398327C4FD23A407008327C4FD84
:105E500083A7C70213850700EFF092378327C4FD9D
:105E600023A607028327C4FE938717002326F4FE88
:105E70008327C4FC83A787030327C4FEE364F7E4F6
:105E80008327C4FC83A7C70313850700EFF05234B0
:105E90008327C4FC23AE07028327C4FC83A74704DF
:105EA00013850700EFF0D2328327C4FC23A2070436
:105EB0008327C4FC83A7C70113850700EFF0523185
:105EC0008327C4FC23AE07008327C4FC83A7C72C09
:105ED00013850700EFF0D22F8327C4FC23A6072CDD
:105EE0000325C4FCEFF0D22E232604FC032504FE78
:105EF000EFB05FD293070000138507008320C10332
:105F000003248103032941038329010313010104AD
:105F100067800000130101FB232611042324810460
:105F2000130401052326A4FE2324B4FE2322C4FE69
:105F30002320D4FE232EE4FC232CF4FC832784FDB1
:105F40002328F1008327C4FD2326F1002324010028
:105F50002322010023200100930800001308000001
:105F6000832704FE032744FE832684FE0326C4FE03
:105F70009305100013051000EF10806493070500CF
:105F8000138507008320C104032481041301010544
:105F900067800000130101F32326110C2324810CD8
:105FA0002322210D2320310D232E410B232C510BB5
:105FB000232A610B2328710B2326810B2324910BA9
:105FC0002322A10B2320B10B1304010D232EA4F6D1
:105FD000232CB4F6232AC4F62328D4F62326E4F689
:105FE0002324F4F6232204F7232014F7232404FCAB
:105FF000232404F8832744F623A00700832704F60C
:1060000023A007008327040023A007008327440060
:1060100023A00700232204FC832744F723800700E2
:10602000832784F723800700832784F6638E070085
:106030008327C4F663860700930750FD6F000001B5
:106040009307D0FB6F0080009307E0FB232EF4FA48
:106050008327C4F76392070297E6060093860670CB
:1060600017F606001306861B9305000E17E50600BB
:106070001305456FEFD04254832784F763920702DC
:1060800097E606009386866F17F606001306061934
:106090009305100E17E506001305C56CEFD0C2512D
:1060A0008327C4F663960702832784F66392070268
:1060B00097E606009386866D17F606001306061609
:1060C0009305200E17E506001305C569EFD0C24EF3
:1060D000930710002320F4FC232C04FA0325C4F7B3
:1060E000EF20930C93070500938717001385070093
:1060F000EFF0120D93070500232AF4FA8325C4F765
:10610000032544FBEF20C332930784F8138607006E
:1061100097E5060093850569032544FBEF30C31A14
:106120002324A4FC6F1000001306300097E506003E
:1061300093858567032584FCEF20D30F9307050023
:10614000638E07021306200097E506009385056617
:10615000032584FCEF20130E9307050063800702DC
:106160001306700097E5060093858564032584FC7B
:10617000EF20530C93070500639A0740832584FCA6
:1061800017E5060013054554EF20936293070500B9
:1061900063840718832784F6638C07128327C4F669
:1061A00063980712832744FC639E071097A7FF019B
:1061B0009387C7E503A7070083A74700B71600002A
:1061C0003379D70093F9070093070900B3E7370144
:1061D0006382070AEFF010429306300017E60600CC
:1061E0001306865D9305800F17F50600130505035A
:1061F000EF00C12F97A7FF019387C7E083A7070090
:10620000638807029757040083A7C7A883A70700DE
:1062100083A7C700938607001306E00093051000CC
:1062200017E506001305C559EFF0C2386F000002EC
:106230009757040083A707A683A7070083A7C70073
:106240009385070013050002EFD0127997570400D9
:1062500083A747A483A7070083A7C700032684FC5E
:1062600097E506009385C55613850700EFD0526C5D
:10627000EFF0103A832704F79387C70413850700CC
:10628000EF208372232AA4F8832704F71387C70417
:10629000832744F93305F70013070028832744F9BF
:1062A000B307F740832684FC17E606001306465220
:1062B00093850700EF1013458327C4FB2326F4FCC6
:1062C0006F00106C832584FC032544F7EF101376D0
:1062D00097E5060093850555032584FCEF20534D73
:1062E0009307050063880700832704F6130710004F
:1062F00023A0E70097E5060093854554032584FC19
:10630000EF20134B930705006388070083270400E1
:106310001307100023A0E700832584FC17E506007F
:1063200013050527EF20D34893070500E39A075488
:10633000832584FC17E5060013054540EF205347ED
:10634000930705006388071297A7FF01938707CC7F
:1063500003A7070083A74700B7160000337AD700CA
:1063600093FA070093070A00B3E757016382070A0D
:10637000EFF050289306300017E606001306C643D8
:106380009305101117F50600130545E9EF000116F6
:1063900097A7FF01938707C783A7070063880702B2
:1063A0009757040083A7078F83A7070083A7C70019
:1063B000938607001306E0009305100017E506001A
:1063C00013050540EFF0021F6F000002975704000D
:1063D00083A7478C83A7070083A7C700938507007F
:1063E00013050002EFD0525F9757040083A7878AF6
:1063F00083A7070083A7C700032684FC97E5060050
:106400009385454613850700EFD09252EFF0502058
:10641000832704F79387C70413850700EF20C35829
:106420002326A4F8832704F71387C7048327C4F817
:106430003305F700130700288327C4F8B307F74094
:10644000832684FC17E606001306C64193850700E1
:10645000EF10532B930784F81386070097E5060087
:106460009385453413050000EF2013662324A4FC14
:106470006F00504B97A7FF01938747B903A7070009
:1064800083A74700B7160000337BD70093FB0700B4
:1064900093070B00B3E777016382070AEFF09015CB
:1064A0009306300017E60600130606319305901197
:1064B00017F50600130585D6EF00410397A7FF01E6
:1064C000938747B483A707006388070297470400B0
:1064D00083A7477C83A7070083A7C700938607008D
:1064E0001306E0009305100017E506001305452D7F
:1064F000EFF0420C6F0000029747040083A78779F2
:1065000083A7070083A7C700938507001305000230
:10651000EFD0924C9747040083A7C77783A7070063
:1065200083A7C700032684FC97E5060093850537FB
:1065300013850700EFD0D23FEFF0900D832704F7CB
:106540009387C70413850700EF2003462328A4F888
:10655000832704F71387C704832704F93305F7005B
:1065600013070028832704F9B307F740832684FC28
:1065700017E606001306863293850700EF1093187E
:106580008327C4FB2326F4FC6F00903F13062000F2
:1065900097E5060093854532032584FCEF20834967
:1065A00093070500639A070097E706009387073172
:1065B0002324F4FC6F00D02C1306200097E506007E
:1065C00093850535032584FCEF20C346930705001A
:1065D000638007021306200097E506009385853344
:1065E000032584FCEF200345930705006390070E05
:1065F000032584FCEF20433B930705009387170096
:10660000232CF4FA032704FC832784FBB307F70049
:106610000327840063E2E70297E606009386C62F0D
:1066200017F60600130686BF9305501217E50600FD
:1066300013054513EFC05278032704FC832784FB1E
:10664000B307F7002320F4FC832584FC032584F79B
:10665000EF10D33D032584F7EF20033593070500A2
:1066600013870700832784F7B387E7001307000227
:106670002380E700A3800700032584FCEF20C332BA
:1066800013070500930720006312F702930784F8AD
:106690001386070097E506009385C51013050000D3
:1066A000EF2093422324A4FC6F00901D930784F8ED
:1066B0001386070097E506009385C50E13050000B5
:1066C000EF2093402324A4FC6F00D0251306200064
:1066D00097E5060093858525032584FCEF20833507
:1066E000930705006394072C032584FCEF20C32B3C
:1066F0001307050093072000631AF72A930784F80D
:106700001386070097E506009385C5091305000069
:10671000EF20933B2324A4FC832784FC638007029F
:106720001306400097E5060093858520032584FC29
:10673000EF204330930705006380071297A7FF01FE
:106740009387C78C03A7070083A74700B7160000ED
:10675000337CD70093FC070093070C00B3E7970145
:106760006384070AEFF000699306300017E606001D
:10677000130686049305601317F50600130505AA92
:10678000EFF0D05697A7FF019387C78783A707002D
:10679000638807029747040083A7C74F83A70700B2
:1067A00083A7C700938607001306E0009305100037
:1067B00017E506001305C500EFE0D25F6F00000289
:1067C0009747040083A7074D83A7070083A7C70047
:1067D0009385070013050002EFD0122097470400AD
:1067E00083A7474B83A7070083A7C70093860700AB
:1067F000130650029305100017E506001305C51394
:10680000EFE0525BEFF0C060832704F79387C70483
:1068100013850700EF2043192326A4FA832704F7E2
:106820001387C7048327C4FAB306F70013070028A9
:106830008327C4FAB307F74017E606001306C60F0E
:106840009385070013850600EF10C36B8327C4FBF5
:106850002326F4FC6F00D012832704F783A7870157
:10686000638007129797FF019387477A03A7070072
:1068700083A74700B7160000337DD70093FD0700BC
:1068800093070D00B3E7B7016384070AEFF0805662
:106890009306300017E60600130606F29305E01390
:1068A00017F5060013058597EFF050449797FF0101
:1068B0009387477583A707006388070297470400FB
:1068C00083A7473D83A7070083A7C70093860700D8
:1068D0001306E0009305100017E50600130545EECA
:1068E000EFE0524D6F0000029747040083A7873AFC
:1068F00083A7070083A7C70093850700130500023D
:10690000EFD0920D9747040083A7C73883A70700ED
:1069100083A7C70093860700130610039305100092
:1069200017E506001305C503EFE0D248EFF0404E2F
:10693000832704F79387C70413850700EF20C30656
:106940002328A4FA832704F71387C704832704FBAB
:10695000B306F70013070028832704FBB307F740AB
:1069600017E606001306C6FF938507001385060089
:10697000EF1043598327C4FB2326F4FC6F0050001B
:10698000832744001307100023A0E700930784F82F
:106990001386070097E506009385C5E01305000000
:1069A000EF2093122324A4FC6F00C0771306D000BD
:1069B00097E50600938505FE032584FCEF208307F9
:1069C0009307050063940716832704F783A78701BD
:1069D000638807129797FF019387476303A7070010
:1069E00083A74700B7160000B376D700232CD4F452
:1069F00093F70700232EF4F4832684F50327C4F5C8
:106A000093870600B3E7E7006384070AEFF0803E50
:106A10009306300017E60600130606DA9305D01435
:106A200017E506001305857FEFF0502C9797FF01BF
:106A30009387475D83A70700638807029747040091
:106A400083A7472583A7070083A7C700938607006E
:106A50001306E0009305100017E50600130545D660
:106A6000EFE052356F0000029747040083A78722AA
:106A700083A7070083A7C7009385070013050002BB
:106A8000EFD082759747040083A7C72083A707002C
:106A900083A7C70093860700130690039305100091
:106AA00017E50600130505F0EFE0D230EFF04036B1
:106AB000832704F79387C70413850700EF10D36E6D
:106AC000232CA4F8832704F71387C704832784F9AA
:106AD000B306F70013070028832784F9B307F740AC
:106AE00017E60600130606EC9385070013850600DB
:106AF000EF1043418327C4FB2326F4FC6F0040685A
:106B0000832744001307100023A0E700930784F8AD
:106B10001386070097E506009385C5C81305000096
:106B2000EF20837A2324A4FC6F00C05F1306F000DB
:106B300097E506009385C5EA032584FCEF10936F63
:106B40009307050063920716832784F6639807125C
:106B50009797FF019387874B03A7070083A74700F9
:106B6000B7160000B376D7002328D4F493F70700B4
:106B7000232AF4F4832604F5032744F593870600BB
:106B8000B3E7E7006384070AEFF0C02693063000FE
:106B900017E60600130646C29305B01517E5060072
:106BA0001305C567EFF090149797FF01938787450A
:106BB00083A70700638807029747040083A7870D10
:106BC00083A7070083A7C700938607001306E0008A
:106BD0009305100017E50600130585BEEFE0921D32
:106BE0006F0000029747040083A7C70A83A7070026
:106BF00083A7C7009385070013050002EFD0C25D8D
:106C00009747040083A7070983A7070083A7C70046
:106C100093860700130620039305100017E506006E
:106C2000130505DDEFE01219EFF0801E832704F74E
:106C30009387C70413850700EF101357232EA4F87A
:106C4000832704F71387C7048327C4F9B306F70023
:106C5000130700288327C4F9B307F74017E6060097
:106C6000130606D99385070013850600EF108329C4
:106C70008327C4FB2326F4FC6F008050832744F64F
:106C80001307100023A0E700930784F8138607007A
:106C900097E50600938505B113050000EF20C36258
:106CA0002324A4FC6F0000481306400197E506006A
:106CB000938545D7032584FCEF10D3579307050030
:106CC000639C0728832784F6639807129797FF0130
:106CD0009387C73303A7070083A74700B7160000B1
:106CE000B376D7002324D4F493F707002326F4F4D3
:106CF000832684F40327C4F493870600B3E7E700F0
:106D00006384070AEFF0000F9306300017E60600D1
:106D1000130686AA9305801617E50600130505508D
:106D2000EFF0C07C9797FF019387C72D83A70700DB
:106D3000638807029747040083A7C7F583A7070066
:106D400083A7C700938607001306E0009305100091
:106D500017E506001305C5A6EFE0D2056F00000297
:106D60009747040083A707F383A7070083A7C700FB
:106D70009385070013050002EFD0024697470400F1
:106D800083A747F183A7070083A7C700938607005F
:106D9000130670039305100017E50600130505CAD6
:106DA000EFE05201EFF0C006832704F79387C70492
:106DB00013850700EF10533F2320A4FA832704F71D
:106DC0001387C704832704FAB306F70013070028C4
:106DD000832704FAB307F74017E60600130606C632
:106DE0009385070013850600EF10C3118327C4FBAA
:106DF0002326F4FC6F00C038832744F683A70700DE
:106E0000639807129797FF019387472003A707000E
:106E100083A74700B7160000B376D7002320D4F429
:106E200093F707002322F4F4832604F4032744F4A1
:106E300093870600B3E7E7006384070AEFE0907BDF
:106E40009306300017E60600130606979305F01622
:106E500017E506001305853CEFF040699797FF01A1
:106E60009387471A83A707006388070297470400A0
:106E700083A747E283A7070083A7C700938607007D
:106E80001306E0009305100017E50600130545936F
:106E9000EFE042726F0000029747040083A787DF8C
:106EA00083A7070083A7C700938507001305000287
:106EB000EFD082329747040083A7C7DD83A707007E
:106EC00083A7C700938607001306000593051000EB
:106ED00017E50600130505BAEFE0C26DEFE0507349
:106EE000832704F79387C70413850700EF10D32B7C
:106EF0002322A4FA832704F71387C704832744FABD
:106F0000B306F70013070028832744FAB307F740B6
:106F100017E60600130606B69385070013850600DC
:106F2000EF00537E8327C4FB2326F4FC6F0040252B
:106F3000930710002322F4FC930784F813860700BC
:106F400097E506009385058613050000EF20C337FB
:106F50002324A4FC6F00001D9797FF019387070B64
:106F600003A7070083A74700B7160000B376D70032
:106F7000232CD4F293F70700232EF4F2832684F314
:106F80000327C4F393870600B3E7E7006382070A89
:106F9000EFE050669306300017E606001306C68140
:106FA0009305B01717E5060013054527EFF00054C9
:106FB0009797FF019387070583A707006388070258
:106FC0009747040083A707CD83A7070083A7C700BF
:106FD000938607001306E0009305100017D50600FE
:106FE0001305057EEFE0025D6F0000029747040085
:106FF00083A747CA83A7070083A7C7009385070015
:1070000013050002EFD0421D9747040083A787C8ED
:1070100083A7070083A7C700032684FC97E5060023
:107020009385C58713850700EFD08210EFE0505E8F
:10703000832704F79387C70413850700EF10D3163F
:107040002324A4FA832704F71387C704832784FA29
:107050003305F70013070028832784FAB307F740A6
:10706000832684FC17E606001306468393850700F3
:10707000EF0053698327C4FB2326F4FC6F00401004
:10708000032584FCEF105312930705009387170024
:10709000232CF4FA032704FC832784FBB307F700AF
:1070A0000327840063E2E70297E606009386C6861C
:1070B00017E60600130686169305F01717D5060087
:1070C0001305456AEFC0424F032704FC832784FB66
:1070D000B307F7002320F4FC832584FC032584F701
:1070E000EF10C314032584F7EF10130C930705006A
:1070F00013870700832784F7B387E700130700028D
:107100002380E700A3800700930784F81386070015
:1071100097D506009385056913050000EF20C31A73
:107120002324A4FC832784FC638407006FE0DFFF33
:10713000232604FC032584F7EF1013072320A4FC67
:10714000832704FC638C0702832704FC9387F7FFE3
:10715000032784F7B307F70003C70700930700026C
:10716000631EF700832704FC9387F7FF032784F748
:10717000B307F700238007006F00800013000000B2
:10718000032544FBEFE0D204232A04FA8327C4FC3E
:10719000138507008320C10C0324810C0329410CB3
:1071A0008329010C032AC10B832A810B032B410B7A
:1071B000832B010B032CC10A832C810A032D410A66
:1071C000832D010A1301010D67800000130101FDE9
:1071D000232611022324810213040103232EA4FC7D
:1071E0008327C4FD83A78703638A071E232604FE23
:1071F0006F00401C8327C4FD03A7C7038327C4FE79
:1072000093976700B307F7002322F4FE832744FE19
:1072100083A7C70213850700EFE0827B832744FE24
:1072200023A60702832744FE03A6070383A647037A
:1072300093070600B3E7D70063960716832744FE3B
:1072400083A7070113850700EFE08278832744FEB8
:1072500023A80700832744FE83A7C70013850700E0
:10726000EFE00277832744FE23A60700232404FED1
:107270006F000008832744FE03A74701832784FE8D
:1072800093975700B307F70083A7470013850700BC
:10729000EFE00274832744FE03A74701832784FE9F
:1072A00093975700B307F70023A20700832744FEF4
:1072B00003A74701832784FE93975700B307F7007E
:1072C00083A7070013850700EFE08270832744FE41
:1072D00003A74701832784FE93975700B307F7005E
:1072E00023A00700832784FE938717002324F4FE3E
:1072F000832744FE83A70700032784FEE36CF7F689
:10730000832744FE83A7470113850700EFE0426C03
:10731000832744FE23AA0700232404FE6F004004B1
:10732000832744FE03A78703832784FE93972700C0
:10733000B307F70083A70700638E0700832744FE87
:1073400003A78703832784FE93972700B307F700DB
:1073500023A00700832784FE938717002324F4FECD
:107360008327C4FD83A7C700032784FEE36AF7FAD7
:10737000832744FE83A7870313850700EFE0426558
:10738000832744FE23AC0702832744FE83A787009C
:1073900013850700EFE0C263832744FE23A40700A0
:1073A0006F008000130000008327C4FE938717003E
:1073B0002326F4FE8327C4FD83A787030327C4FE87
:1073C000E36AF7E28327C4FD83A7C7031385070099
:1073D000EFE002608327C4FD23AE07021300000024
:1073E0008320C1020324810213010103678000008E
:1073F000130101FD2326110223248102130401033A
:10740000232EA4FC8327C4FD03A7072D9307F0FFB9
:107410006318F7008327C4FD83A7870363880718D1
:107420008327C4FD83A707046382070297D606005B
:107430009386866917E60600130646DF9305C01B90
:1074400017D5060013050532EFC002170325C4FD4A
:10745000EFF0DFD78327C4FD23AC07028327C4FDE9
:107460001307F0FF23A8E72C232604FE6F008012E9
:107470008327C4FD03A787048327C4FE93972700AF
:10748000B307F70083A7070013850700EFE0425416
:107490008327C4FD03A787048327C4FE939727008F
:1074A000B307F70023A007008327C4FD83A6470482
:1074B0000327C4FE9307070093972700B387E700CD
:1074C00093973700B387E700B387F600130690025F
:1074D0009305000013850700EFF082048327C4FDA5
:1074E00083A787016382070A8327C4FD03A7470296
:1074F0008327C4FE93972700B307F70083A70700ED
:1075000013850700EFE0C24C8327C4FD03A74702A1
:107510008327C4FE93972700B307F70023A0070033
:107520008327C4FD03A707028327C4FE9397270080
:10753000B307F70023A007008327C4FD03A7470371
:107540008327C4FE93972700B307F70083A707009C
:1075500013850700EFE0C2478327C4FD03A7470355
:107560008327C4FE93972700B307F70023A00700E3
:107570008327C4FD03A707038327C4FE939727002F
:10758000B307F70023A007008327C4FE93871700E3
:107590002326F4FE8327C4FD83A7C7000327C4FE68
:1075A000E368F7EC8327C4FD23860704130000007B
:1075B0008320C102032481021301010367800000BC
:1075C0001301018B232611742324817423229174C7
:1075D00023202175232E3173232C4173232A5173C9
:1075E00023286173232671732324817323229173CB
:1075F0002320A173232EB17113040175232EA494AB
:10760000232CB494232AC4942328D4942326E494CA
:107610002324F494232204952320149523280496EC
:10762000232604962324049623220496232C04FA6A
:10763000232C04F8232A04FA232804FA232204FA28
:107640009305000017D506001305C549EFE0806FCC
:10765000232AA4F88327849563860700930750FFA5
:107660006F008000930710FF2328F4F883274495C8
:107670006394070E9797FF019387479903A7070025
:1076800083A74700B71600003379D70093F90700A6
:1076900093070900B3E73701638A070AEFE08075B3
:1076A0009306300017D60600130606119305A01F97
:1076B00017E50600130545B9EFE050639797FF0102
:1076C0009387479483A707006388070297370400CE
:1076D00083A7475C83A7070083A7C700938607009B
:1076E000130600029305100017D506001305054187
:1076F000EFD0526C6F00C0029737040083A7875900
:1077000083A7070083A7C7009386070013063001ED
:107710009305100017D5060013058540EFD0926938
:107720009737040083A7075783A7070083A7C700DD
:1077300017D606001306064097D506009385C54068
:1077400013850700EFC0D21EEFE0806C930740FD69
:10775000232EF4FA6F10D019832704956388070E3F
:107760008327C4946394070E9797FF019387078A32
:1077700003A7070083A74700B7160000337AD70096
:1077800093FA070093070A00B3E75701638A070AD1
:10779000EFE040669306300017D606001306C601D8
:1077A0009305C01F17E50600130505AAEFE0105466
:1077B0009797FF019387078583A7070063880702D0
:1077C0009737040083A7074D83A7070083A7C70047
:1077D000938607001306E0019305100017D50600F5
:1077E0001305C536EFD0125D6F00C0029737040055
:1077F00083A7474A83A7070083A7C700938607008C
:10780000130610019305100017D506001305053661
:10781000EFD0525A9737040083A7C74783A70700C2
:1078200083A7C70017D606001306863597D506002E
:107830009385853113850700EFC0920FEFE0405D1F
:10784000930720FE232EF4FA6F10900A83270495E5
:107850006398070E8327C4946384070E9787FF01FC
:107860009387C77A03A7070083A74700B7160000CE
:10787000337BD70093FB070093070B00B3E7770137
:10788000638A070AEFE000579306300017D6060018
:10789000130686F29305E01F17E506001305C59A47
:1078A000EFE0D0449787FF019387C77583A7070050
:1078B000638807029737040083A7C73D83A70700A3
:1078C00083A7C700938607001306E0019305100005
:1078D00017D5060013058527EFD0D24D6F00C002E3
:1078E0009737040083A7073B83A7070083A7C70038
:1078F00093860700130610019305100017D50600A4
:107900001305C526EFD0124B9737040083A787389D
:1079100083A7070083A7C70017D60600130606290A
:1079200097D506009385452213850700EFC05200C6
:10793000EFE0004E930720FE232EF4FA6F10407BF9
:107940008327C4006398070E832704016384070E0E
:107950009787FF019387876B03A7070083A74700DB
:10796000B7160000337CD70093FC070093070C0088
:10797000B3E79701638A070AEFE0C0479306300038
:1079800017D60600130646E39305102017E50600F8
:107990001305858BEFE090359787FF019387876606
:1079A00083A70700638807029737040083A7872E01
:1079B00083A7070083A7C700938607001306E0018B
:1079C0009305100017D5060013054518EFD0923E19
:1079D0006F00C0029737040083A7C72B83A7070057
:1079E00083A7C700938607001306100193051000B4
:1079F00017D5060013058517EFD0D23B9737040043
:107A000083A7472983A7070083A7C70017D60600C7
:107A10001306861C97D5060093850513138507006A
:107A2000EFC00271EFE0C03E930720FE232EF4FA70
:107A30006F10006C8327449583A707046384070EA7
:107A40009787FF019387875C03A7070083A74700F9
:107A5000B7160000337DD70093FD070093070D0094
:107A6000B3E7B701638A070AEFE0C0389306300036
:107A700017D60600130646D49305402017D50600F6
:107A80001305857CEFE090269787FF019387875742
:107A900083A70700638807029737040083A7871F1F
:107AA00083A7070083A7C700938607001306200259
:107AB0009305100017D506001305C514EFD0922FBB
:107AC0006F00C0029737040083A7C71C83A7070075
:107AD00083A7C70093860700130650019305100083
:107AE00017D5060013054514EFD0D22C97370400A4
:107AF00083A7471A83A7070083A7C70093860700B9
:107B00001306C0019305100017D506001305451391
:107B1000EFD0522AEFE0C02F930750FC232EF4FA47
:107B20006F10005D8327449583A787016398071032
:107B30008327449583A747026392071083274495C0
:107B400083A7C702639C070E9787FF019387074CA3
:107B500003A7070083A74700B7160000B376D70036
:107B6000232CD49293F70700232EF4928326849338
:107B70000327C49393870600B3E7E700638A070AE5
:107B8000EFE040279306300017D606001306C6C262
:107B90009305702017D506001305056BEFE010154F
:107BA0009787FF019387074683A70700638807022B
:107BB0009737040083A7070E83A7070083A7C70092
:107BC00093860700130600029305100017D50600E0
:107BD0001305C5F2EFD0121E6F00C00297370400E4
:107BE00083A7470B83A7070083A7C70093860700D7
:107BF000130630019305100017D50600130545F252
:107C0000EFD0521B9737040083A7C70883A707004C
:107C100083A7C700938607001306A00893051000EA
:107C200017D506001305C503EFD0D218EFE0401EAC
:107C3000930740FD232EF4FA6F10804B8327449561
:107C400083A787016390071083278495639C070EA1
:107C50009787FF019387873B03A7070083A7470008
:107C6000B7160000B376D7002328D49293F7070005
:107C7000232AF492832604930327449393870600D0
:107C8000B3E7E700638A070AEFE0C0169306300007
:107C900017D60600130646B29305002117D5060035
:107CA0001305855AEFE090049787FF019387873586
:107CB00083A70700638807029737040083A787FD1F
:107CC00083A7070083A7C700938607001306200237
:107CD0009305100017D506001305C5F2EFD0920DDD
:107CE0006F00C0029737040083A7C7FA83A7070075
:107CF00083A7C70093860700130650019305100061
:107D000017D50600130545F2EFD0D20A97370400C5
:107D100083A747F883A7070083A7C70093860700B8
:107D2000130630039305100017D50600130505FC54
:107D3000EFD05208EFE0C00D930750FC232EF4FA69
:107D40006F10003B8327449583A747006342F002EE
:107D500097D606009386C6FC17D606001306C64EB5
:107D60009305502117D506001305C59FEFB0D20427
:107D700083274495238607048327449583A7C70157
:107D800013850700EFD0D2448327449523AE070024
:107D9000832744F96380070A83278494638A070052
:107DA00003258494EF005340930705006F00800083
:107DB000930700002326F4F8032544F9EF00D33E8F
:107DC000130705008327C4F8B307F700938727003C
:107DD0002326F4F80325C4F8EFD0923E930705005C
:107DE0002322F4FA832744FA23800700832784940C
:107DF000638A070283258494032544FAEF004363D2
:107E0000032544FAEF00533A930705001387070050
:107E1000832744FA3387E700930700022300F70023
:107E2000A3000700832544F9032544FAEF0003402B
:107E30006F00C000832784942322F4FA832744FA36
:107E400063860708032544FAEF0013362326A4FAB5
:107E50008327C4FA938707202324F4F8032584F8A2
:107E6000EFD0123693070500138707008327449548
:107E700023AEE7008327449583A5C7019306449664
:107E80001307049713064497832784F82324F100EB
:107E9000930784962322F1009307C4962320F100D0
:107EA0009388060013080700832784950327C49549
:107EB00083264495032544FAEFE0CF8D232EA4FAC0
:107EC0008327C4FB638407006F10C01C9787FF01E2
:107ED0009387C71303A7070083A74700937647003C
:107EE0002324D49293F707002326F49283268492C6
:107EF0000327C49293870600B3E7E7006386070A67
:107F0000EFD0506F9306100017D60600130646E315
:107F10009305A02317D5060013050533EFE0005D98
:107F20009787FF019387070E83A7070063880702DF
:107F30009737040083A707D683A7070083A7C70046
:107F4000938607001306E0009305100017D506007E
:107F500013050587EFD002666F0000029737040013
:107F600083A747D383A7070083A7C700938507008C
:107F700013050002EFC042269737040083A787D17C
:107F800083A7070003A7C7008327449583A7C701DA
:107F90001386070097D50600938505DB13050700B8
:107FA000EFC00219EFD0D06603274496832744958B
:107FB00023A8E700832744966382070E9787FF0173
:107FC0009387C70403A7070083A74700B7160000DD
:107FD00093860680B376D7002320D49293F70700C8
:107FE0002322F49283260492032744929387060067
:107FF000B3E7E7006384070AEFD0D05F9306200061
:1080000017D60600130686D69305202417D506003A
:1080100013058523EFE0804D9787FF01938787FE47
:1080200083A70700638807029737040083A787C6E2
:1080300083A7070083A7C700938607001306E00005
:108040009305100017C5060013058577EFD08256FB
:108050006F0000029737040083A7C7C383A70700F8
:1080600083A7C7009385070013050002EFC0C2165F
:108070009737040083A707C283A7070083A7C70019
:1080800093860700130620059305100017D50600F8
:10809000130545CEEFD00252EFD0905783270495B9
:1080A000639007028327449583A7C7002328F4948D
:1080B0008327449583A747012326F4946F00000388
:1080C00023200496930704961386070083250495BE
:1080D0000325C494EFB0406E232CA4FA83270496A2
:1080E0002328F494832784FB2326F49403254495C2
:1080F000EFF00FB0232A04FA6F00D02483274495B1
:1081000003A74701832744FB93972700B307F70092
:1081100083A707002320F4F8232004FA232604FA77
:108120006F0040038327C4FA939727000327C49462
:10813000B307F70083A70700032704F86316F700C7
:10814000930710002320F4FA8327C4FA93871700BB
:108150002326F4FA0327C4FA83270495E364F7FC83
:10816000832704FAE380071C8327C49663860724C9
:10817000832704F803A7070D83A7470D9376070805
:10818000232CD49093F70700232EF4908326849118
:108190000327C49193870600B3E7E700639E072097
:1081A0009787FF01938787E603A7070083A7470008
:1081B000B7160000B376D7002328D49093F70700B2
:1081C000232AF49083260491032744919387060081
:1081D000B3E7E7006384070AEFD0D041930630008D
:1081E00017C606001306465D9305802617D50600C0
:1081F00013058505EFE0802F9787FF01938787E0C0
:1082000083A70700638807029737040083A787A81E
:1082100083A7070083A7C700938607001306E00023
:108220009305100017C5060013058559EFD0823855
:108230006F0000029737040083A7C7A583A7070034
:1082400083A7C7009385070013050002EFB0D2781B
:108250009737040083A707A483A7070083A7C70055
:1082600093860700130600089305100017D5060033
:10827000130585B5EFD00234EFD0903983274495AC
:108280009387C70413850700EF000372232EA4F61B
:10829000832744951387C7048327C4F7B306F700E1
:1082A000130700288327C4F7B307F74017D6060043
:1082B000130686B19385070013850600EFF09244FC
:1082C0009787FF01938787D403A7070083A74700F9
:1082D000B7160000B376D7002324D49093F7070095
:1082E0002326F490832684900327C4909387060066
:1082F000B3E7E700638C070AEFD0D02F9306300076
:1083000017C606001306464B9305902617D50600A0
:10831000130585F3EFE0801D9787FF01938787CED4
:1083200083A70700638807029737040083A787960F
:1083300083A7070083A7C700938607001306E00101
:108340009305100017D50600130545B0EFD082261F
:108350006F00C0029737040083A7C79383A7070065
:1083600083A7C7009386070013061001930510002A
:1083700017D50600130585AFEFD0C2239737040049
:1083800083A7479183A7070003A7C700832704F8A3
:1083900083A7C7161386070097D50600938545AEB9
:1083A00013050700EFB0D258EFD09026832704F9C9
:1083B000232EF4FA6F00D044832704FB9387170021
:1083C0002328F4FA8327449583A7C702639007768E
:1083D0008327449583A78701638A07209787FF0136
:1083E0009387C7C203A7070083A74700B7160000FB
:1083F000B376D7002320D49093F707002322F4907C
:10840000832604900327449093870600B3E7E70090
:108410006384070AEFD0101E9306300017C60600CB
:10842000130686399305602817D506001305C5E1A4
:10843000EFE0C00B9787FF019387C7BC83A70700B6
:10844000638807029737040083A7C78483A70700C0
:1084500083A7C700938607001306E000930510006A
:1084600017C506001305C535EFD0C2146F00000212
:108470009737040083A7078283A7070083A7C70055
:108480009385070013050002EFB0125597370400DB
:1084900083A7478083A7070083A7C70093860700A9
:1084A000130690059305100017D506001305C5A502
:1084B000EFD04210EFD0D015832744959387C7049F
:1084C00013850700EF00434E232AA4F68327449523
:1084D0001387C704832744F7B306F7001307002860
:1084E000832744F7B307F74017D606001306C6A143
:1084F0009385070013850600EFF0D2209787FF01D0
:108500009387C7B003A7070083A74700B7160000EB
:10851000B376D700232CD48E93F70700232EF48E46
:108520008326848F0327C48F93870600B3E7E70071
:108530006388070AEFD0100C9306300017C60600B8
:10854000130686279305902817D506001305C5CF77
:10855000EFD0D0799787FF019387C7AA83A7070039
:10856000638807029727040083A7C77283A70700C1
:1085700083A7C700938607001306700293051000B7
:1085800017D506001305059EEFD0C2026F00C0028A
:108590009727040083A7077083A7070083A7C70056
:1085A000938607001306A0019305100017D5060057
:1085B0001305C59DEFD002009727040083A7876DA0
:1085C00083A7070003A7C700832744959387C704A1
:1085D0009305070013850700EFB09251EFD05003C9
:1085E0009307D0FF232EF4FA6F0090218327449540
:1085F00003A74702832744FB93972700B307F7009D
:1086000083A70700638807228327449503A74703AE
:10861000832744FB93972700B307F70083A707003E
:10862000639A07209787FF019387479E03A7070058
:1086300083A74700B7160000B376D7002328D48E4F
:1086400093F70700232AF48E8326048F0327448F91
:1086500093870600B3E7E7006384070AEFD08079C9
:108660009306300017C60600130606159305A02BC7
:1086700017D50600130545BDEFD050679787FF015A
:108680009387479883A7070063880702972704000A
:1086900083A7476083A7070083A7C70093860700C7
:1086A0001306E0009305100017C5060013054511D9
:1086B000EFC052706F0000029727040083A7875D08
:1086C00083A7070083A7C70093850700130500024F
:1086D000EFB092309727040083A7C75B83A70700FA
:1086E00083A7C700938607001306000693051000B2
:1086F00017D506001305458BEFC0D26BEFD0407144
:10870000832744959387C70413850700EF00C32987
:10871000232CA4F6832744951387C704832784F763
:10872000B306F70013070028832784F7B307F74041
:1087300017D60600130646879385070013850600A3
:10874000EFF0427C9787FF019387478C03A70700D0
:1087500083A74700B7160000B376D7002324D48E32
:1087600093F707002326F48E8326848E0327C48E76
:1087700093870600B3E7E7006388070AEFD08067B6
:108780009306300017C60600130606039305D02B88
:1087900017D50600130545ABEFD050559787FF015D
:1087A0009387478683A707006388070297270400FB
:1087B00083A7474E83A7070083A7C70093860700B8
:1087C000130670029305100017C50600130585797E
:1087D000EFC0525E6F00C0029727040083A7874B4B
:1087E00083A7070083A7C700938607001306A0018D
:1087F0009305100017C5060013054579EFC0925B7D
:108800009727040083A7074983A7070003A7C7008A
:10881000832744959387C7049305070013850700B2
:10882000EFB0122DEFD0C05E9307D0FF232EF4FAE5
:108830006F00007D8327449503A74703832744FBEC
:1088400093972700B307F70083A70700638E070CF1
:108850009777FF019387877B03A7070083A74700CC
:10886000937617002320D48E93F707002322F48EEB
:108870008326048E0327448E93870600B3E7E70020
:10888000638A072AEFD000579306100017C6060028
:108890001306C6779305302C17D506001305C59A25
:1088A000EFD0D0449777FF019387C77583A7070060
:1088B000638807029727040083A7C73D83A70700A3
:1088C00083A7C700938607001306E00093051000F6
:1088D00017C506001305C5EEEFC0D24D6F000002AC
:1088E0009727040083A7073B83A7070083A7C70038
:1088F0009385070013050002EFB0120E97270400BE
:1089000083A7473983A7070083A7C700032644FB33
:1089100097C506009385057013850700EFB05201D7
:10892000EFD0004F6F0000218327849563800710EC
:1089300083274400638C070E9777FF019387076DA9
:1089400003A7070083A74700B7160000B376D70038
:10895000232CD48C93F70700232EF48C8326848D4C
:108960000327C48D93870600B3E7E700638A070AED
:10897000EFD040489306300017C606001306C6E342
:108980009305F02E17D506001305058CEFD0103691
:108990009777FF019387076783A70700638807021C
:1089A0009727040083A7072F83A7070083A7C70083
:1089B00093860700130650029305100017C50600A2
:1089C00013058567EFC0123F6F00C00297270400B0
:1089D00083A7472C83A7070083A7C70093860700B8
:1089E000130680019305100017C50600130545679F
:1089F000EFC0523C9727040083A7C72983A707002D
:108A000083A7C700938607001306D00493051000C0
:108A100017C5060013058566EFC0D239EFD0403F79
:108A20009307F0FE232EF4FA6F00805D9777FF0125
:108A30009387C75D03A7070083A74700B716000009
:108A4000B376D7002328D48C93F70700232AF48C1D
:108A50008326048D0327448D93870600B3E7E70040
:108A6000638C070AEFD000399306300017C6060062
:108A7000130686D49305702F17C506001305C57C11
:108A8000EFD0D0269777FF019387C75783A70700BA
:108A9000638807029727040083A7C71F83A70700DF
:108AA00083A7C700938607001306F0019305100003
:108AB00017C5060013058561EFC0D22F6F00C002F5
:108AC0009727040083A7071D83A7070083A7C70074
:108AD00093860700130620019305100017C50600B2
:108AE0001305C560EFC0122D9727040083A7871ACE
:108AF00083A7070003A7C700832704F883A7C71627
:108B00001386070097C506009385855F1305070048
:108B1000EFB00262EFD0C02F930760FD232EF4FA6E
:108B20006F00004E130000006F00000113000000F2
:108B30006F00800013000000832744FB9387170019
:108B4000232AF4FA8327449583A7C700032744FB0D
:108B50006366F7DA032704FB83270495637CF70E2B
:108B60009777FF019387874A03A7070083A74700EA
:108B7000B7160000B376D7002324D48C93F70700F0
:108B80002326F48C8326848C0327C48C93870600C9
:108B9000B3E7E700638A070AEFD0C02593063000E9
:108BA00017C60600130646C19305603117C50600B7
:108BB00013058569EFD090139777FF01938787445A
:108BC00083A70700638807029727040083A7870C01
:108BD00083A7070083A7C700938607001306E00159
:108BE0009305100017C5060013054526EFC0921C1B
:108BF0006F00C0029727040083A7C70983A7070057
:108C000083A7C70093860700130610019305100081
:108C100017C5060013058525EFC0D2199727040054
:108C200083A7470783A7070083A7C700938607008A
:108C3000130640069305100017C50600130585505E
:108C4000EFC05217EFD0C01C832704F9232EF4FA8B
:108C50006F00003B8327449523A8072C8327449566
:108C60001307400023AAE72C832704976388070093
:108C7000832744951307200023AAE72C8327C49554
:108C8000638C0700832784956398070083274495A6
:108C90001307100023AAE72C8327449583A7870393
:108CA0006382070297C606009386465017C60600E1
:108CB000130686599305803217C50600130585AA49
:108CC000EFA0920F8327449503A7472D93074000F9
:108CD0006306F700232E04FA6F00003E232A04FAED
:108CE0006F0000168327449583A7C702638A070C89
:108CF0008327449503A787028327449523ACE70283
:108D00008327449583A787036386071483274495A5
:108D100003A74701832744FB93972700B307F70076
:108D200083A707002322F4F88327449583A78703AA
:108D30009305000413850700EFA092119307050027
:108D4000138707008327449523AEE702232E04F8F8
:108D50006F00C005832744F883A7472503A8C70CE5
:108D6000832744F883A687198327449503A7C7025E
:108D70008327C4F993972700B307F70083A507005B
:108D80008327449503A7C7038327C4F993976700F4
:108D9000B307F7001386070013850600E7000800F5
:108DA0008327C4F993871700232EF4F8832744956B
:108DB00083A787030327C4F9E36EF7F86F008009E0
:108DC0008327449503A74703832744FB93972700F2
:108DD000B307F70083A70700638E0704832544FBCE
:108DE00003254495EFE0404413070500832744958D
:108DF00023ACE7028327449583A787036380070694
:108E00008327449583A787039305000413850700F0
:108E1000EFA01204930705001387070083274495EA
:108E200023AEE702832544FB03254495EFE0104180
:108E30006F00C002832744FB93871700232AF4FAAC
:108E40008327449583A7C700032744FBE36CF7E817
:108E50006F000001130000006F008000130000008D
:108E60008327449583A7C700032744FB636CF70E51
:108E70009777FF019387871903A7070083A7470008
:108E8000B7160000B376D7002320D48C93F70700E1
:108E90002322F48C8326048C0327448C93870600BA
:108EA000B3E7E700638A070AEFC0D0749306300087
:108EB00017C60600130646909305303617C5060000
:108EC00013058538EFD080629777FF01938787136A
:108ED00083A70700638807029727040083A787DB1F
:108EE00083A7070083A7C700938607001306F00136
:108EF0009305100017C506001305451DEFC0826BD2
:108F00006F00C0029727040083A7C7D883A7070074
:108F100083A7C7009386070013062001930510005E
:108F200017C506001305851CEFC0C268972704000B
:108F300083A747D683A7070083A7C70093860700A8
:108F4000130630039305100017C506001305C52747
:108F5000EFC04266EFC0D06B930760FD232EF4FA9A
:108F60006F00000A232404FA6F0000088327449549
:108F700083A6C7008327449503A7C703832784FAE2
:108F800093976700B304F70093050001138506006B
:108F9000EFA0026C9307050023A6F40283274495F3
:108FA00083A7C702639C0702232A04FA6F0000020A
:108FB000032644FB832584FA03254495EF500101E1
:108FC000832744FB93871700232AF4FA83274495C9
:108FD00083A7C700032744FBE36CF7FC832784FACD
:108FE000938717002324F4FA8327449583A78703E4
:108FF000032784FAE36CF7F6232E04FA6F00C00B04
:1090000003254495EFE08F9C8327449523A0070414
:10901000232A04FA6F00C0068327449583A787019B
:10902000638A07048327449503A74702832744FBE9
:1090300093972700B307F70083A70700138507005E
:10904000EFC012198327449503A74702832744FBE7
:1090500093972700B307F70023A0070083274495C1
:1090600003A70702832744FB93972700B307F70062
:1090700023A00700832744FB93871700232AF4FAD1
:109080008327449583A7C700032744FBE366F7F8CB
:109090006F00800013000000032744FA83278494A4
:1090A0006306F700032544FAEFC092128327449524
:1090B0001307E0FF23A8E72C8327449583A74700E5
:1090C00063D2070297C606009386461317C60600AA
:1090D000130686179305B03817B506001305856883
:1090E000EFA0824D032584FBEFC0920E232C04FADF
:1090F0008327C400638A07008327C40083250401F3
:1091000003254495E78007008327C4FB13850700E8
:109110008320C1740324817483244174032901745E
:109120008329C173032A8173832A4173032B01733B
:10913000832BC172032C8172832C4172032D017227
:10914000832DC1711301017567800000130101FBBC
:109150002326110423248104232221052320310501
:10916000232E4103232C5103232A61032328710357
:10917000232681032324910313040105232EA4FA3B
:10918000232CB4FA232AC4FA232604FC232404FC47
:10919000832684FB6394060E9777FF01938707E786
:1091A00003A7070083A74700B7160000337CD7004A
:1091B00093FC070093070C00B3E79701638A070A43
:1091C000EFC050439306300017260700130686951C
:1091D0009305000317250700130545C8EFD000319C
:1091E0009777FF01938707E283A707006388070249
:1091F0009727040083A707AA83A7070083A7C700B0
:10920000938607001306E001930510001725070059
:109210001305C591EFC0023A6F00C0029727040002
:1092200083A747A783A7070083A7C70093860700E4
:10923000130610019305100017250700130505916B
:10924000EFC042379727040083A7C7A483A707006E
:1092500083A7C700172607001306869097250700E7
:109260009385859113850700EFA0926CEFC0503A6B
:10927000930720FE2324F4FC6F0090108326C4FB88
:109280006394060E9777FF01938747D803A70700DB
:1092900083A74700B7160000337FD70093FF07006E
:1092A00093070F00B3E7F701638A070AEFC0903412
:1092B00093063000172607001306C6869305200381
:1092C00017250700130585B9EFD040229777FF01D6
:1092D000938747D383A70700638807029727040073
:1092E00083A7479B83A7070083A7C7009386070030
:1092F00013060002930510001725070013050588C3
:10930000EFC0422B6F00C0029727040083A7879805
:1093100083A7070083A7C7009386070013063001C1
:10932000930510001725070013058587EFC08228D5
:109330009727040083A7079683A7070083A7C70082
:109340001726070013060687972507009385C58211
:1093500013850700EFA0D25DEFC0902B930740FD6F
:109360002324F4FC6F00D0018326C4FB83A6C6002F
:109370006394060E9777FF01938747C903A70700F9
:1093800083A74700B7160000337ED70093FE07007F
:1093900093070E00B3E7D701638A070AEFC0902551
:1093A00093063000171607001306C677930540038F
:1093B00017250700130585AAEFD040139777FF0103
:1093C000938747C483A70700638807029727040091
:1093D00083A7478C83A7070083A7C700938607004E
:1093E00013060002930510001715070013050579F1
:1093F000EFC0421C6F00C0029727040083A7878933
:1094000083A7070083A7C7009386070013063001D0
:10941000930510001715070013058578EFC0821912
:109420009727040083A7078783A7070083A7C700A0
:10943000938607001306A002930510001715070076
:1094400013058578EFC00217EFC0901C930740FD0D
:109450002324F4FC6F00C0728326C4FB03A6062DF0
:109460009306F0FF6314D60E9777FF01938707BA30
:1094700003A7070083A74700B71600003373D70080
:1094800093F3070093070300B3E77700638A070AA3
:10949000EFC05016930630001716070013068668B3
:1094A00093057003172507001305459BEFD00004B3
:1094B0009777FF01938707B583A7070063880702A3
:1094C0009717040083A7077D83A7070083A7C7001A
:1094D000938607001306B0029305100017150700C6
:1094E00013054571EFC0020D6F00C002971704000D
:1094F00083A7477A83A7070083A7C700938607003F
:109500001306E001930510001715070013054571B8
:10951000EFC0420A9717040083A7C77783A7070005
:1095200083A7C700938607001306E0049305100085
:10953000171507001305C570EFC0C207EFC0500D27
:10954000930730FD2324F4FC6F0080638326C4FB63
:1095500083A6062D6384060E9777FF01938707ABDA
:1095600003A7070083A74700B71600003378D7008A
:1095700093F8070093070800B3E71701638A070A07
:10958000EFC05007930630001716070013068659E0
:109590009305B003172507001305458CEFC0107520
:1095A0009777FF01938707A683A7070063880702C1
:1095B0009717040083A7076E83A7070083A7C70038
:1095C000938607001306B0029305100017150700D5
:1095D00013054562EFB0127E6F00C00297170400BA
:1095E00083A7476B83A7070083A7C700938607005D
:1095F0001306E001930510001715070013054562D7
:10960000EFB0527B9717040083A7C76883A70700B2
:1096100083A7C70093860700130670029305100006
:10962000171507001305C566EFB0D278EFC0407E6E
:10963000930730FD2324F4FC6F0080548326C4FB81
:1096400083A6C602639A060E8326C4FB83A6C62C95
:109650006394060E9776FF019386469B03A6060049
:1096600083A64600B71500003377B60093F70600CF
:1096700093060700B3E6F600638A060AEFC0807718
:1096800093063000171607001306C6499305E0033A
:10969000171507001305857CEFC050659777FF010C
:1096A0009387479683A707006388070297170400EC
:1096B00083A7475E83A7070083A7C7009386070099
:1096C0001306B00293051000171507001305855205
:1096D000EFB0526E6F00C0029717040083A7875B3C
:1096E00083A7070083A7C700938607001306E0013E
:1096F000930510001715070013058552EFB0926B04
:109700009717040083A7075983A7070083A7C700FB
:10971000938607001306D004930510001715070061
:1097200013058559EFB01269EFC0806E930730FDC5
:109730002324F4FC6F00C0449305000213051000BD
:10974000EF901271930705002326F4FC8327C4FCD5
:109750006394070E9777FF019387478B03A7070052
:1097600083A74700B7160000337BD70093FB0700A1
:1097700093070B00B3E77701638A070AEFC080679E
:1097800093063000171607001306C63993055004D8
:10979000171507001305856CEFC050559777FF012B
:1097A0009387478683A707006388070297170400FB
:1097B00083A7474E83A7070083A7C70093860700A8
:1097C0001306300293051000171507001305C55343
:1097D000EFB0525E6F00C0029717040083A7874B5B
:1097E00083A7070083A7C7009386070013066001BD
:1097F000930510001715070013054553EFB0925B52
:109800009717040083A7074983A7070083A7C7000A
:1098100093860700130670029305100017150700C2
:1098200013054552EFB01259EFC0805E9307A0FFB9
:109830002324F4FC6F00C0348327C4FC13071000FA
:1098400023A2E700232204FC6F00C0038327C4FB8C
:1098500003A7C703832744FC93976700B307F70068
:1098600083A7C700832584FB13850700EFE09224BC
:109870009307050063820702832744FC9387170040
:109880002322F4FC8327C4FB83A78703032744FC1C
:10989000E36EF7FA6F008000130000008327C4FB1B
:1098A00083A78703032744FC6362F70E9767FF01D2
:1098B0009387C77503A7070083A74700B716000063
:1098C000337AD70093FA070093070A00B3E75701EA
:1098D0006388070AEFC0005293063000171607008E
:1098E000130646249305E0041715070013050557D2
:1098F000EFC0D03F9767FF019387C77083A707002A
:10990000638807029717040083A7C73883A7070057
:1099100083A7C70093860700130640029305100033
:109920001715070013058544EFB0D2486F00C00239
:109930009717040083A7073683A7070083A7C700EC
:109940009386070013067001930510001715070092
:1099500013054544EFB012469717040083A78733D9
:1099600083A7070083A7C700032684FB971507007A
:109970009385C54313850700EFA0827BEFC0404964
:10998000930720FD2324F4FC6F00801F8327C4FB72
:1099900003A7C703832744FC939767003307F700A7
:1099A0008327C4FC23A8E7008327C4FC83A70701FF
:1099B00003A7C7008327C4FC23AAE7008327C4FBAF
:1099C00003A787008327C4FC23A4E7008327C4FCE4
:1099D0000327C4FB23A6E7008327C4FC83A7070152
:1099E00083A707009305800113850700EF90524677
:1099F00093070500138707008327C4FC23ACE70007
:109A00008327C4FC83A787016394070E9767FF0130
:109A10009387C75F03A7070083A74700B716000017
:109A20003379D70093F9070093070900B3E73701AB
:109A3000638A070AEFC0003C930630001716070040
:109A40001306460E930590051715070013050541EB
:109A5000EFC0D0299767FF019387C75A83A70700F4
:109A6000638807029717040083A7C72283A707000C
:109A700083A7C700938607001306300293051000E2
:109A80001715070013054528EFB0D2326F00C0024A
:109A90009717040083A7072083A7070083A7C700A1
:109AA0009386070013066001930510001715070041
:109AB0001305C527EFB012309717040083A7871D41
:109AC00083A7070083A7C7001716070013064631B0
:109AD000971507009385450A13850700EFA0426597
:109AE000EFC000339307A0FF2324F4FC6F0040096C
:109AF0008327C4FB83A747006342F0029716070041
:109B00009386063017160700130646359305C005E1
:109B1000171507001305C530EF90122A8327C4FBE1
:109B200003A707048327C4FC23AEE7008327C4FBF5
:109B30000327C4FC23A0E7048327C4FB83A74700B3
:109B4000138717008327C4FB23A2E7008327C4FBE6
:109B500083A7470063D20702971607009386062E55
:109B6000171607001306862F9305F0051715070033
:109B70001305052BEF905224232404FC6F004003AF
:109B80008327C4FC638E07008327C4FC83A7870157
:109B900013850700EFB0D2638327C4FC23AC070012
:109BA0000325C4FCEFB0D262232604FC232604FC68
:109BB000832744FB63880700832744FB032784FC37
:109BC00023A0E7008327C4FC138507008320C1047A
:109BD000032481040329410483290104032AC103C6
:109BE000832A8103032B4103832B0103032CC1022E
:109BF000832C81021301010567800000130101FD20
:109C0000232611022324810223222103232031034E
:109C100013040103232EA4FC8325C4FD6392050EC7
:109C20009767FF019387873E03A7070083A7470035
:109C3000B71500003376B70093F6070093070600C8
:109C4000B3E7D700638A070AEFC0C01A9306300053
:109C500017560700130686FB9305100217550700D9
:109C60001305C50EEFC090089767FF0193878739EA
:109C700083A70700638807029717040083A787015B
:109C800083A7070083A7C700938607001306F00188
:109C900093051000175507001305C5F7EFB0921193
:109CA0006F00C0029717040083A7C7FE83A70700B1
:109CB00083A7C700938607001306200193051000B1
:109CC00017550700130505F7EFB0D20E97170400DC
:109CD00083A747FC83A7070083A7C7001756070081
:109CE000130686F697550700938545F713850700F9
:109CF000EFA00244EFC0C011930700FD6F00003BCE
:109D00008326C4FD83A646006342D002975607000F
:109D1000938606F51756070013064603930520029F
:109D200017550700130585F5EF9012098326C4FD2A
:109D300083A646009386F6FF0326C4FD2322D600A1
:109D40002322D4FE8326C4FD83A6460063D20602E6
:109D500097560700938646F417560700130606FF2A
:109D60009305200217550700130545F1EF90D20423
:109D70009766FF019386862903A6060083A6460000
:109D80001377060493F7060093060700B3E6F60080
:109D90006384060AEFC000069306100017560700FA
:109DA000130686F19305300217550700130505FACF
:109DB000EFC0C0739767FF019387C72483A707008D
:109DC000638807029717040083A7C7EC83A70700DF
:109DD00083A7C700938607001306E00093051000D1
:109DE00017550700130505EEEFB0C27C6F000002A7
:109DF0009717040083A707EA83A7070083A7C70074
:109E00009385070013050002EFA0023D9717040099
:109E100083A747E883A7070083A7C700832644FEDC
:109E20000326C4FD975507009385C5EA13850700EF
:109E3000EFA00230EFB0D07D832744FE6396072663
:109E40009767FF019387871C03A7070083A7470035
:109E50001379070493F9070093070900B3E7370163
:109E60006382070AEFB010799306100017560700B7
:109E7000130686E49305700217550700130505EDD8
:109E8000EFC0C0669767FF019387C71783A70700D6
:109E9000638807029717040083A7C7DF83A707001B
:109EA00083A7C700938607001306E0009305100000
:109EB00017550700130505E1EFB0C26F6F000002F0
:109EC0009717040083A707DD83A7070083A7C700B0
:109ED0009385070013050002EFA0023097170400D6
:109EE00083A747DB83A7070083A7C7000326C4FD1A
:109EF00097550700938585DF13850700EFA0422360
:109F0000EFB010718327C4FD83A7C7002320F4FEA0
:109F1000832704FE6392070297560700938606DEA6
:109F200017560700130686E293059002175507009F
:109F30001305C5D4EF904268832704FE83A747002A
:109F40006342F00297560700938646DC17560700D7
:109F50001306C6DF9305C00217550700130505D287
:109F6000EF908265832704FE83A707040327C4FDBF
:109F7000631EF700832704FE83A7070403A7C70116
:109F8000832704FE23A0E7046F008005832704FED7
:109F900083A707042324F4FE6F000001832784FEB7
:109FA00083A7C7012324F4FE832784FE83A7C70168
:109FB000638A0700832784FE83A7C7010327C4FDA4
:109FC000E31EF7FC832784FE83A7C701638A07008B
:109FD0008327C4FD03A7C701832784FE23AEE700C0
:109FE0008327C4FD83A78701638C0704232604FE0F
:109FF0006F00C0038327C4FD83A687010327C4FE27
:10A000009307070093971700B387E70093973700EC
:10A01000B387F60083A7070113850700EF60901749
:10A020008327C4FE938717002326F4FE8327C4FDED
:10A0300083A7070183A707000327C4FEE36CF7FA91
:10A040008327C4FD23AA07008327C4FD23A8070094
:10A050008327C4FD83A7870113850700EFB052173C
:10A060008327C4FD23AC07000325C4FDEFB05216BF
:10A07000232E04FC832704FE83A7470063D2070234
:10A0800097560700938686CA17560700130606CC14
:10A090009305A00317550700130545BEEF90C25165
:10A0A000032504FEEFB0CFEA9307000013850700F5
:10A0B0008320C10203248102032941028329010272
:10A0C0001301010367800000130101F72326110823
:10A0D000232481082322210923203109232E41072B
:10A0E000232C5107232A6107232871072326810780
:10A0F000232491072322A1072320B1071304010978
:10A10000232EA4F8232CB4F8232AC4F82328D4F847
:10A110008326C4F96392060E9767FF01938707EFC2
:10A1200003A7070083A74700B7160000337ED700B8
:10A1300093FE070093070E00B3E7D701638A070A6F
:10A14000EFB0504B93063000178607001306867455
:10A150009305C00217950700130585B0EFC00039BD
:10A160009767FF01938707EA83A7070063880702C1
:10A170009717040083A707B283A7070083A7C70028
:10A18000938607001306F00193051000178507005A
:10A190001305C570EFB002426F00C00297170400AC
:10A1A00083A747AF83A7070083A7C700938607004D
:10A1B000130620019305100017850700130505708D
:10A1C000EFB0423F9717040083A7C7AC83A70700EF
:10A1D00083A7C700178607001306866F97850700B9
:10A1E0009385457013850700EF909274EFB050424D
:10A1F000930700FD6F0090378326C4F983A60601FC
:10A2000083A60600032684F96368D60E9767FF01CC
:10A210009387C7DF03A7070083A74700B71600008F
:10A220003373D70093F3070093070300B3E7770076
:10A230006380070CEFB0103C9306300017860700D0
:10A24000130646659305E00217950700130545A11F
:10A25000EFC0C0299767FF019387C7DA83A707007C
:10A26000638807029717040083A7C7A283A7070084
:10A2700083A7C700938607001306200293051000EA
:10A280001785070013054566EFB0C2326F00C002A4
:10A290009717040083A707A083A7070083A7C70019
:10A2A00093860700130650019305100017850700D9
:10A2B0001305C565EFB002309717040083A7879D8B
:10A2C00083A7070003A7C7008327C4F983A7070153
:10A2D00083A70700832684F9138607009785070064
:10A2E0009385456413050700EF909264EFB05032F8
:10A2F0009307F0FC6F0090278326C4F983A686019C
:10A300006392060E9767FF01938747D003A7070064
:10A3100083A74700B71600003378D70093F80700EB
:10A3200093070800B3E71701638A070AEFB0902C80
:10A3300093063000178607001306C65593053003B1
:10A34000179507001305C591EFC0401A9767FF01E5
:10A35000938747CB83A707006388070297170400FA
:10A3600083A7479383A7070083A7C70093860700A7
:10A370001306F00193051000178507001305055219
:10A38000EFB042236F00C0029717040083A78790A5
:10A3900083A7070083A7C700938607001306200141
:10A3A000930510001785070013054551EFB0822073
:10A3B0009717040083A7078E83A7070083A7C7000A
:10A3C000938607001306F002930510001785070017
:10A3D00013050558EFB0021EEFB09023930700FD60
:10A3E0006F00D0188326C4F983A6060103A6460190
:10A3F000832684F993965600B306D600232CD4FA0C
:10A40000832684FB03A68600B7F6FFFF938646E605
:10A41000B306D60093B6160093F6F60F232AD4FAA5
:10A420009766FF01938686BE03A5060083A54600B6
:10A4300093060500B3E6B60063860614232204FCE7
:10A44000832684FB03A6860193061000630AD600C8
:10A45000832684FB03A6860193062000631CD60096
:10A46000832604F963880600832604F983A6060080
:10A470002322D4FC232004FC832604F9638E0600E7
:10A48000032644F9930640006318D600832604F996
:10A4900083A606002320D4FC9766FF01938606B7A7
:10A4A00003A6060083A646001377160093F706005E
:10A4B00093060700B3E6F6006386060CEFB0901330
:10A4C00093061000178607001306864B9305500469
:10A4D000178507001305C578EFC040019767FF0196
:10A4E000938747B283A70700638807029707040092
:10A4F00083A7477A83A7070083A7C700938607002F
:10A500001306E00093051000178507001305C547E3
:10A51000EFB0420A6F0000029707040083A7877715
:10A5200083A7070083A7C7009385070013050002D0
:10A53000EF90924A9707040083A7C77583A7070087
:10A5400003A5C7008327C4F903A64701832784FB1B
:10A5500003A70700832704FC2322F100832744FC80
:10A560002320F100832804F9032844F9832744FBBE
:10A57000832684F99785070093850542EF90523B27
:10A58000EFB01009832704F9638C070E832744FB7F
:10A590006388070E9767FF01938747A703A7070004
:10A5A00083A74700B7160000B376D7002324D4F85A
:10A5B00093F707002326F4F8832684F80327C4F8CA
:10A5C00093870600B3E7E7006388070AEFB09002BD
:10A5D00093063000178607001306C62B9305C004A8
:10A5E000178507001305C567EFB050709767FF0127
:10A5F000938747A183A70700638807029707040092
:10A6000083A7476983A7070083A7C700938607002E
:10A610001306200293051000178507001305053F58
:10A62000EFA052796F00C0029707040083A78766E6
:10A6300083A7070083A7C70093860700130650016E
:10A6400093051000178507001305853EEFA092764D
:10A650009707040083A7076483A7070083A7C700A1
:10A66000032684F9978507009385053E1385070027
:10A67000EF90122CEFB0C0799307E0FC6F00006FF1
:10A68000832704F9639C070E832744FB6398070E16
:10A69000832784FB03A78701930710006300F70E4D
:10A6A0009767FF019387879603A7070083A7470053
:10A6B000B7160000337DD70093FD070093070D0008
:10A6C000B3E7B7016388070AEFB0C07293063000A2
:10A6D000178607001306061C93052005178507003B
:10A6E00013050558EFB090609767FF019387879136
:10A6F00083A70700638807029707040083A7875989
:10A7000083A7070083A7C7009386070013062002CC
:10A7100093051000178507001305452FEFA09269D8
:10A720006F00C0029707040083A7C75683A70700DE
:10A7300083A7C700938607001306500193051000F6
:10A74000178507001305C52EEFA0D26697070400F2
:10A7500083A7475483A7070083A7C700032684F96C
:10A76000978507009385C53113850700EF90521C2C
:10A77000EFB0006A9307E0FC6F00405F832744F965
:10A780006394070E832744FB6380070E9767FF01DE
:10A790009387C78703A7070083A74700B716000062
:10A7A000337CD70093FC070093070C00B3E79701B5
:10A7B0006388070AEFB0006493063000178607002D
:10A7C0001306460D9305B005178507001305454987
:10A7D000EFB0D0519767FF019387C78283A7070027
:10A7E000638807029707040083A7C74A83A7070067
:10A7F00083A7C70093860700130610029305100075
:10A80000178507001305852BEFA0D25A6F00C002F1
:10A810009707040083A7074883A7070083A7C700FB
:10A820009386070013064001930510001785070063
:10A830001305052BEFA012589707040083A787453F
:10A8400083A7070083A7C700032684F9978507001D
:10A850009385852A13850700EF90920DEFB0405B3A
:10A860009307D0FC6F008050832784FB03A78701E8
:10A87000930730006316F70E832704F96392070EDF
:10A880009757FF019387877803A7070083A747009F
:10A89000B7160000337BD70093FB070093070B002C
:10A8A000B3E77701638A070AEFB0C054930630001C
:10A8B00017860700130606FE9305F00517850700A7
:10A8C0001305053AEFB090429757FF0193878773BE
:10A8D00083A70700638807029707040083A7873BC5
:10A8E00083A7070083A7C70093860700130600020B
:10A8F000930510001785070013054523EFA0924B21
:10A900006F00C0029707040083A7C73883A707001A
:10A9100083A7C70093860700130630019305100034
:10A92000178507001305C522EFA0D248970704003A
:10A9300083A7473683A7070083A7C700938607002E
:10A940001306A00293051000178507001305852143
:10A95000EFA05246EFB0C04B930770FD6F0000416F
:10A96000832784FB03A78701930710006302F70284
:10A97000832784FB03A7870193072000630AF7005E
:10A98000832784FB03A7870193073000631AF70E20
:10A99000832744FB63920722032744F9930740006F
:10A9A000630CF7209757FF019387476603A70700BB
:10A9B00083A74700B7160000337AD70093FA070041
:10A9C00093070A00B3E757016388070AEFB0804294
:10A9D00093063000178607001306C6EB9305500652
:10A9E000178507001305C527EFB050309757FF01B3
:10A9F0009387476183A707006388070297070400CE
:10AA000083A7472983A7070083A7C700938607006A
:10AA10001306100293051000178507001305050A99
:10AA2000EFA052396F00C0029707040083A7872662
:10AA300083A7070083A7C70093860700130640017A
:10AA4000930510001785070013058509EFA09236BE
:10AA50009707040083A7072483A7070083A7C700DD
:10AA6000032684F9978507009385851213850700CF
:10AA7000EF90026CEFB0C0399307D0FC6F00002F4D
:10AA8000832784FB83A7C701638A0712832744F9BE
:10AA9000232EF4FA0327C4FB93073000B377F702A1
:10AAA000639C07000327C4FB93073000B357F702EA
:10AAB00093972700232EF4FA832784FB83A7C701EB
:10AAC0000327C4FB630CF70E9757FF0193870754C6
:10AAD00003A7070083A74700B71600003379D70004
:10AAE00093F9070093070900B3E737016382070C66
:10AAF000EFB040309306300017860700130686D962
:10AB0000930500071785070013058515EFB0101E84
:10AB10009757FF019387074F83A7070063880702B2
:10AB20009707040083A7071783A7070083A7C70019
:10AB3000938607001306100293051000178507007F
:10AB40001305C5F7EFA012276F00C0029707040096
:10AB500083A7471483A7070083A7C700938607002E
:10AB6000130640019305100017850700130545F7EC
:10AB7000EFA052249707040083A7C71183A70700FB
:10AB800003A5C700832784FB83A60700832784FBD4
:10AB900003A70700832784FB83A7C701032684F943
:10ABA0009785070093850503EF908258EFB0402604
:10ABB0009307D0FC6F00801B130000008327C4F9AB
:10ABC00083A68701032784F993070700939717004B
:10ABD000B387E70093973700B387F6002328F4FA8A
:10ABE0008327C4F983A747006342F00297860700D2
:10ABF000938686011786070013068606930570075D
:10AC00001785070013050502EF80121B832704FB3D
:10AC100023AA0700832704F96380070E832784FB98
:10AC200003A78701930710006318F700832704F92F
:10AC300083A707006382070C832704FB83A7070110
:10AC400013850700EF501055832704FB23A8070046
:10AC5000032544F9EF5050232326A4FC0327C4FC0A
:10AC60009307F00763F6E700930700082326F4FC38
:10AC7000832744F92324F4FC032784FC8327C4FCA2
:10AC80006376F7008327C4FC2324F4FC832584FC2B
:10AC90000325C4FCEF50D0462326A4FA8327C4FA28
:10ACA000639C07028327C4F983A7470063D2070286
:10ACB000978607009386C6F817860700130646FA9C
:10ACC0009305E008178507001305C5F5EF80D20E40
:10ACD0009307A0FF6F008009032644F9832504F938
:10ACE0000325C4FAEFB00260832704FB0327C4FAEC
:10ACF00023A8E7006F00C001832704FB83A7070197
:10AD000013850700EF501049832704FB23A8070091
:10AD1000832744F92320F4F8232204F8832704FB33
:10AD2000832604F8032744F823A0D70023A2E700D2
:10AD3000832704FB1307100023AAE7008327C4F925
:10AD400083A7470063D2070297860700938646EFE2
:10AD5000178607001306C6F09305400A17850700FB
:10AD6000130545ECEF80520593070000138507009B
:10AD70008320C1080324810803294108832901088D
:10AD8000032AC107832A8107032B4107832B01076D
:10AD9000032CC106832C8106032D4106832D010659
:10ADA0001301010967800000130101FD23268102C0
:10ADB00013040103232EA4FC232CB4FC6F004002D7
:10ADC0008327C4FD2326F4FE032784FD8327C4FDC7
:10ADD000B377F702232EF4FC8327C4FE232CF4FC64
:10ADE0008327C4FDE39E07FC832784FD13850700AA
:10ADF0000324C1021301010367800000130101FE57
:10AE0000232E1100232C8100130401022326A4FE0B
:10AE10002324B4FE0327C4FE832784FE6376F70051
:10AE20008327C4FE6F00C004832784FE6398070253
:10AE300097C60700938686D317C607001306466693
:10AE40009305500417C50700130505D3EF80C2769C
:10AE5000832784FE9387F7FF2324F4FE0327C4FE91
:10AE6000832784FEB377F702E39407FE832784FEEB
:10AE7000138507008320C10103248101130101020E
:10AE800067800000130101FE232E810013040102DC
:10AE90002326A4FE2324B4FE2322C4FE032784FE1B
:10AEA0008327C4FEB377F702639E0700032744FE9F
:10AEB000832784FEB377F702639607009307100099
:10AEC0006F00800093070000138507000324C10171
:10AED0001301010267800000130101E12326111E06
:10AEE0002324811E2322911E2320211F232E311D66
:10AEF000232C411D232A511D2328611D2326711D4A
:10AF00002324811D2322911D2320A11D232EB11B4B
:10AF10001304011F2326A4F02324B4F02322C4F039
:10AF20002320D4F0232EE4EE232CF4EE232A04EF86
:10AF3000232814EF930701002322F4E2232A04FAC2
:10AF4000832744FB2328F4FA832704FB2326F4FAFF
:10AF5000232A04F6832744F72328F4F6832704F7EB
:10AF60002326F4F6232404FA832784FA232EF4FA02
:10AF70008327C4FB232CF4FA232C04F8232404F69F
:10AF8000832784F083A7070183A70700138717008F
:10AF9000930707009387F7FF2322F4F6130F0700A8
:10AFA000930F00009357BF0193935F00B3E37700C3
:10AFB00013135F0013090700930900009357B901A9
:10AFC000939E5900B3EED701131E59009317270023
:10AFD0009387F70093D74700939747003301F140D9
:10AFE000930781009387370093D727009397270013
:10AFF0002320F4F6832784F083A7070103A7070023
:10B00000832744EFB307F700138717009307070060
:10B010009387F7FF232EF4F4130C0700930C000022
:10B020009357BC01939A5C00B3EA5701131A5C0072
:10B03000130D0700930D00009357BD01939B5D0016
:10B04000B3EB7701131B5D00931727009387F7007D
:10B0500093D74700939747003301F140930781004E
:10B060009387370093D7270093972700232CF4F476
:10B070008327C4F0639A070E9757FF01938707F958
:10B0800003A7070083A74700B7160000B376D700D1
:10B090002324D4EE93F707002326F4EE832684EED0
:10B0A0000327C4EE93870600B3E7E700638A070A25
:10B0B000EFA050549306300017C60700130606AEE3
:10B0C0009305400717C507001305C53BEFB00042C5
:10B0D0009757FF01938707F383A707006388070249
:10B0E0009707040083A707BB83A7070083A7C700B0
:10B0F00093860700130660029305100017C507002A
:10B10000130545AAEFA0024B6F00C0029707040089
:10B1100083A747B883A7070083A7C70093860700C4
:10B12000130690019305100017C50700130505AA23
:10B13000EFA042489707040083A7C7B583A707007D
:10B1400083A7C70017C60700130606AA97C50700FE
:10B15000938505AB13850700EF80927DEFA0504BE0
:10B160009307C0FD6F204054832784F0639A070E35
:10B170009757FF01938787E903A7070083A7470035
:10B18000B7160000B376D7002320D4EE93F707005C
:10B190002322F4EE832604EE032744EE9387060071
:10B1A000B3E7E700638A070AEFA0D04493063000B4
:10B1B00017C607001306869E9305600717C507008C
:10B1C0001305452CEFB080329757FF01938787E333
:10B1D00083A70700638807029707040083A787AB4C
:10B1E00083A7070083A7C700938607001306F00113
:10B1F0009305100017C507001305C5A0EFA0823BFB
:10B200006F00C0029707040083A7C7A883A70700A1
:10B2100083A7C7009386070013062001930510003B
:10B2200017C50700130505A0EFA0C2389707040053
:10B2300083A747A683A7070083A7C70017C60700F1
:10B240001306869F97C507009385859B1385070086
:10B25000EF80126EEFA0D03B930700FD6F20C0443B
:10B260008327C4F003A78700832784F083A7870080
:10B27000630AF70E9757FF01938747D903A7070083
:10B2800083A74700B7160000B376D700232CD4EC71
:10B2900093F70700232EF4EC832684ED0327C4EDF7
:10B2A00093870600B3E7E700638A070AEFA09034AC
:10B2B0009306300017C607001306468E93058007D5
:10B2C00017C507001305051CEFB040229757FF0173
:10B2D000938747D383A70700638807029707040073
:10B2E00083A7479B83A7070083A7C7009386070010
:10B2F000130600029305100017C5070013050595F6
:10B30000EFA0422B6F00C0029707040083A7879825
:10B3100083A7070083A7C7009386070013063001A1
:10B320009305100017C5070013058594EFA0822828
:10B330009707040083A7079683A7070083A7C70082
:10B3400093860700130670039305100017C50700C6
:10B3500013054593EFA00226EFA0902B9307E0FD85
:10B360006F208034032604EF832544EF0325C4F0C7
:10B37000EF801030232CA4F8832784F9638607001C
:10B38000832784F96F204032832744F0639A070EA5
:10B390009757FF01938787C703A7070083A7470035
:10B3A000B7160000B376D7002328D4EC93F7070034
:10B3B000232AF4EC832604ED032744ED938706004B
:10B3C000B3E7E700638A070AEFA0D02293063000B4
:10B3D00017B607001306867C9305100817C50700EB
:10B3E0001305450AEFB080109757FF01938787C177
:10B3F00083A70700638807029707040083A787894C
:10B4000083A7070083A7C70093860700130670026F
:10B410009305100017C507001305458AEFA0821990
:10B420006F00C0029707040083A7C78683A70700A1
:10B4300083A7C700938607001306A0019305100099
:10B4400017C507001305058AEFA0C2169707040069
:10B4500083A7478483A7070083A7C70017C60700F1
:10B460001306068A97B5070093858579138507002B
:10B47000EF80124CEFA0D0199307B0FC6F20C022D0
:10B480008327C4F083A7C70003A74702832744F09C
:10B49000637AF70E9757FF01938747B703A7070013
:10B4A00083A74700B7160000B376D7002324D4EC57
:10B4B00093F707002326F4EC832684EC0327C4ECDF
:10B4C00093870600B3E7E700638A070AEFA09012AC
:10B4D0009306300017B607001306466C9305200844
:10B4E00017C50700130505FAEFB040009757FF0195
:10B4F000938747B183A707006388070297F7030084
:10B5000083A7477983A7070083A7C700938607000F
:10B51000130670029305100017B507001305057A8E
:10B52000EFA042096F00C00297F7030083A7877658
:10B5300083A7070083A7C700938607001306A0010F
:10B540009305100017B507001305C579EFA0820613
:10B5500097F7030083A7077483A7070083A7C70093
:10B5600093860700130620039305100017B5070004
:10B570001305057AEFA00204EFA090099307B0FC31
:10B580006F2080128327C4F083A7C70003A7470258
:10B590009307300063F2E70297B607009386867A36
:10B5A00017C60700130606EE9305700817B50700C7
:10B5B0001305855CEF8042008327C4F083A7C70092
:10B5C00013850700EF80C01A2324A4F6832704F014
:10B5D000638E0704832704F083A707002326F4FA69
:10B5E000032744F09307100063FAE700832704F071
:10B5F0009387470083A707006F0080009307000030
:10B600002328F4FA032744F09307200063FAE700A5
:10B61000832704F09387870083A707006F008000CB
:10B6200093070000232AF4FA6F000001232604FA8E
:10B63000232804FA232A04FA8327C4EF83A70700E8
:10B640002326F4F6032744F09307100063FAE7007B
:10B650008327C4EF9387470083A707006F0080000C
:10B66000930710002328F4F6032744F093072000E3
:10B6700063FAE7008327C4EF9387870083A7070057
:10B680006F00800093071000232AF4F68327C4F686
:10B69000638A0700832704F763860700832744F73C
:10B6A000639A070E9757FF019387479603A70700F2
:10B6B00083A74700B7160000B376D7002320D4EC49
:10B6C00093F707002322F4EC832604EC032744ECD1
:10B6D00093870600B3E7E700638A070AEFA080714B
:10B6E0009306300017B607001306464B9305C009B2
:10B6F00017C50700130505D9EFA0505F9757FF0145
:10B700009387479083A707006388070297F7030092
:10B7100083A7475883A7070083A7C700938607001E
:10B72000130690029305100017B507001305056571
:10B73000EF9052686F00C00297F7030083A7875508
:10B7400083A7070083A7C700938607001306C001DD
:10B750009305100017B5070013050565EF90926576
:10B7600097F7030083A7075383A7070083A7C700A2
:10B7700017B607001306466597B507009385454839
:10B7800013850700EF80D21AEFA08068930710FCA2
:10B790006F1090718327C4F083A7C70083A7C702E7
:10B7A000232AF4F4032744F09307100063FAE70018
:10B7B0008327C4F083A7C70083A707036F00800017
:10B7C000930710002328F4F4032744F09307200084
:10B7D00063FAE7008327C4F083A7C70083A7470362
:10B7E0006F008000930710002326F4F48327C4F031
:10B7F00083A7C70083A787032324F4F4832784EF58
:10B8000063880776832784EF83A70700232CF4FA45
:10B81000032744F09307100063FAE700832784EFBF
:10B820009387470083A707006F00800093071000ED
:10B83000232EF4FA032744F09307200063FAE7006D
:10B84000832784EF9387870083A707006F0080001A
:10B85000930710002324F4FA032784FB8327C4FBF7
:10B860003307F702832784FA3307F702832784F428
:10B8700063FAE70E9747FF019387477903A707000D
:10B8800083A74700B7160000B376D700232CD4EA6D
:10B8900093F70700232EF4EA832684EB0327C4EBF7
:10B8A00093870600B3E7E700638A070AEFA0805496
:10B8B0009306300017B607001306462E9305C00AFC
:10B8C00017C50700130505BCEFA050429747FF01BD
:10B8D0009387477383A707006388070297F70300DE
:10B8E00083A7473B83A7070083A7C700938607006A
:10B8F000130680029305100017B5070013050550C5
:10B90000EF90524B6F00C00297F7030083A7873870
:10B9100083A7070083A7C700938607001306B0011B
:10B920009305100017B5070013050550EF909248D6
:10B9300097F7030083A7073683A7070083A7C700ED
:10B94000938607001306D0039305100017B5070070
:10B950001305454FEF901246EFA0804B9307A0FCD4
:10B960006F109054032784FB832744F563FAE70E96
:10B970009747FF019387876903A7070083A74700BD
:10B98000B7160000B376D7002328D4EA93F7070050
:10B99000232AF4EA832604EB032744EB938706006B
:10B9A000B3E7E700638A070AEFA0C04493063000BC
:10B9B00017B607001306861E9305000B17C5070070
:10B9C000130545ACEFA090329747FF01938787633B
:10B9D00083A707006388070297F7030083A7872BD5
:10B9E00083A7070083A7C70093860700130670028A
:10B9F0009305100017B507001305C548EF90923B5B
:10BA00006F00C00297F7030083A7C72883A707002A
:10BA100083A7C700938607001306A00193051000B3
:10BA200017B5070013058548EF90D23897F7030044
:10BA300083A7472683A7070083A7C700938607002D
:10BA4000130630039305100017B507001305C5470B
:10BA5000EF905236EFA0C03B930790FC6F10D0449C
:10BA6000032744F09307100063F0E7100327C4FB9B
:10BA7000832704F563FAE70E9747FF019387075979
:10BA800003A7070083A74700B7160000B376D700C7
:10BA90002324D4EA93F707002326F4EA832684EAD2
:10BAA0000327C4EA93870600B3E7E700638A070A1F
:10BAB000EFA040349306300017B607001306060EB9
:10BAC0009305500B17C507001305C59BEFA0102267
:10BAD0009747FF019387075383A7070063880702EF
:10BAE00097F7030083A7071B83A7070083A7C70057
:10BAF00093860700130670029305100017B5070020
:10BB000013054538EF90122B6F00C00297F7030022
:10BB100083A7471883A7070083A7C700938607005A
:10BB20001306A0019305100017B50700130505388B
:10BB3000EF90522897F7030083A7C71583A7070044
:10BB400083A7C700938607001306300393051000F0
:10BB500017B507001305853AEF90D225EFA0402BCB
:10BB6000930790FC6F105034032744F09307200094
:10BB700063F0E710032784FA8327C4F463FAE70E1F
:10BB80009747FF019387874803A7070083A74700CC
:10BB9000B7160000B376D7002320D4EA93F7070046
:10BBA0002322F4EA832604EA032744EA9387060063
:10BBB000B3E7E700638A070AEFA0C02393063000CB
:10BBC00017B60700130686FD9305A00B17C50700DF
:10BBD0001305458BEFA090119747FF01938787428C
:10BBE00083A707006388070297F7030083A7870AE4
:10BBF00083A7070083A7C700938607001306700278
:10BC00009305100017B507001305C527EF90921A8A
:10BC10006F00C00297F7030083A7C70783A7070039
:10BC200083A7C700938607001306A00193051000A1
:10BC300017B5070013058527EF90D21797F7030074
:10BC400083A7470583A7070083A7C700938607003C
:10BC5000130630039305100017B507001305452D93
:10BC6000EF905215EFA0C01A930790FC6F10D023ED
:10BC70000327C4F6832784FBB377F702638A070E92
:10BC80009747FF019387873803A7070083A74700DB
:10BC9000B7160000B376D700232CD4E893F707003B
:10BCA000232EF4E8832684E90327C4E9938706005A
:10BCB000B3E7E700638A070AEFA0C01393063000DA
:10BCC00017B60700130686ED9305200C17B507007D
:10BCD0001305457BEFA090019747FF0193878732BB
:10BCE00083A707006388070297F7030083A787FAF3
:10BCF00083A7070083A7C700938607001306800267
:10BD00009305100017B507001305450FEF90920A31
:10BD10006F00C00297F7030083A7C7F783A7070048
:10BD200083A7C700938607001306B0019305100090
:10BD300017B507001305450FEF90D20797F70300DB
:10BD400083A747F583A7070083A7C70017B6070097
:10BD50001306462197B50700938585EA13850700EA
:10BD6000EF80023DEFA0C00A9307A0FC6F10D01334
:10BD7000032704F78327C4FBB377F702638A070E10
:10BD80009747FF019387872803A7070083A74700EA
:10BD9000B7160000B376D7002328D4E893F707003E
:10BDA000232AF4E8832604E9032744E9938706005D
:10BDB000B3E7E700638A070AEFA0C00393063000E9
:10BDC00017B60700130686DD9305400C17B507006C
:10BDD0001305456BEFA080719747FF01938787227A
:10BDE00083A707006388070297F7030083A787EA02
:10BDF00083A7070083A7C700938607001306800266
:10BE00009305100017B50700130545FFEF90827AE0
:10BE10006F00C00297F7030083A7C7E783A7070057
:10BE200083A7C700938607001306B001930510008F
:10BE300017B50700130545FFEF90C27797F703008A
:10BE400083A747E583A7070083A7C70017B60700A6
:10BE50001306061397B50700938585DA1385070047
:10BE6000EF80022DEF90D07A9307A0FC6F10D003E3
:10BE7000032744F7832784FAB377F702638A070E10
:10BE80009747FF019387871803A7070083A74700F9
:10BE9000B7160000B376D7002324D4E893F7070041
:10BEA0002326F4E8832684E80327C4E89387060062
:10BEB000B3E7E700638A070AEF90D0739306300078
:10BEC00017B60700130686CD9305600C17B507005B
:10BED0001305455BEFA080619747FF0193878712A9
:10BEE00083A707006388070297F7030083A787DA11
:10BEF00083A7070083A7C700938607001306800265
:10BF00009305100017B50700130545EFEF90826AFF
:10BF10006F00C00297F7030083A7C7D783A7070066
:10BF200083A7C700938607001306B001930510008E
:10BF300017B50700130545EFEF90C26797F70300A9
:10BF400083A747D583A7070083A7C70017B60700B5
:10BF50001306C60497B50700938585CA13850700A5
:10BF6000EF80021DEF90D06A9307A0FC6F10C073A2
:10BF7000832784F083A7070183A70702638C071434
:10BF8000832784F083A7070183A7470263840714EC
:10BF9000832784F083A7070183A78702638C071296
:10BFA000832784EF63800704832784F083A7070136
:10BFB00083A70702032784FB6316F702832784F015
:10BFC00083A7070183A747020327C4FB631CF7006D
:10BFD000832784F083A7070183A78702032784FAB6
:10BFE0006300F7769747FF019387470203A707008F
:10BFF00083A74700B7160000B376D7002320D4E804
:10C0000093F707002322F4E8832604E8032744E893
:10C0100093870600B3E7E700638A070AEF90905D15
:10C020009306300017B60700130646B79305300D88
:10C0300017B5070013050545EFA0404B9747FF01D3
:10C04000938747FC83A707006388070297F70300DD
:10C0500083A747C483A7070083A7C7009386070069
:10C06000130680029305100017B50700130505D9C4
:10C07000EF9042546F00C00297F7030083A787C177
:10C0800083A7070083A7C700938607001306B001A4
:10C090009305100017B50700130505D9EF908251DD
:10C0A00097F7030083A707BF83A7070083A7C700ED
:10C0B00017B60700130646F097B50700938545B4F9
:10C0C00013850700EF80C206EF9090549307A0FC01
:10C0D0006F10805D832784EF63960766832784F65D
:10C0E00083A7C703232AF4F8832744F9639607003C
:10C0F00093071000232AF4F89747FF01938707F16D
:10C1000003A7070083A7470093761700232CD4E6E4
:10C1100093F70700232EF4E6832684E70327C4E77A
:10C1200093870600B3E7E7006382070AEF90904C1D
:10C130009306100017B60700130606F29305E00EEB
:10C1400017B5070013050534EFA0403A9747FF01E4
:10C15000938747EB83A707006388070297F70300DD
:10C1600083A747B383A7070083A7C7009386070069
:10C170001306E0009305100017B50700130545EE00
:10C18000EF9042436F00000297F7030083A787B048
:10C1900083A7070083A7C700938507001305000244
:10C1A000EF80820397F7030083A7C7AE83A707003A
:10C1B00083A7C700032644F997B50700938545EB8D
:10C1C00013850700EF70D276EF9090448325C4F674
:10C1D000032544F9EFE05FBD2322A4F4832504F78F
:10C1E000032544F9EFE05FBC2320A4F4832544F742
:10C1F000032544F9EFE05FBB232EA4F20327C4F626
:10C20000832744F4B356F702032744F5832744F405
:10C21000B357F7029385070013850600EFE01FBEB2
:10C22000232CA4FA032784FB832744F4B307F702E3
:10C23000232CF4FA032744F09307100063F0E7047B
:10C24000032704F7832704F4B356F702032704F502
:10C25000832704F4B357F70293850700138506007C
:10C26000EFE0DFB9232EA4FA0327C4FB832704F4ED
:10C27000B307F702232EF4FA6F00C00093071000F3
:10C28000232EF4FA032744F09307200063F0E70419
:10C29000032744F78327C4F3B356F7020327C4F4F4
:10C2A0008327C4F3B357F70293850700138506006D
:10C2B000EFE0DFB42324A4FA032784FA8327C4F32E
:10C2C000B307F7022324F4FA6F00C0199307100094
:10C2D0002324F4FA6F000019832784FA93F71700D8
:10C2E000639A0702832784FA93D71700032644F73B
:10C2F000938507000325C4F3EFE0DFB8930705003B
:10C30000638A0700832784FA93D717002324F4FA5B
:10C310006F0040158327C4FB93F71700639A070249
:10C320008327C4FB93D71700032604F793850700E0
:10C33000032504F4EFE01FB593070500638A0700A7
:10C340008327C4FB93D71700232EF4FA6F008011C4
:10C35000832784FB93F71700639A0702832784FBE4
:10C3600093D717000326C4F693850700032544F4EA
:10C37000EFE05FB193070500638A0700832784FB22
:10C3800093D71700232CF4FA6F00C00D032784FA0B
:10C390009307100063F4E7020327C4F3832744F4F0
:10C3A00063EEE7000327C4F3832704F463E8E700A0
:10C3B000930710002324F4FA6F00C00A0327C4FB7C
:10C3C0009307100063F4E702032704F48327C4F300
:10C3D00063EEE700032704F4832744F463E8E700EF
:10C3E00093071000232EF4FA6F00C007032784FB85
:10C3F0009307100063F4E702032744F4832704F44F
:10C4000063EEE700032744F48327C4F363E8E700FF
:10C4100093071000232CF4FA6F00C004032784FA5A
:10C420009307100063F8E700930710002324F4FA41
:10C430006F0000030327C4FB9307100063F8E700B5
:10C4400093071000232EF4FA6F008001032784FB6A
:10C450009307100063F8E70093071000232CF4FA09
:10C4600013000000032784FB8327C4FB3307F70274
:10C47000832784FAB307F702032784F4E36EF7E413
:10C48000832744F993972700232CF4F28327C4F0E1
:10C4900083A7C70083A74701232AF4F20327C4F622
:10C4A000832784FBB357F7022328F4F8032704F704
:10C4B0008327C4FBB357F7022326F4F8032744F776
:10C4C000832784FAB357F7022324F4F86F0000227D
:10C4D000032784FA832744F8B377F70263980704A5
:10C4E000032784FA832744F8B357F702032644F757
:10C4F000938507000325C4F3EFE0DF989307050059
:10C5000063860702032784FA832744F8B357F702A8
:10C510002324F4FA032784F8832744F8B307F702A7
:10C520002324F4F8232204F86F00800C0327C4FBB3
:10C53000832744F8B377F702639807040327C4FB03
:10C54000832744F8B357F702032604F793850700BF
:10C55000032504F4EFE01F939307050063860702A9
:10C560000327C4FB832744F8B357F702232EF4FABA
:10C570000327C4F8832744F8B307F7022326F4F807
:10C58000232204F86F00C006032784FB832744F8A6
:10C59000B377F70263980704032784FB832744F8E3
:10C5A000B357F7020326C4F693850700032544F426
:10C5B000EFE05F8D9307050063860702032784FB86
:10C5C000832744F8B357F702232CF4FA032704F91E
:10C5D000832744F8B307F7022328F4F8232204F84A
:10C5E0006F000001832744F89387F7FF2322F4F8B4
:10C5F000032744F893071000E3ECE7EC832744F8A3
:10C60000639407006F00800E032784FA93071000DD
:10C6100063F2E704032784FA832784FB63ECE702D1
:10C62000032784FA8327C4FB63E6E702032784FB1E
:10C630008327C4FBB307F702032784F363ECE70007
:10C64000930710002324F4FA832744F72324F4F8F3
:10C650006F00C0090327C4FB9307100063F2E704CF
:10C660000327C4FB832784FA63ECE7020327C4FB98
:10C67000832784FB63E6E702032784FA832784FB8E
:10C68000B307F702032784F363ECE7009307100076
:10C69000232EF4FA832704F72326F4F86F0000050D
:10C6A000032784FB9307100063FEE708032784FB3E
:10C6B0008327C4FB63E8E708032784FB832784FA06
:10C6C00063E2E7080327C4FB832784FAB307F70272
:10C6D000032784F363E8E70693071000232CF4FA9A
:10C6E0008327C4F62328F4F813000000032704F975
:10C6F0008327C4F83307F702832784F8B307F702C8
:10C70000032744F3B357F7022322F4F8032744F82E
:10C710009307100063F8E702032784FB8327C4FB19
:10C720003307F702832784FA3307F702832644F896
:10C73000832784F3B387F602E3ECE7EA6F00800017
:10C74000130000009747FF019387478C03A707005A
:10C7500083A74700937617002328D4E693F70700B2
:10C76000232AF4E6832604E7032744E79387060099
:10C77000B3E7E7006380070EEF90C06793061000F1
:10C7800017B607001306468D9305101C17B5070052
:10C79000130545CFEF9090559747FF019387878604
:10C7A00083A707006388070297E7030083A7874EE4
:10C7B00083A7070083A7C700938607001306E0003E
:10C7C0009305100017B5070013058589EF80925E69
:10C7D0006F00000297E7030083A7C74B83A70700FA
:10C7E00083A7C7009385070013050002EF70D21ED0
:10C7F00097E7030083A7074A83A7070003A5C7009D
:10C80000832784F003A647010327C4F6832784FB0C
:10C81000B356F702032704F78327C4FBB355F70287
:10C82000032744F7832784FAB357F7022320F10044
:10C830009388050013880600832784FA0327C4FB26
:10C84000832684FB97B5070093858584EF70520E8D
:10C85000EF90005C032784FB8327C4FB3307F702B8
:10C86000832784FAB307F702032784F46372F7027D
:10C8700097B607009386C68617B60700130686C0CC
:10C880009305901C17A507001305052FEF60D252E2
:10C89000032784FB832744F563F2E70297B607007A
:10C8A0009386068717B607001306C6BD9305A01C1E
:10C8B00017A507001305452CEF6012500327C4FB92
:10C8C000832704F563F2E70297B607009386C685CF
:10C8D00017B60700130606BB9305B01C17A5070083
:10C8E00013058529EF60524D032784FA8327C4F48A
:10C8F00063F2E70297B607009386868417B60700AF
:10C90000130646B89305C01C17A507001305C526D6
:10C91000EF60924A0327C4F6832784FBB377F702BC
:10C920006382070297B607009386068317B607004F
:10C93000130646B59305F01C17A507001305C5237C
:10C94000EF609247032704F78327C4FBB377F7020E
:10C950006382070297B607009386868117B60700A1
:10C96000130646B29305001D17A507001305C52041
:10C97000EF609244032744F7832784FAB377F702E2
:10C980006382070297B607009386068017B60700F2
:10C99000130646AF9305101D17A507001305C51D07
:10C9A000EF609241232204FA232004FA232E04F894
:10C9B0006F009010832784F083A7070103A7470126
:10C9C0008327C4F993975700B307F7002324F4F2A1
:10C9D000832784F083A687010327C4F99307070000
:10C9E00093971700B387E70093973700B387F60054
:10C9F0002322F4F2832744F283A74701639A070EA8
:10CA00009737FF019387876003A7070083A7470035
:10CA1000B7160000B376D7002324D4E693F70700B7
:10CA20002326F4E6832684E60327C4E693870600DC
:10CA3000B3E7E7006388070AEF90C03B9306300036
:10CA400017A60700130686159305C01D17B5070026
:10CA5000130545A3EF9090299737FF019387875AD5
:10CA600083A707006388070297E7030083A787224D
:10CA700083A7070083A7C700938607001306400219
:10CA80009305100017A5070013058571EF809232FA
:10CA90006F00C00297E7030083A7C71F83A70700A3
:10CAA00083A7C70093860700130670019305100043
:10CAB00017A5070013054571EF80D22F97E70300F4
:10CAC00083A7471D83A7070083A7C7000326C4F9D0
:10CAD00097A507009385C57013850700EF70426521
:10CAE000EF9000339307C0FC232CF4F86F00903BC9
:10CAF000832784F203A7870193072000630AF702C4
:10CB0000832784F203A78700B71700009387C7190C
:10CB1000630EF778832784F203A787019307100039
:10CB20006316F778832744F283A7070163800778A9
:10CB3000832744F283A7070183A70700232EF4F07D
:10CB4000832784F203A78701930720006316F73E2B
:10CB5000232004F86F0080038327C4F183A7870292
:10CB600003A78700832704F893972700B307F700EC
:10CB700003A707008327C4F083A7C7006304F70255
:10CB8000832704F8938717002320F4F88327C4F140
:10CB900083A7870283A70701032704F8E36EF7FA48
:10CBA0006F008000130000008327C4F183A7870271
:10CBB00083A70701032704F86362F70297A607001B
:10CBC0009386866417B607001306C68B9305901EDE
:10CBD00017A50700130545FAEF60121E8327C4F15D
:10CBE00083A7870203A78700832704F8939727006A
:10CBF000B307F70083A7070083A78708639A071086
:10CC00009737FF019387874003A7070083A7470053
:10CC1000B7160000B376D7002320D4E693F70700B9
:10CC20002322F4E6832604E6032744E693870600DE
:10CC3000B3E7E7006388070CEF90C01B9306300052
:10CC400017A60700130686F59305901E17B5070073
:10CC500013054583EF9090099737FF019387873A33
:10CC600083A707006388070297E7030083A787026B
:10CC700083A7070083A7C700938607001306200237
:10CC80009305100017A507001305455AEF8092126F
:10CC90006F00C00297E7030083A7C7FF83A70700C1
:10CCA00083A7C70093860700130650019305100061
:10CCB00017A507001305C559EF80D20F97E70300AA
:10CCC00083A747FD83A7070083A6C7008327C4F176
:10CCD00083A7870203A78700832704F89397270079
:10CCE000B307F70083A7070083A70717138607007A
:10CCF00097A507009385455713850600EF704243BB
:10CD0000EF900011930750FC232CF4F86F0090195A
:10CD10008327C4F103A74704832704F893972700C8
:10CD2000B307F70083A7070093F72700639C070E5C
:10CD30009737FF019387872D03A7070083A7470035
:10CD4000B7160000B376D700232CD4E493F707007E
:10CD5000232EF4E4832684E50327C4E593870600A5
:10CD6000B3E7E700638A070AEF90C0089306300034
:10CD700017A60700130686E29305901E17A5070065
:10CD800013054570EF9080769737FF0193878727CB
:10CD900083A707006388070297E7030083A787EF4D
:10CDA00083A7070083A7C700938607001306B00276
:10CDB0009305100017A507001305454DEF80827FEE
:10CDC0006F00C00297E7030083A7C7EC83A70700A3
:10CDD00083A7C700938607001306E00193051000A0
:10CDE00017A507001305454DEF80C27C97E70300A8
:10CDF00083A747EA83A7070083A7C7009386070096
:10CE00001306F0029305100017A507001305C54C83
:10CE1000EF80427AEF80D07F930760FF232CF4F8F5
:10CE20006F0050088327C4F103A74704832704F841
:10CE300093972700B307F70083A7070093F717001E
:10CE4000639C073A9737FF019387471C03A70700A6
:10CE500083A74700B7160000B376D7002328D4E491
:10CE600093F70700232AF4E4832604E5032744E527
:10CE700093870600B3E7E700638A070AEF8090779D
:10CE80009306300017A60700130646D19305901E9F
:10CE900017A507001305055FEF9040659737FF0161
:10CEA0009387471683A707006388070297E7030065
:10CEB00083A747DE83A7070083A7C70093860700E1
:10CEC000130630029305100017A507001305C5438C
:10CED000EF80426E6F00C00297E7030083A787DBF5
:10CEE00083A7070083A7C700938607001306600186
:10CEF0009305100017A5070013054543EF80826BCB
:10CF000097E7030083A707D983A7070083A7C70074
:10CF1000938607001306F0029305100017A507007B
:10CF200013054542EF800269EF80906E930780FD04
:10CF3000232CF4F86F0000778327C4F183A7C7037D
:10CF4000638A07108327C4F103A7C7018327C4F0AE
:10CF500083A7C70083A7C70BB377F702638C070EBD
:10CF60009737FF019387870A03A7070083A7470026
:10CF7000B7160000B376D7002324D4E493F7070054
:10CF80002326F4E4832684E40327C4E4938706007D
:10CF9000B3E7E700638A070AEF80D06593063000A5
:10CFA00017A60700130686BF9305D01E17A5070016
:10CFB0001305454DEF9080539737FF019387870402
:10CFC00083A707006388070297E7030083A787CC3E
:10CFD00083A7070083A7C700938607001306D00224
:10CFE0009305100017A507001305C538EF80825C74
:10CFF0006F00C00297E7030083A7C7C983A7070094
:10D0000083A7C7009386070013060002930510004C
:10D0100017A5070013050539EF80C25997E70300EC
:10D0200083A747C783A7070083A7C7009386070086
:10D03000130610039305100017A507001305C53844
:10D04000EF804257EF80D05C930730FF232CF4F839
:10D050006F0040658327C4F183A7C7036386070475
:10D060000327C4F1832744F283A707010327C703DB
:10D0700023A0E7008327C4F183A7C7012320F4E49A
:10D08000232204E4832744F2832604E4032744E4B0
:10D0900023A4D70023A6E7008327C4F183A7C703EF
:10D0A000232EF4F06F008001832744F293060000E2
:10D0B0001307000023A4D70023A6E7008327C4F1A9
:10D0C00083A78701232CF4E2232E04E28327C4F0F4
:10D0D00083A7C70003A7070883A74708032584E39E
:10D0E0008325C4E3138605009386070063EEC6001C
:10D0F00013860500938607006310D610930605007B
:10D100009307070063FAD70E9737FF01938707F05D
:10D1100003A7070083A74700B7160000B376D70020
:10D120002328D4E293F70700232AF4E2832604E3BA
:10D13000032744E393870600B3E7E7006388070A01
:10D14000EF80504B9306300017A60700130606A584
:10D150009305801F17A507001305C532EF9000390E
:10D160009737FF01938707EA83A7070063880702C1
:10D1700097E7030083A707B283A7070083A7C70029
:10D1800093860700130610029305100017A50700E9
:10D190001305C526EF8002426F00C00297E7030027
:10D1A00083A747AF83A7070083A7C700938607001D
:10D1B000130640019305100017A507001305452627
:10D1C000EF80423F97E7030083A7C7AC83A7070020
:10D1D00083A7C7000326C4F997A507009385C52533
:10D1E00013850700EF60D274EF8090429307B0FF81
:10D1F000232CF4F86F00004B832704FA13871700E1
:10D200002320E4FA0327C4F1832604F6939727002A
:10D21000B387F60023A0E7008327C4F11385070036
:10D22000EF70DFD78327C4F183A747036398070014
:10D230008327C4F1032784F623AAE7028327C4F1D6
:10D2400083A74703638E07048327C4F183A747039B
:10D2500003A7871A8327C4F083A7C70083A7871A69
:10D260006300F704832744FA138717002322E4FAA4
:10D2700093972700032784F5B307F7001306C4F13B
:10D28000938807001308000093070000930600002E
:10D2900013070000930510000325C4F0EF20C038E9
:10D2A0008327C4F1032784F623AAE7028327C4F95E
:10D2B00093871700232EF4F8832784F083A70701B0
:10D2C00083A707000327C4F96366F7EE832744EFBB
:10D2D00063860702832744FA93972700032784F580
:10D2E0003307F700832744EF93972700138607003F
:10D2F000832504EF13050700EF80D27E032744FA4D
:10D30000832744EFB307F70013860700032744FA87
:10D31000832744EFB307F70063860700832784F56C
:10D320006F00800093070000032704FA832604F6A9
:10D33000130504F29388060013080700130706007C
:10D3400083260400371600001306061F8325C4F049
:10D35000EF30505D232CA4F8832784F963920734BF
:10D36000832704F2371700001307071F23ACE704D5
:10D37000832704F2032784F023A4E700832704F221
:10D38000032784FB23A2E702832704F20327C4FBBD
:10D3900023A4E702832704F2032784FA23A6E702E3
:10D3A000832704F2032744F023AEE702832704F225
:10D3B0008326C4F6032784FB33D7E60223A6E700BF
:10D3C000832704F2832604F70327C4FB33D7E6023E
:10D3D00023A8E700832704F2832644F7032784FA6F
:10D3E00033D7E60223AAE700832704F20327C4FA0F
:10D3F00023ACE700832704F2032704FB23AEE700F6
:10D40000832704F2032744FB23A0E702832784F049
:10D4100083A7C700832584F613850700EFA0105B60
:10D420002328A4F2832704F363D2070297A60700F8
:10D430009386460417A607001306C60493056023C7
:10D440001795070013054573EF600217832704F251
:10D45000032704F323A8E706832784F083A70701A3
:10D4600083A6C702832704F313974700832704F298
:10D470003387E60023A0E700832784F083A7070112
:10D4800003A707009307070093971700B387E700E8
:10D4900093973700832404F213850700EF804252EC
:10D4A0009307050023A0F404232E04F86F00C0178F
:10D4B000832704F283A607040327C4F99307070010
:10D4C00093971700B387E70093973700B387F60069
:10D4D0002326F4F2832784F083A687010327C4F967
:10D4E0009307070093971700B387E70093973700D8
:10D4F000B387F60003A7070083A74700232EE4F6AF
:10D500008327C4F72324F4E2232604E28327C4F20A
:10D51000832684E20327C4E223A0D70023A2E700E6
:10D52000832784F083A687010327C4F993070700A4
:10D5300093971700B387E70093973700B387F600F8
:10D5400003A7870083A7C7008326C4F223A4E600AD
:10D5500023A6F600832784F083A687010327C4F956
:10D560009307070093971700B387E7009397370057
:10D57000B387F60083A70701639807008327C4F2E7
:10D5800023A807006F0080090325C4F7EF30C00F00
:10D59000232CA4F6032784F79307F00763F6E7002C
:10D5A00093070008232CF4F60327C4F7832784F796
:10D5B0006376F700832784F7232EF4F68325C4F7D8
:10D5C000032584F7EF30C033130705008327C4F227
:10D5D00023A8E7008327C4F203A50701832784F06B
:10D5E00083A687010327C4F99307070093971700C1
:10D5F000B387E70093973700B387F60083A6070148
:10D600008327C4F203A7070083A7470093070700F7
:10D610001386070093850600EF80D24C8327C4F958
:10D6200093871700232EF4F8832784F083A707013C
:10D6300083A707000327C4F9E36CF7E6832704F206
:10D6400023AE0704032584F0EF60416297D70300FF
:10D6500083A7C76383A7070063880702832704F2B1
:10D6600083A7470613850700EFA09021032584F0C8
:10D67000EF60C15F832704F283A7470683A7C7052E
:10D68000032784F023A0E700832704F29385070093
:10D690000325C4F0EF301075232C04F86F008000D0
:10D6A00013000000832784F9032144E21385070057
:10D6B000130104E18320C11E0324811E8324411E23
:10D6C0000329011E8329C11D032A811D832A411DAF
:10D6D000032B011D832BC11C032C811C832C411C9B
:10D6E000032D011C832DC11B1301011F6780000046
:10D6F000130101FE232E1100232C810013040102CB
:10D700002326A4FE2324B4FE2322C4FE832684FE03
:10D710006396060E8326C4FE6382060E9737FF01CA
:10D720009387C78E03A7070083A74700B71600009B
:10D730003373D70093F3070093070300B3E7770031
:10D74000638A070AEF80006B9306300017F6070024
:10D750001306C6209305700F17F507001305C52B98
:10D76000EF80D0589737FF019387C78983A70700B9
:10D770006388070297D7030083A7C75183A70700D1
:10D7800083A7C700938607001306E00193051000E6
:10D7900017F507001305051DEF70D2616F00C00279
:10D7A00097D7030083A7074F83A7070083A7C70066
:10D7B00093860700130610019305100017F5070064
:10D7C0001305451CEF70125F97D7030083A7874CA2
:10D7D00083A7070083A7C70017F607001306C61B19
:10D7E00097F507009385C51D13850700EF60521458
:10D7F000EF800062930720FE6F004021832684FEA5
:10D800006386060E8326C4FE6392060E9727FF01E9
:10D810009387C77F03A7070083A74700B7160000B9
:10D820003378D70093F8070093070800B3E7170190
:10D83000638A070AEF80005C9306300017F6070042
:10D840001306C6119305A00F17F507001305C51C95
:10D85000EF80D0499727FF019387C77A83A70700F6
:10D860006388070297D7030083A7C74283A70700EF
:10D8700083A7C700938607001306E00193051000F5
:10D8800017F507001305050EEF70D2526F00C002A6
:10D8900097D7030083A7074083A7070083A7C70084
:10D8A00093860700130610019305100017F5070073
:10D8B0001305450DEF70125097D7030083A7873DDE
:10D8C00083A7070083A7C70017F607001306860F74
:10D8D00097F507009385C50E13850700EF60520585
:10D8E000EF800053930720FE6F004012832644FE12
:10D8F0006396060E8326C4FE6392060E9726FF01EA
:10D900009386C67003A6060083A64600B7150000DE
:10D910003377B60093F7060093060700B3E6F600E8
:10D92000638A060AEF80004D9306300017F6070061
:10D930001306C6029305D00F17F507001305C50D92
:10D94000EF80D03A9727FF019387C76B83A7070023
:10D950006388070297D7030083A7C73383A707000D
:10D9600083A7C700938607001306E0019305100004
:10D9700017F50700130505FFEF70D2436F00C002D3
:10D9800097D7030083A7073183A7070083A7C700A2
:10D9900093860700130610019305100017F5070082
:10D9A000130545FEEF70124197D7030083A7872E1A
:10D9B00083A7070083A7C70017F60700130606030F
:10D9C00097F507009385C5FF13850700EF60427642
:10D9D000EF800044930720FE6F004003832784FEFE
:10D9E000638A0700832784FE17F707001307C7F62B
:10D9F00023A0E700832744FE63880700832744FEB3
:10DA00001307100023A0E700930700001385070009
:10DA10008320C101032481011301010267800000FA
:10DA2000130101FC232E1102232C8102232A21033E
:10DA30002328310313040104232EA4FC2328B4FC5F
:10DA4000232AC4FC232CD4FC2326E4FC2324F4FC4A
:10DA5000232404FE232604FE8327C4FD6392070EBD
:10DA60009727FF019387875A03A7070083A74700DB
:10DA7000B7160000337ED70093FE070093070E0011
:10DA8000B3E7D701638A070AEF80C03693063000F8
:10DA900017060800130606029305900217050800F2
:10DAA00013058512EF8090249727FF0193878755F0
:10DAB00083A707006388070297D7030083A7871D02
:10DAC00083A7070083A7C7009386070013061002E9
:10DAD0009305100017050800130545FEEF70922D01
:10DAE0006F00C00297D7030083A7C71A83A7070058
:10DAF00083A7C70093860700130640019305100013
:10DB0000170508001305C5FDEF70D22A97D703004B
:10DB100083A7471883A7070083A7C7001706080035
:10DB2000130686FD97050800938545FE13850700BB
:10DB3000EF600260EF80C02D930700FE6F0040375A
:10DB4000832784FD6396070E8327C4FC6382070E38
:10DB50009727FF019387874B03A7070083A74700F9
:10DB6000B71600003373D70093F307009307030041
:10DB7000B3E77700638A070AEF80C0279306300077
:10DB800017060800130606F39305B00217050800F0
:10DB900013058503EF8090159727FF01938787462C
:10DBA00083A707006388070297D7030083A7870E20
:10DBB00083A7070083A7C700938607001306E00129
:10DBC0009305100017050800130585F4EF70921EE9
:10DBD0006F00C00297D7030083A7C70B83A7070076
:10DBE00083A7C70093860700130610019305100052
:10DBF000170508001305C5F3EF70D21B97D7030074
:10DC000083A7470983A7070083A7C7001706080053
:10DC1000130646F397050800938545EF1385070023
:10DC2000EF600251EF80C01E930720FE6F00402876
:10DC3000832784FC6396070E8327C4FC6392070E38
:10DC40009727FF019387873C03A7070083A7470017
:10DC5000B71600003378D70093F807009307080041
:10DC6000B3E71701638A070AEF80C01893063000F4
:10DC700017060800130606E49305C00217050800FE
:10DC8000130585F4EF8090069727FF019387873768
:10DC900083A707006388070297D7030083A787FF3E
:10DCA00083A7070083A7C700938607001306E00138
:10DCB0009305100017050800130585E5EF70920F16
:10DCC0006F00C00297D7030083A7C7FC83A7070094
:10DCD00083A7C70093860700130610019305100061
:10DCE000170508001305C5E4EF70D20C97D70300A1
:10DCF00083A747FA83A7070083A7C7001706080072
:10DD00001306C6E697050800938545E013850700CE
:10DD1000EF600242EF80C00F930720FE6F004019B2
:10DD2000930704FE130600009385070013051000F7
:10DD3000EFF01F9C832704FE0327C4FD6302F70E48
:10DD40009727FF019387872C03A7070083A7470026
:10DD5000B71600003379D70093F90700930709003D
:10DD6000B3E73701638A070AEF80C00893063000E3
:10DD700017060800130606D49305F00217050800DD
:10DD8000130585E4EF8080769727FF019387872727
:10DD900083A707006388070297D7030083A787EF4D
:10DDA00083A7070083A7C700938607001306100206
:10DDB0009305100017050800130545D0EF70827F0A
:10DDC0006F00C00297D7030083A7C7EC83A70700A3
:10DDD00083A7C70093860700130640019305100030
:10DDE000170508001305C5CFEF70C27C97D7030055
:10DDF00083A747EA83A7070083A7C7009386070086
:10DE00001306F00293051000170508001305C5D886
:10DE1000EF70427AEF70D07F930700FE6F004009E9
:10DE2000EFC000162322A4FE832744FE638607006A
:10DE3000832744FE6F00C007032504FD832544FDAE
:10DE4000EFB09027930705002324F4FE832784FE78
:10DE5000639607009307F0FF6F0080058327C4FCDB
:10DE600063800702832684FD0326C4FC032504FD8A
:10DE7000832544FDEFB0100A930705002326F4FE26
:10DE8000832784FC63880700032784FE832784FCA0
:10DE900023A0E7008327C4FE6346F000832784FDA8
:10DEA00063960700930700006F0080009307F0FF60
:10DEB000138507008320C103032481030329410341
:10DEC000832901031301010467800000130101FB92
:10DED0002326110423248104232221052320310534
:10DEE000232E4103232C5103232A6103232871038A
:10DEF00013040105232EA4FA232CB4FA232AC4FA0E
:10DF0000232C04FC8327C4FB23A60700832784FB60
:10DF1000638C0742832784FB232AF4FC130744FC09
:10DF2000930784FC13060700938507001305100070
:10DF3000EFF00FFC232C04FC6F008037832784FB59
:10DF40002328F4FC6F008010832704FD03A707003B
:10DF5000832744FD83A707006314F70E9727FF016B
:10DF60009387C70A03A7070083A74700B7160000D7
:10DF70003379D70093F9070093070900B3E7370116
:10DF80006386070AEF7010679306300017360800A3
:10DF90001306C67A9305D003174508001305C59EDE
:10DFA000EF80C0549727FF019387C70583A7070019
:10DFB0006388070297D7030083A7C7CD83A707000D
:10DFC00083A7C700938607001306E000930510009F
:10DFD0001735080013050577EF70C25D6F0000026A
:10DFE00097D7030083A707CB83A7070083A7C700A2
:10DFF0009385070013050002EF60021E97D7030008
:10E0000083A747C983A7070003A7C700832704FD89
:10E0100083A707001386070097350800938585734B
:10E0200013050700EF60C210EF70905E832744FB7A
:10E03000130700FC23A0E700930700006F00803265
:10E04000832704FD938787002328F4FC032704FD1E
:10E05000832744FDE36AF7EE832744FD03A7070007
:10E06000B717000093874708631CF714232604FCA6
:10E07000232E04FC6F000004832744FD9387470090
:10E0800083A70700138707008327C4FD9397270002
:10E09000930604FEB387F60083A787FE6316F70096
:10E0A000930710002326F4FC8327C4FD93871700F1
:10E0B000232EF4FC832744FC0327C4FDE36EF7FA08
:10E0C0008327C4FC6396070E9727FF01938707F405
:10E0D00003A7070083A74700B7160000337AD700CD
:10E0E00093FA070093070A00B3E757016388070A0A
:10E0F000EF70505093063000173608001306066480
:10E100009305E0041745080013050588EF80003EDD
:10E110009727FF01938707EF83A70700638807020C
:10E1200097D7030083A707B783A7070083A7C70074
:10E13000938607001306E0009305100017350800CA
:10E1400013054560EF7002476F00000297D7030088
:10E1500083A747B483A7070083A7C7009385070059
:10E1600013050002EF60420797D7030083A787B229
:10E1700083A7070003A7C700832744FD93874700B1
:10E1800083A7070013860700973508009385455E2F
:10E1900013050700EF50D279EF709047832744FBB7
:10E1A000130700FE23A0E700930700006F00801B09
:10E1B000832744FD93878700232AF4FC6F00800E99
:10E1C0009727FF01938787E403A7070083A74700EA
:10E1D000B7160000337BD70093FB070093070B00B3
:10E1E000B3E777016386070AEF70D04093063000EB
:10E1F0001736080013068654930570051735080076
:10E2000013058578EF80802E9727FF01938787DF9E
:10E2100083A707006388070297D7030083A787A710
:10E2200083A7070083A7C700938607001306E000B3
:10E2300093051000173508001305C550EF7082379D
:10E240006F00000297D7030083A7C7A483A7070026
:10E2500083A7C7009385070013050002EF50D2770C
:10E2600097D7030083A707A383A7070003A7C700C7
:10E27000832744FD83A7070013860700973508000E
:10E280009385C55013050700EF50926AEF70503820
:10E29000832744FB130700FC23A0E700930700003B
:10E2A0006F00400C832784FD93871700232CF4FC18
:10E2B000832744FD83A70700E39207C8832784FDD3
:10E2C00093971700938717009397270013850700EC
:10E2D000EF70026F93070500138707008327C4FBC5
:10E2E00023A6E7008327C4FB83A7C700639C07001E
:10E2F000832744FB1307A0FF23A0E7009307000038
:10E300006F0040068327C4FB03A7C700832784FD53
:10E31000939717009387170093972700138607009A
:10E32000832584FB13050700EF70D27B032784FD50
:10E330008327C4FB23AAE700832744FB23A007000D
:10E34000832784FD6F0000028327C4FB23A60700F8
:10E350008327C4FB23AA0700832744FB23A00700CD
:10E3600093070000138507008320C1040324810460
:10E370000329410483290104032AC103832A810359
:10E38000032B4103832B0103130101056780000068
:10E39000130101F9232611062324810623222107D4
:10E3A00023203107232E4105232C5105232A610503
:10E3B0002328710523268105232491052322A10505
:10E3C0002320B105130401072326A4FA2324B4FA59
:10E3D0002322C4FA2320D4FA232EE4F8232CF4F8C1
:10E3E000232E04FA232404FC832744FA63860700BF
:10E3F000832784FA6394070E9727FF01938707C149
:10E4000003A7070083A74700B71600003373D700A0
:10E4100093F3070093070300B3E77700638A070AC3
:10E42000EF70501D930630001736080013060631B2
:10E43000930590081735080013058556EF80000BEB
:10E440009727FF01938707BC83A70700638807020C
:10E4500097D7030083A7078483A7070083A7C70074
:10E46000938607001306E001930510001735080096
:10E470001305C533EF7002146F00C00297D7030075
:10E4800083A7478183A7070083A7C7009386070058
:10E490001306100193051000173508001305053306
:10E4A000EF70421197C7030083A7C77E83A70700B9
:10E4B00083A7C70017360800130686329735080071
:10E4C0009385853413850700EF509246EF70501402
:10E4D000930720FE232EF4FA6F00407A832704FA74
:10E4E0006398070E8327C4F96384070E9727FF01FB
:10E4F0009387C7B103A7070083A74700B71600009B
:10E500003378D70093F8070093070800B3E71701A3
:10E51000638A070AEF70100E930630001736080062
:10E520001306C6219305B0081735080013054547A3
:10E53000EF70D07B9727FF019387C7AC83A70700B5
:10E540006388070297C7030083A7C77483A70700E0
:10E5500083A7C700938607001306E0019305100008
:10E560001735080013058524EF70C2046F00C00240
:10E5700097C7030083A7077283A7070083A7C70075
:10E580009386070013061001930510001735080045
:10E590001305C523EF70020297C7030083A7876F97
:10E5A00083A7070083A7C7001736080013060626AF
:10E5B000973508009385452513850700EF5052379E
:10E5C000EF701005930720FE232EF4FA6F00006B06
:10E5D000930500001735080013050526EF70C06E7F
:10E5E0002322A4FCEFB0D01993070500232EF4FAE0
:10E5F0000327C4FB9307F0FF6316F7009307F0FDB2
:10E60000232EF4FA8327C4FB6384070E9727FF01A8
:10E610009387C79F03A7070083A74700B71600008B
:10E62000337DD70093FD070093070D00B3E7B701D3
:10E63000638A070AEF70007C9306300017360800E3
:10E640001306C60F9305A0091735080013054535B5
:10E65000EF70D0699727FF019387C79A83A70700B8
:10E660006388070297C7030083A7C76283A70700D1
:10E6700083A7C70093860700130650019305100077
:10E68000173508001305C51CEF60D2726F00C00279
:10E6900097C7030083A7076083A7070083A7C70066
:10E6A00093860700130680009305100017350800B5
:10E6B0001305851BEF60127097C7030083A7875D62
:10E6C00083A7070083A7C700938607001306D0011E
:10E6D00093051000173508001305C519EF60926DFA
:10E6E000EF7000738327C4FB232EF4FA6F000059E8
:10E6F0009305800513051000EF4092759307050000
:10E700002324F4FC832784FC639807009307A0FF6D
:10E71000232EF4FA6F008056832784FC1307100021
:10E7200023A2E7009307C4FB138607008325C4FADE
:10E73000032584FCEFF08FF98327C4FB639E075207
:10E74000832784FC9387070113860700832584FAB7
:10E75000032544FAEF50400613070500832784FC85
:10E7600023A4E700832784FC83A78700639807001E
:10E770009307A0FF232EF4FA6F004050232604FCD9
:10E780006F008038832784FC03A787008327C4FC9D
:10E79000938617002326D4FC93972700B307F7002E
:10E7A00083A707002320F4FC832704FC639E070C47
:10E7B0009727FF019387878503A7070083A7470053
:10E7C000B7160000337AD70093FA070093070A00C0
:10E7D000B3E757016384070AEF70C0619306300006
:10E7E00017360800130686F59305A00B17350800A9
:10E7F0001305051BEF70904F9727FF0193878780C4
:10E8000083A707006388070297C7030083A7874889
:10E8100083A7070083A7C700938607001306E000BD
:10E8200093051000173508001305C5F1EF609258E5
:10E830006F00000297C7030083A7C74583A707009F
:10E8400083A7C7009385070013050002EF50D21875
:10E8500097C7030083A7074483A7070083A7C700C0
:10E86000938607001306A0029305100017350800D1
:10E8700013054502EF601254EF7080599307F0FDC5
:10E88000232EF4FA6F00003C832744FC639A07129E
:10E89000832704FC03A78712930710006302F71273
:10E8A0009717FF019387877603A7070083A7470081
:10E8B000B716000093860680337BD70093FB0700D2
:10E8C00093070B00B3E777016386070AEF70805266
:10E8D0009306200017360800130686FE9305100CD9
:10E8E000173508001305C50BEF7050409717FF014F
:10E8F0009387477183A707006388070297C70300C0
:10E9000083A7473983A7070083A7C700938607001B
:10E910001306E0009305100017350800130585E283
:10E92000EF6052496F00000297C7030083A7873644
:10E9300083A7070083A7C70093850700130500027C
:10E94000EF50920997C7030083A7C73483A7070036
:10E9500003A7C700832704FC83A7071713860700B4
:10E9600097350800938545F613050700EF50427C64
:10E97000EF70004A832784FC03A78700832784FC69
:10E9800083A707019386F7FF832784FC23A8D7007A
:10E99000832784FC83A70701939727003307F70099
:10E9A000832784FC83A687008327C4FC93972700D2
:10E9B000B387F6000327070023A0E7006F00C01409
:10E9C000832704FC03A7C71293071000630AF712FA
:10E9D000832704FC03A78712930710006302F71232
:10E9E0009717FF019387876203A7070083A7470054
:10E9F000B716000093860680337CD70093FC07008F
:10EA000093070C00B3E797016386070AEF70803E17
:10EA10009306200017360800130686EA9305600C5B
:10EA2000173508001305C5F7EF70502C9717FF0135
:10EA30009387475D83A707006388070297C7030092
:10EA400083A7472583A7070083A7C70093860700EE
:10EA50001306E0009305100017350800130585CE56
:10EA6000EF6052356F00000297C7030083A787222B
:10EA700083A7070083A7C70093850700130500023B
:10EA8000EF50827597C7030083A7C72083A70700AD
:10EA900003A7C700832704FC83A707171386070073
:10EAA00097350800938545E613050700EF50426847
:10EAB000EF700036832784FC03A78700832784FC3C
:10EAC00083A707019386F7FF832784FC23A8D70039
:10EAD000832784FC83A70701939727003307F70058
:10EAE000832784FC83A687008327C4FC9397270091
:10EAF000B387F6000327070023A0E7006F00C000DC
:10EB0000032504FCEF109005832784FC83A70701ED
:10EB10000327C4FCE368F7C6832784FC83A70701A7
:10EB2000639E070C9717FF019387474E03A70700C3
:10EB300083A74700B71600003379D70093F9070081
:10EB400093070900B3E737016384070AEF70802A4F
:10EB50009306300017360800130646BE9305F00CE6
:10EB6000173508001305C5E3EF7050189717FF011C
:10EB70009387474983A707006388070297C7030065
:10EB800083A7471183A7070083A7C70093860700C1
:10EB90001306E0009305100017350800130585BA29
:10EBA000EF6052216F00000297C7030083A7870E12
:10EBB00083A7070083A7C7009385070013050002FA
:10EBC000EF50826197C7030083A7C70C83A7070094
:10EBD00083A7C70093860700130610039305100050
:10EBE00017350800130505D7EF60D21CEF704022DF
:10EBF0009307F0FD232EF4FA6F00C004032584FC74
:10EC0000EF401075832784F963860700832784F912
:10EC100023A00700832784FC13071000238CE70040
:10EC200097C7030083A7C70683A7070013871700AA
:10EC300097C7030083A7C70523A0E700832784FCA9
:10EC40006F000006832784FC83A7870013850700D5
:10EC5000EF601258832784FC23A40700832784FCD9
:10EC600083A7C70013850700EF609256832784FCB3
:10EC700023A607006F00800013000000032584FC1A
:10EC8000EF601255232404FC832784F9638807006E
:10EC90000327C4FB832784F923A0E7009307000020
:10ECA000138507008320C10603248106032941063A
:10ECB00083290106032AC105832A8105032B410507
:10ECC000832B0105032CC104832C8104032D4104F3
:10ECD000832D01041301010767800000130101F96E
:10ECE000232611062324810623222107232031070E
:10ECF000232E4105232C5105232A61052328710564
:10ED000023268105232491052322A1052320B10573
:10ED100013040107232EA4FA232CB4FA232AC4FADD
:10ED20002328D4FA2326E4FA2324F4FA232204FB2A
:10ED3000232014FB232004FC8327C4FB6392070ECB
:10ED40009717FF019387872C03A7070083A7470026
:10ED5000B7160000337DD70093FD070093070D0021
:10ED6000B3E7B701638A070AEF70C0089306300063
:10ED700017760800130646EA9305D00217750800B7
:10ED80001305451DEF7080769717FF01938787273E
:10ED900083A707006388070297C7030083A787EF4D
:10EDA00083A7070083A7C7009386070013066002A6
:10EDB0009305100017750800130585E6EF60827F44
:10EDC0006F00C00297C7030083A7C7EC83A70700A3
:10EDD00083A7C700938607001306900193051000D0
:10EDE00017750800130545E6EF60C27C97C703005E
:10EDF00083A747EA83A7070083A7C7001776080001
:10EE0000130646E697750800938545E713850700C6
:10EE1000EF500232EF60D07F9307C0FD6F00007D9E
:10EE2000832784FB6392070E9717FF019387071EC2
:10EE300003A7070083A74700B7160000337CD7005D
:10EE400093FC070093070C00B3E79701638A070A56
:10EE5000EF60507A93063000177608001306C6DB81
:10EE60009305F002177508001305C50EEF700068D2
:10EE70009717FF019387071983A707006388070285
:10EE800097C7030083A707E183A7070083A7C700ED
:10EE900093860700130630029305100017750800CB
:10EEA000130505DEEF6002716F00C00297C7030013
:10EEB00083A747DE83A7070083A7C70093860700C1
:10EEC000130660019305100017750800130585DD12
:10EED000EF60426E97C7030083A7C7DB83A70700D5
:10EEE00083A7C70017760800130646DD977508004C
:10EEF0009385C5D813850700EF508223EF605071CA
:10EF00009307A0FD6F00806E832784FB83A7C70350
:10EF100063800710832784FB03A7C7018327C4FBF3
:10EF200083A7C70083A7C70BB377F7026382070ED7
:10EF30009717FF019387870D03A7070083A7470053
:10EF4000B7160000337BD70093FB070093070B0035
:10EF5000B3E77701638A070AEF60D0699306300050
:10EF600017760800130646CB9305100317750800A3
:10EF7000130545FEEF7080579717FF0193878708A9
:10EF800083A707006388070297C7030083A787D07A
:10EF900083A7070083A7C700938607001306D00244
:10EFA0009305100017750800130585D2EF60826085
:10EFB0006F00C00297C7030083A7C7CD83A70700D0
:10EFC00083A7C7009386070013060002930510006D
:10EFD000177508001305C5D2EF60C25D97C703001F
:10EFE00083A747CB83A7070083A7C70093860700A3
:10EFF000130610039305100017750800130585D23A
:10F00000EF60425BEF60D060930730FF6F00005EFF
:10F010008327C4FB03A78700832784FB83A787027A
:10F020006302F70E9717FF01938747FE03A70700B8
:10F0300083A74700B7160000337AD70093FA07007A
:10F0400093070A00B3E75701638A070AEF60905AF3
:10F050009306300017760800130606BC93053003AC
:10F0600017750800130505EFEF7040489717FF016B
:10F07000938747F983A707006388070297C70300B0
:10F0800083A747C183A7070083A7C700938607000C
:10F090001306000293051000177508001305C5CB71
:10F0A000EF6042516F00C00297C7030083A787BE7D
:10F0B00083A7070083A7C7009386070013063001C4
:10F0C0009305100017750800130545CBEF60824EBD
:10F0D00097C7030083A707BC83A7070083A7C700C0
:10F0E0009386070013067003930510001775080038
:10F0F000130505CAEF60024CEF6090519307E0FDE5
:10F100006F00C04E832784FB03A7070183A7470135
:10F11000137F073093FF070093070F00B3E7F70152
:10F120006382070E9717FF01938747EE03A7070037
:10F1300083A74700B7160000337ED70093FE070071
:10F1400093070E00B3E7D701638A070AEF60904A7E
:10F150009306300017760800130606AC930560038B
:10F1600017750800130505DFEF7040389717FF018A
:10F17000938747E983A707006388070297C70300BF
:10F1800083A747B183A7070083A7C700938607001B
:10F190001306200293051000177508001305C5C259
:10F1A000EF6042416F00C00297C7030083A787AE9C
:10F1B00083A7070083A7C7009386070013065001A3
:10F1C0009305100017750800130545C2EF60823ED5
:10F1D00097C7030083A707AC83A7070083A7C700CF
:10F1E000938607001306C0049305100017750800E6
:10F1F000130545C1EF60023CEF609041930750FC5E
:10F200006F00C03E832784FA6392070E9717FF01B1
:10F210009387C7DF03A7070083A74700B71600003F
:10F220003373D70093F3070093070300B3E7770026
:10F23000638A070AEF60103C9306300017760800D7
:10F240001306869D9305C00317750800130585D026
:10F25000EF70C0299717FF019387C7DA83A70700CC
:10F260006388070297C7030083A7C7A283A7070085
:10F2700083A7C700938607001306E00193051000DB
:10F2800017750800130505BDEF60C2326F00C0029C
:10F2900097C7030083A707A083A7070083A7C7001A
:10F2A00093860700130610019305100017750800D8
:10F2B000130545BCEF60023097C7030083A7879D05
:10F2C00083A7070083A7C700177608001306C6BBED
:10F2D000977508009385859A13850700EF4052655E
:10F2E000EF601033930720FE6F004030832784FBCC
:10F2F0000326C4FA832504FB13850700EF20D031D1
:10F300009307050063860700930720FE6F00002E19
:10F31000832784FB83A7C70363820702832784FBB9
:10F3200083A7C701032704FBB307F7002328F4FAD8
:10F33000832784FB83A7C703232CF4FA832784FB4A
:10F3400083A78701232CF4F8232E04F88327C4FB1A
:10F3500083A7C70003A7070883A74708032584F9E5
:10F360008325C4F9138605009386070063EEC60063
:10F3700013860500938607006318D60E93060500D2
:10F380009307070063F2D70E9717FF01938707C80B
:10F3900003A7070083A74700B71600003379D700FB
:10F3A00093F9070093070900B3E73701638A070A57
:10F3B000EF60502493063000177608001306C685C8
:10F3C00093053004177508001305C5B8EF700012D7
:10F3D0009717FF01938707C383A707006388070276
:10F3E00097C7030083A7078B83A7070083A7C700DE
:10F3F0009386070013061002930510001775080086
:10F40000130585A9EF60021B6F00C00297C70300B8
:10F4100083A7478883A7070083A7C70093860700B1
:10F42000130640019305100017750800130505A980
:10F43000EF60421897C7030083A7C78583A707001B
:10F4400083A7C700938607001306200393051000C7
:10F4500017750800130505A8EF60C215EF60501B73
:10F460009307B0FF6F008018032604FA832544FA3F
:10F470000325C4FBEF40D01F2324A4FC832784FC76
:10F4800063860700832784FC6F0040168327C4FB34
:10F4900083A7C70013850700EF40802D2322A4FC1B
:10F4A000232604FC6F0040038327C4FB83A7870047
:10F4B00003A787008327C4FC93972700B307F700AF
:10F4C00083A70700032744FC6304F7028327C4FCD7
:10F4D000938717002326F4FC8327C4FB83A78700A8
:10F4E00083A707010327C4FCE360F7FC6F008000DB
:10F4F000130000008327C4FB83A7870083A70701AD
:10F500000327C4FC6362F702977608009386C69FC0
:10F5100017760800130606A49305C00417750800A3
:10F52000130505A1EF404209032744FA930784FB22
:10F53000130504FC9388070013081000832704FABE
:10F5400083260400371600001306461F8325C4FBDC
:10F55000EF10503D2324A4FC832784FC638607001E
:10F56000832784FC6F008008832704FC032784FA28
:10F5700023A0E700832784FB83A6C702832744FCDC
:10F5800083A7471A13974700832704FC3387E600B5
:10F5900023A2E700832704FC032704FB23A4E7003E
:10F5A000832704FC0327C4FA23A6E700832784FBF0
:10F5B00013850700EF509F9E832784FB0327C4FB1E
:10F5C0000327C70023AAE702832704FC93850700CB
:10F5D0000325C4FBEF200001832744FB638607005B
:10F5E0000325C4FBEF0010159307000013850700E7
:10F5F0008320C106032481060329410683290106CD
:10F60000032AC105832A8105032B4105832B0105AC
:10F61000032CC104832C8104032D4104832D010498
:10F620001301010767800000130101F92326110669
:10F63000232481062322910623202107232E31052E
:10F64000232C4105232A5105232861052326710512
:10F650002324810523229105130401072326A4FAFC
:10F660002324B4FA2322C4FA232CD4F8232EE4F85A
:10F670002320F4FA232A04F9232814F9232A04FA6C
:10F68000232204FC8327C4FA6392070E9717FF0115
:10F690009387C79703A7070083A74700B716000003
:10F6A000337CD70093FC070093070C00B3E7970166
:10F6B000638A070AEF6000749306300017A60800FB
:10F6C0001306065A9305A00217A508001305057531
:10F6D000EF60D0619717FF019387C79283A7070058
:10F6E0006388070297B7030083A7C75A83A7070059
:10F6F00083A7C700938607001306600293051000D6
:10F7000017A5080013054556EF50D26A6F00C002D6
:10F7100097B7030083A7075883A7070083A7C700ED
:10F7200093860700130690019305100017A50800A3
:10F7300013050556EF50126897B7030083A7875546
:10F7400083A7070083A7C70017A60800130606565D
:10F7500097A508009385055713850700EF40521DB4
:10F76000EF60006B9307C0FD6F004079832784FA38
:10F770006392070E9717FF019387478903A7070036
:10F7800083A74700B7160000337BD70093FB070021
:10F7900093070B00B3E77701638A070AEF60806580
:10F7A0009306300017A608001306864B9305B00297
:10F7B00017A5080013058566EF6050539717FF01E2
:10F7C0009387478483A707006388070297B70300DE
:10F7D00083A7474C83A7070083A7C700938607002A
:10F7E0001306E0019305100017A508001305C54D89
:10F7F000EF50525C6F00C00297B7030083A78749A0
:10F8000083A7070083A7C70093860700130610018C
:10F810009305100017A508001305054DEF509259E8
:10F8200097B7030083A7074783A7070083A7C700ED
:10F8300017A608001306864C97A5080093858548EF
:10F8400013850700EF40D20EEF60805C930720FE27
:10F850006F00C06A832744FA6392070E9707FF017F
:10F860009387C77A03A7070083A74700B71600004E
:10F87000337FD70093FF070093070F00B3E7F7012B
:10F88000638A070AEF6000579306300017A6080046
:10F890001306063D9305C00217A508001305055879
:10F8A000EF60D0449707FF019387C77583A70700D0
:10F8B0006388070297B7030083A7C73D83A70700A4
:10F8C00083A7C700938607001306E0019305100085
:10F8D00017A508001305453FEF50D24D6F00C00239
:10F8E00097B7030083A7073B83A7070083A7C70039
:10F8F00093860700130610019305100017A5080052
:10F900001305853EEF50124B97B7030083A7873846
:10F9100083A7070083A7C70017A608001306863F22
:10F9200097A508009385053A13850700EF4052001C
:10F93000EF60004E930720FE6F00405C1307C0FF8E
:10F940009307F0FF232CE4FA232EF4FA832784F99B
:10F950000327C4F9B3E7E70063840710032784F99A
:10F96000832784FB337EF7000327C4F98327C4FB76
:10F97000B37EF70093070E00B3E7D7016382070E4B
:10F980009707FF019387876803A7070083A74700AE
:10F99000B71600003373D70093F3070093070300F3
:10F9A000B3E77700638A070AEF60C044930630002C
:10F9B00017A608001306C62A9305000317A508001A
:10F9C0001305C545EF6090329707FF019387876362
:10F9D00083A707006388070297B7030083A7872BD5
:10F9E00083A7070083A7C700938607001306E001DB
:10F9F0009305100017A508001305052DEF50923B45
:10FA00006F00C00297B7030083A7C72883A707002A
:10FA100083A7C70093860700130610019305100003
:10FA200017A508001305452CEF50D23897B70300EF
:10FA300083A7472683A7070083A7C70017A6080048
:10FA40001306C62E97A508009385C52713850700C2
:10FA5000EF40026EEF60C03B930720FE6F00004A4C
:10FA6000032644F9832504FA0325C4FAEF404040F5
:10FA70002324A4FC832784FC63860700832784FC5B
:10FA80006F00C047832584FA13054000EF30523CD5
:10FA9000930705002322F4FC232604FC6F00C030EA
:10FAA0008327C4FC93972700032744FAB307F70082
:10FAB00083A707006394070E9707FF0193870755F5
:10FAC00003A7070083A74700B71600003379D700C4
:10FAD00093F9070093070900B3E73701638A070A20
:10FAE000EF6040319306300017A608001306461752
:10FAF0009305D00317A5080013054532EF60101FCA
:10FB00009707FF019387075083A7070063880702C1
:10FB100097B7030083A7071883A7070083A7C70029
:10FB200093860700130630029305100017A50800FE
:10FB300013058522EF5012286F00C00297B703000B
:10FB400083A7471583A7070083A7C70093860700ED
:10FB5000130660019305100017A508001305052280
:10FB6000EF50522597B7030083A7C71283A707005A
:10FB700083A7C70017A608001306C62197A508008B
:10FB80009385451413850700EF40825AEF604028A3
:10FB90009307A0FD2324F4FC6F0000348327C4FCEA
:10FBA00093972700032744FAB307F70083A70700BA
:10FBB00003A787028327C4FA83A787006304F70E8D
:10FBC0009707FF019387874403A7070083A7470090
:10FBD000B7160000337AD70093FA070093070A009C
:10FBE000B3E75701638A070AEF60C020930630002D
:10FBF00017A608001306C6069305F00317A508000C
:10FC00001305C521EF60900E9707FF019387873F8B
:10FC100083A707006388070297B7030083A78707B6
:10FC200083A7070083A7C700938607001306000277
:10FC30009305100017A5080013058517EF509217BC
:10FC40006F00C00297B7030083A7C70483A707000C
:10FC500083A7C700938607001306300193051000A1
:10FC600017A5080013050517EF50D21497B7030026
:10FC700083A7470283A7070083A7C70017A608002A
:10FC80001306861697A508009385C50313850700FC
:10FC9000EF40024AEF60C0179307E0FD2324F4FC15
:10FCA0006F0080238327C4FC93972700032744FA1F
:10FCB000B307F70083A7070083A7C703639807026A
:10FCC0008327C4FC93972700032744FA3307F700E0
:10FCD0008327C4FC93972700832644FCB387F60050
:10FCE0000327070023A0E7006F0000038327C4FC5D
:10FCF00093972700032744FAB307F70003A70700E9
:10FD00008327C4FC93972700832644FCB387F6001F
:10FD10000327C70323A0E7008327C4FC939727008A
:10FD2000032744FCB307F70083A7070083A78704D2
:10FD3000638207048327C4FC93972700032744FCAE
:10FD4000B307F70083A7070003A78700B7170000D2
:10FD50009387670F6310F7028327C4FC93972700EC
:10FD6000032744FCB307F70083A7070083A7C7074F
:10FD70006F0080018327C4FC93972700032744FC6E
:10FD8000B307F70083A707000327C4FC1317270056
:10FD9000832644FC3387E6002320F7008327C4FC36
:10FDA000938717002326F4FC0327C4FC832784FAD7
:10FDB000E368F7CE032704FA130544FB832844FCC9
:10FDC000032884FA832744F9832604F937160000B0
:10FDD000130666208325C4FAEF10C0342324A4FC44
:10FDE000832784FC6398070E8327C4FA03A7C70000
:10FDF000832744FB0327871923A0E700832744FBBD
:10FE0000032784FA23A2E700832744FB032744FC4B
:10FE100023A4E700832784FA93972700832444FBD5
:10FE200013850700EF50D2399307050023A6F4008D
:10FE3000232604FC6F00C0078327C4FC9397270088
:10FE4000032744FCB307F70083A7070013850700C7
:10FE5000EF50CF948327C4FC93972700032744FCDB
:10FE6000B307F70003A70700832744FB83A6C70057
:10FE70008327C4FC93972700B387F6000327470323
:10FE800023A0E7008327C4FC93972700032744FCA3
:10FE9000B307F70083A707000327C4FA0327C700A7
:10FEA00023AAE7028327C4FC938717002326F4FCC8
:10FEB0000327C4FC832784FAE360F7F8832744FB15
:10FEC000938507000325C4FAEF10C0719307000063
:10FED0006F00C00213000000032544FCEF50522FB6
:10FEE000232204FC832744FB13850700EF50522E86
:10FEF000032504F9EF50D22D832784FC13850700D6
:10FF00008320C106032481068324410603290106B8
:10FF10008329C105032A8105832A4105032B010595
:10FF2000832BC104032C8104832C4104130101079A
:10FF300067800000130101FE232E1100232C810095
:10FF4000130401022326A4FE0325C4FEEF000004CF
:10FF50008327C4FE83A7C70083A7472503A787007D
:10FF60008327C4FE83A7C7008325C4FE138507002B
:10FF7000E700070093070000138507008320C101F5
:10FF8000032481011301010267800000130101FEB7
:10FF9000232E1100232C8100130401022326A4FE2A
:10FFA0008327C4FE83A7C70083A7472583A7C7006D
:10FFB000638407028327C4FE83A7C70083A747255E
:10FFC00003A7C7008327C4FE83A7C7008325C4FEF9
:10FFD00013850700E700070093070000138507005B
:10FFE0008320C10103248101130101026780000005
:10FFF000130101FD23261102232481022322210360
:02000004800179
:100000002320310313040103232EA4FC8325C4FD04
:100010006392050E9707FF01938747FF03A7070029
:1000200083A74700B71500003376B70093F60700A3
:1000300093070600B3E7D700638A070AEF50905B87
:1000400093063000175609001306C6D59305D00154
:1000500017550900130505E4EF6040499707FF01B4
:10006000938747FA83A707006388070297B70300BF
:1000700083A747C283A7070083A7C700938607000B
:100080001306F0019305100017550900130505D25A
:10009000EF5042526F00C00297B7030083A787BF9B
:1000A00083A7070083A7C7009386070013062001D4
:1000B0009305100017550900130545D1EF50824FE5
:1000C00097B7030083A707BD83A7070083A7C700CF
:1000D000175609001306C6D097550900938585D198
:1000E00013850700EF40C204EF5090529307F0FDD4
:1000F0006F0000258326C4FD83A686016396060053
:10010000930700006F00C0238326C4FD83A646002A
:100110006342D00297560900938606CE175609000F
:10012000130646D79305300217550900130585CEEF
:10013000EF3082488326C4FD83A646009386F6FFEF
:100140000326C4FD2322D6002326D4FE8326C4FD25
:1001500083A6460063D2060297560900938646CDD1
:1001600017560900130606D39305300217550900E8
:10017000130545CAEF3042448326C4FE6398060E39
:100180008327C4FD83A7471613850700EF50520449
:100190008327C4FD23A207169707FF01938707E76C
:1001A00003A7070083A747001379070493F9070003
:1001B00093070900B3E737016382070AEF509043C2
:1001C0009306100017560900130686C8930590027F
:1001D00017550900130505CCEF6040319707FF0163
:1001E000938747E283A707006388070297B7030056
:1001F00083A747AA83A7070083A7C70093860700A2
:100200001306E0009305100017550900130505C5F6
:10021000EF50423A6F00000297B7030083A787A709
:1002200083A7070083A7C700938507001305000273
:10023000EF30927A97B7030083A7C7A583A707007B
:1002400083A7C7000326C4FD97550900938505C2FF
:1002500013850700EF30D26DEF50903B0325C4FDAE
:10026000EF500277232E04FC6F00400D9706FF012C
:100270009386C6D903A6060083A646001377060414
:1002800093F7060093060700B3E6F6006388060AB4
:10029000EF5050369306100017560900130646BB60
:1002A0009305D002175509001305C5BEEF60002461
:1002B0009707FF01938707D583A707006388070285
:1002C00097B7030083A7079D83A7070083A7C700ED
:1002D000938607001306E0009305100017550900E8
:1002E0001305C5B7EF50022D6F00000297B703004A
:1002F00083A7479A83A7070083A7C70093850700B2
:1003000013050002EF30526D97B7030083A787985B
:1003100083A7070003A7C7008327C4FD83A747005F
:10032000938607000326C4FD97550900938505B5FC
:1003300013050700EF30D25FEF50902D93070000B8
:10034000138507008320C10203248102032941028F
:10035000832901021301010367800000130101FDDD
:10036000232611022324810213040103232EA4FC5B
:100370008326C4FD83A686016396060093070000CA
:100380006F0000148326C4FD83A646006342D0029A
:10039000978609009386064F17860900130646576D
:1003A00093050002178509001305854FEF30C22021
:1003B0008326C4FD83A64600938616000326C4FD4B
:1003C0002322D6002326D4FE8326C4FD83A646001E
:1003D00063D20602978609009386464E1786090067
:1003E0001306065393050002178509001305454BB4
:1003F000EF30821C9706FF01938646C103A60600D4
:1004000083A646001377060493F7060093060700B9
:10041000B3E6F6006384060AEF50D01D9306100081
:10042000178609001306864B9305100217850900ED
:100430001305054EEF60800B9707FF01938787BC7C
:1004400083A707006388070297B7030083A7878401
:1004500083A7070083A7C700938607001306E00061
:10046000930510001785090013050548EF50821405
:100470006F00000297B7030083A7C78183A7070017
:1004800083A7C7009385070013050002EF30D254FD
:1004900097B7030083A7078083A7070083A7C70038
:1004A0008326C4FE0326C4FD978509009385C544B1
:1004B00013850700EF30D247EF50901593070000E7
:1004C000138507008320C102032481021301010365
:1004D00067800000130101FE232E81001304010236
:1004E0002326A4FE8327C4FE83A7470293B71700E1
:1004F00093F7F70F138507000324C10113010102CD
:1005000067800000130101FE232E81001304010205
:100510002326A4FE130000000324C10113010102DD
:1005200067800000130101FF2326810013040101ED
:1005300093070000138507000324C1001301010184
:1005400067800000130101FE232E810013040102C5
:100550002326A4FE130000000324C101130101029D
:1005600067800000130101FF2326810013040101AD
:10057000130000000324C100130101016780000083
:10058000130101FF232681001304010193070000DA
:10059000138507000324C1001301010167800000D7
:1005A000130101FE232E8100130401022326A4FE61
:1005B000130000000324C101130101026780000041
:1005C000130101FD2326810213040103232EA4FC41
:1005D00093870500A30DF4FC8347B4FD63960700E1
:1005E0008327C4FD6F0000038327C4FD2326F4FE88
:1005F0008347F4FE2304F4FE8347E4FEA304F4FEE1
:100600008347D4FE2305F4FE8347C4FEA305F4FE0E
:10061000832784FE138507000324C102130101030D
:1006200067800000130101FD2326810213040103EA
:10063000232EA4FC93870500A30DF4FC8347B4FD8F
:10064000639607008327C4FD6F0000038327C4FD62
:100650002326F4FE8347F4FE2304F4FE8347E4FEDE
:10066000A304F4FE8347D4FE2305F4FE8347C4FEAF
:10067000A305F4FE832784FE138507000324C1022B
:100680001301010367800000130101FE232E810086
:10069000130401022326A4FE8327C4FE9387F7FFD9
:1006A0002326F4FE8327C4FE93D717000327C4FE36
:1006B000B367F7002326F4FE8327C4FE93D72700F1
:1006C0000327C4FEB367F7002326F4FE8327C4FE86
:1006D00093D747000327C4FEB367F7002326F4FE31
:1006E0008327C4FE93D787000327C4FEB367F700B0
:1006F0002326F4FE8327C4FE93D707010327C4FEF5
:10070000B367F7002326F4FE8327C4FE9387170000
:100710002326F4FE8327C4FE138507000324C101AA
:100720001301010267800000130101FD23268102ED
:10073000232421032322310323204103232E5101AB
:1007400013040103232CA4FC232EB4FC032F84FDEB
:10075000832FC4FD130AF0FF930AF0FF33054F0106
:1007600093020500B3B2E201B3855F01338FB2009B
:1007700093050F00232CA4FC232EB4FC8325C4FD79
:100780009395F501032584FD135E150033EEC50135
:100790008325C4FD93DE1500832584FDB3E5C501E3
:1007A000232CB4FC8325C4FDB3E5D501232EB4FC72
:1007B0008325C4FD9395E501032584FD135325008E
:1007C00033E365008325C4FD93D32500832584FD91
:1007D000B3E56500232CB4FC8325C4FDB3E57500A7
:1007E000232EB4FC8325C4FD9395C501032584FD08
:1007F0001358450033E805018325C4FD93D845000F
:10080000832584FDB3E50501232CB4FC8325C4FDB9
:10081000B3E51501232EB4FC8325C4FD9395850112
:10082000032584FD1356850033E6C5008325C4FDEA
:1008300093D68500832584FDB3E5C500232CB4FC45
:100840008325C4FDB3E6D500232ED4FC8326C4FD46
:1008500093960601032684FD1357060133E7E6004D
:100860008326C4FD93D70601832684FDB3E6E60004
:10087000232CD4FC8326C4FDB3E7F600232EF4FC1E
:100880008327C4FD13D9070093090000832784FD43
:10089000B3E72701232CF4FC8327C4FDB3E737011A
:1008A000232EF4FC032684FD8326C4FD13051000CB
:1008B000930500003307A600130807003338C8006B
:1008C000B387B600B306F80093870600232CE4FC38
:1008D000232EF4FC032784FD8327C4FD13050700A2
:1008E000938507000324C102032981028329410261
:1008F000032A0102832AC10113010103678000005A
:10090000130101FD23261102232481021304010394
:10091000232EA4FC232CB4FC8327C4FD938737002B
:100920002326F4FE0327C4FE832784FDB307F700C4
:1009300013850700EF50C208930705002324F4FE37
:10094000832784FE63960700930700006F0040032F
:10095000032784FE8327C4FE3307F7008327C4FDE3
:10096000B307F040B377F7002322F4FE832744FE59
:100970009387C7FF032784FE23A0E700832744FE55
:10098000138507008320C1020324810213010103A0
:1009900067800000130101FE232E1100232C81002B
:1009A000130401022326A4FE8327C4FE638C0700E0
:1009B0008327C4FE9387C7FF83A70700138507001B
:1009C000EF500201130000008320C10103248101C4
:1009D0001301010267800000130101FE232E1100A4
:1009E000232C8100130401022326A4FE2324B4FE39
:1009F0000327C4FE832784FE6312F70297C609000B
:100A00009386468817C609001306464B93050014C3
:100A100017C509001305C587EF20123A8327C4FEC6
:100A200003A78701832784FE83A787016312F70248
:100A300097C609009386468717C60900130606481D
:100A40009305101417C5090013058584EF20D236CD
:100A50008327C4FE03A78701832784FE83A787011A
:100A6000637EF7048327C4FE83A747006342F00236
:100A700097C609009386868417C6090013060644A4
:100A80009305401417C5090013058580EF20D23265
:100A9000832784FE83A74700634EF00697C60900AC
:100AA0009386868317C609001306464193055014A2
:100AB00017B509001305C57DEF201230832784FE8A
:100AC00083A747006342F00297C609009386C68059
:100AD00017C609001306863E9305901417B5090042
:100AE0001305057BEF20522D8327C4FE83A7470003
:100AF0006342F00297B609009386467C17C6090048
:100B00001306C63B9305A01417B5090013054578D5
:100B1000EF20922A130000008320C10103248101E9
:100B20001301010267800000130101FE232E110052
:100B3000232C8100130401022326A4FE2324B4FEE7
:100B40000327C4FE832784FE6312F70297B60900C9
:100B50009386467317C609001306063893051015C9
:100B600017B509001305C572EF2012258327C4FEAF
:100B700003A78701832784FE83A787016312F702F7
:100B800097B609009386467217C609001306C63445
:100B90009305201517B509001305856FEF20D221A5
:100BA0008327C4FE03A78701832784FE83A78701C9
:100BB000637EF7048327C4FE83A7470063D207023E
:100BC00097B609009386067317C609001306C63048
:100BD0009305501517B509001305856BEF20D21D3D
:100BE000832784FE83A7470063DE070697B60900C4
:100BF0009386067217C609001306062E9305601524
:100C000017B509001305C568EF20121B832784FE62
:100C100083A7470063D2070297B609009386466F01
:100C200017C609001306462B9305A01517B5090032
:100C300013050566EF2052188327C4FE83A74700DB
:100C400063D2070297B609009386C66A17C60900E1
:100C5000130686289305B01517B5090013054563DB
:100C6000EF209215130000008320C10103248101AD
:100C70001301010267800000130101FC232E110201
:100C8000232C8102232A91022328210323263103C6
:100C900013040104232EA4FC232CB4FC232AC4FC3B
:100CA0002328D4FC2326E4FC2324F4FC832784FC9F
:100CB00063880700832784FC83C787016396070046
:100CC0009307E0FD6F00401D8327C4FD6384071C6C
:100CD000EF50400D130705008327C4FD23A0E70054
:100CE0008327C4FD83A70700639607009307A0FF2F
:100CF0006F00801A8327C4FD83A70700032784FCA5
:100D000023A4E700032584FCEF1011158327C4FDFD
:100D100083A70700032784FD23A6E700832784FD1C
:100D200063860700032584FDEF10D1378327C4FDB8
:100D300083A70700032744FD23A8E70097B709000E
:100D40009387075403A707008327C4FD83A70700E1
:100D50001307170023ACE7008327C4FD83A7070010
:100D6000032704FD23A6E70297F7FE019387072ACE
:100D700003A7070083A747001379870093F90700AB
:100D800093070900B3E737016388070AEF5080062D
:100D90009306100017B60900130646599305A017CD
:100DA00017C5090013050515EF50407497F7FE01AC
:100DB0009387472583A707006388070297A7030047
:100DC00083A747ED83A7070083A7C7009386070083
:100DD0001306E0009305100017B5090013058555AB
:100DE000EF40427D6F00000297A7030083A787EAC8
:100DF00083A7070083A7C700938507001305000298
:100E0000EF30823D97A7030083A7C7E883A70700B9
:100E100003A7C7008327C4FD83A7070083A7870113
:100E20001386070097B509009385C5511305070080
:100E3000EF300230EF40D07D832704FD6384070448
:100E4000832704FD139727008327C4FD83A407008D
:100E500013050700EF40D2369307050023A4F402E0
:100E60008327C4FD83A7070003A78702832704FD08
:100E700093972700138607008325C4FC13050700FA
:100E8000EF5042468327C4FD83A7070013073000B5
:100E900023A8E70293070000138507008320C103FE
:100EA0000324810383244103032901038329C1020D
:100EB0001301010467800000130101FD23261102C4
:100EC0002324810213040103232EA4FC232CB4FC4D
:100ED000232604FE232404FE832684FD6396060055
:100EE000930700006F00C02297F6FE01938606125A
:100EF00003A6060083A646001377860093F7060034
:100F000093060700B3E6F600638A060AEF40906E88
:100F10009306100017B60900130646419305001901
:100F200017C50900130545FEEF50405C97F7FE0119
:100F30009387470D83A707006388070297A70300DD
:100F400083A747D583A7070083A7C7009386070019
:100F50001306E0009305100017B509001305853D41
:100F6000EF4042656F00000297A7030083A787D276
:100F700083A7070083A7C700938507001305000216
:100F8000EF30822597A7030083A7C7D083A7070068
:100F900003A7C7008327C4FD03A68701832784FD19
:100FA00083A787019386070097B509009385453B82
:100FB00013050700EF30C217EF409065832584FDCD
:100FC0000325C4FDEFF05FA1832784FD83A74700BD
:100FD0006392070297B609009386463B17C609003D
:100FE000130686F29305501917B509001305452A13
:100FF000EF20825C0327C4FD832784FD6312F70280
:1010000097B609009386C63A17C609001306C6EFBD
:101010009305601917B5090013058527EF20C259FC
:101020008327C4FD83A747022324F4FE6F00000238
:10103000832784FE83A70700032784FD630CF70A38
:10104000832784FE83A747002324F4FE832784FE9E
:10105000E39007FE832784FD83A707036380070AC5
:101060009305800013051000EF20825E93070500B2
:101070002326F4FE9305800013051000EF20425D47
:10108000930705002324F4FE8327C4FE638607002C
:10109000832784FE639607009307A0FF6F00400735
:1010A0008327C4FE0327C4FD23A0E700832784FE13
:1010B000032784FD23A0E7008327C4FE032784FDC4
:1010C0000327070223A2E7000327C4FE832784FD2A
:1010D00023A0E702832784FE0327C4FD03274702DA
:1010E00023A2E700032784FE8327C4FD23A2E7028F
:1010F0006F000001130000006F008000130000006B
:10110000832584FD0325C4FDEFF01FA29307000093
:10111000138507008320C102032481021301010308
:1011200067800000130101FB23261104232481049E
:101130002322210523203105232E4103232C510393
:10114000232A610323287103130401052326A4FC29
:101150002324B4FC2322C4FC2320D4FC232EE4FA51
:10116000232CF4FA232A04FB232814FB232C04FC4D
:10117000832784FB639607008327C4FB639A0700D9
:10118000832784FB638607028327C4FB63920702DD
:1011900097B609009386C62317C60900130646D8DA
:1011A0009305C01B17B509001305850EEF20C2403B
:1011B000232E04FC6F0000038327C4FD93972700B0
:1011C000032784FBB307F70083A707006396070094
:1011D000930770FC6F00403E8327C4FD9387170080
:1011E000232EF4FC0327C4FD8327C4FBE346F7FC4E
:1011F0009305800713051000EF2082459307050033
:10120000138707008327C4FC23A0E7008327C4FCBF
:1012100083A70700639607009307A0FF6F00C039FC
:101220008327C4FC83A70700032744FC23ACE704FF
:101230008327C4FC83A7070093874706232CF4FC6D
:10124000832784FC83A78700032704FB832644FBB2
:1012500013060000832584FC032584FDEFF0DFA145
:10126000232AA4FC832744FD638207028327C4FC4E
:1012700083A7070013850700EF4082758327C4FC0E
:1012800023A00700832744FD6F000033832784FDDC
:1012900083A70700032744FC23A8E700832704FC57
:1012A000638E070E97F7FE01938747D603A70700C3
:1012B00083A74700137B870093FB070093070B006E
:1012C000B3E777016384070AEF40D032930610003A
:1012D00017B60900130686059305C01D17C509003A
:1012E000130505C4EF50802097F7FE01938787D13F
:1012F00083A707006388070297A7030083A787993E
:1013000083A7070083A7C700938607001306E000A2
:101310009305100017B509001305C501EF40822998
:101320006F00000297A7030083A7C79683A7070053
:1013300083A7C7009385070013050002EF20D26939
:1013400097A7030083A7079583A7070083A7C70074
:1013500093860700130670019305100017B5090066
:1013600013054507EF400225EF40902A832784FDAF
:1013700003A70700832704FC23A0E700832784FD3D
:1013800083A7070023A00706832784FD83A7070000
:101390001307200023A2E7006F004002832784FD8B
:1013A00083A707001307100023A0E706832784FD07
:1013B00083A707001307100023A2E7008327C4FCBC
:1013C00083A70700032784FC0327C70023A6E7069B
:1013D0008327C4FC83A7070083A747060327C4FC11
:1013E0000327070023AAE700832784FC03A707013C
:1013F00083A74701137A170093FA070093070A009F
:10140000B3E7570163940708832784FC83A7470049
:101410006342F00297B60900938646FD17C609009D
:10142000130606B09305E01E17B50900130545E63F
:10143000EF208218832784FC83A747026382070278
:101440008327C4FC83A7070003A74706832784FCE0
:1014500083A747029385070013050700EFF0DFA578
:10146000832784FC83A7470063D2070297B609004D
:10147000938606FA17C60900130686AA9305401F2D
:1014800017B509001305C5E0EF200213232E04FC55
:101490006F0000048327C4FD93972700032784FB74
:1014A000B307F70083A707002328F4FC8327C4FCB5
:1014B00083A7070083A74706832504FD138507003C
:1014C000EFF09F9F8327C4FD93871700232EF4FC22
:1014D0000327C4FD8327C4FBE34EF7FA97F7FE0109
:1014E0009387C7B203A7070083A747001379870034
:1014F00093F9070093070900B3E73701638C070AE4
:10150000EF40500F9306100017B60900130606E2CD
:101510009305C01F17C50900130585A0EF40107D76
:1015200097F7FE01938707AE83A70700638807023A
:101530009797030083A7077683A7070083A7C700B1
:10154000938607001306E0009305100017B5090005
:10155000130545DEEF4002066F0000029797030077
:1015600083A7477383A7070083A7C7009385070056
:1015700013050002EF2052469797030083A7877157
:1015800083A7070003A7C7008327C4FC83A707001E
:1015900083A7470683A78701832644FC1386070099
:1015A00097B50900938505E913050700EF20523828
:1015B000EF40100693070000138507008320C10445
:1015C000032481040329410483290104032AC1035C
:1015D000832A8103032B4103832B0103130101059C
:1015E00067800000130101FD2326110223248102DC
:1015F000232221032320310313040103232EA4FCFF
:10160000232CB4FC832784FD83A7470683A74700C8
:101610006342F00297B60900938686E417C6090074
:10162000130646919305702017B50900130545C6AA
:10163000EF109278832784FD83A7470603A707034B
:10164000930730006302F70297B60900938686E39A
:1016500017C609001306068E9305802017B50900EA
:10166000130505C3EF105275832784FD83A7470632
:1016700083A7C7000327C4FD6302F70297B60900DA
:10168000938686E217C609001306C68A9305902042
:1016900017B509001305C5BFEF101272832784FD2B
:1016A00083A7470683A7470063D2070297B60900BE
:1016B0009386C6E117C609001306C6879305A020C6
:1016C00017B509001305C5BCEF10126F8327C4FDC1
:1016D00083A747006342F00297B60900938606D1BC
:1016E00017C60900130606859305C02017B5090023
:1016F000130505BAEF10526C8327C4FD83A70702B8
:10170000138717008327C4FD23A0E702832784FDE6
:1017100003A78705B717000093875720630CF700CE
:10172000832784FD03A78705B71700009387E71F6A
:101730006314F704832784FD83A74700639E070291
:101740008327C4FD83A787012326F4FE6F00400290
:10175000832784FD83A747068325C4FE13850700DE
:10176000EFF08FF58327C4FE83A747062326F4FEF8
:101770008327C4FEE39E07FC832784FD03A7870518
:10178000B717000093875720631CF700832784FD59
:1017900003A747068327C4FD23AEE7006F00C002FE
:1017A0008327C4FD83A7C70163800702832784FDC5
:1017B00003A747068327C4FD83A7C70193850700B6
:1017C00013050700EFF04FEF8327C4FD83A78701C0
:1017D000638C07048327C4FD03A78701832784FD47
:1017E00083A747060327870623A4E7068327C4FDAC
:1017F00083A7870183A78706032784FD032747065E
:1018000023A2E7068327C4FD83A78701032784FD5E
:101810000327470623A4E706832784FD83A74706FB
:1018200023A207066F004003832784FD03A7470612
:101830008327C4FD23ACE7008327C4FD83A787016A
:101840000327C4FD0327870123A4E7068327C4FDDC
:1018500083A7870123A2070697E7FE019387077BEB
:1018600003A7070083A747001379870093F90700B0
:1018700093070900B3E737016388070AEF408057F1
:101880009306100017B60900130646AA9305102206
:1018900017B509001305056AEF40504597E7FE01AB
:1018A0009387477683A7070063880702979703000B
:1018B00083A7473E83A7070083A7C7009386070037
:1018C0001306E0009305100017B50900130585A65F
:1018D000EF30524E6F0000029797030083A7873BBB
:1018E00083A7070083A7C70093850700130500029D
:1018F000EF20920E9797030083A7C73983A70700AD
:1019000003A7C700832784FD83A7470683A7870112
:101910001386070097B50900938585BD1305070059
:10192000EF201201EF40C04E832784FD03A7470636
:101930008327C4FD23A2E7028327C4FD83A74700B2
:1019400063D2070297B60900938686AC17B60900E2
:101950001306465E9305302217B50900130545931B
:10196000EF109245832784FD83A7470683A747008E
:101970006342F00297B60900938686AE17B6090057
:101980001306465B9305502217B5090013054590D1
:10199000EF109242832784FD83A747061385070033
:1019A000EF20D03E8327C4FD83A7C70083A7472528
:1019B00083A747008325C4FD032584FDE780070036
:1019C000130000008320C102032481020329410285
:1019D000832901021301010367800000130101FE46
:1019E000232E1100232C8100130401022326A4FEC0
:1019F0002324B4FE2322C4FE8327C4FE639207027D
:101A000097B60900938686B017B6090013060654E8
:101A10009305202317B5090013058587EF10D239E8
:101A2000832784FE83A707006386070A832784FE33
:101A300083A7070083A70706638E0708832784FE12
:101A400083A7070083A7070603A78705B71700002A
:101A5000938757206310F708832744FE83A7070066
:101A600063860704832744FE83A7070003A70706AE
:101A70008327C4FE23A0E706832744FE03A70700AD
:101A80008327C4FE23AEE704832744FE83A7070011
:101A90000327C4FE23A0E7068327C4FE83A7070607
:101AA0000327C4FE23AEE7046F00C0018327C4FEF2
:101AB0000327C4FE23A0E7068327C4FE0327C4FE32
:101AC00023AEE704832744FE0327C4FE23A0E700D8
:101AD0006F0000128327C4FE83A747061385070003
:101AE000EFE05F9F93070500638807088327C4FE24
:101AF00083A7470613850700EF209038832784FECD
:101B000083A7070063860704832784FE83A7070053
:101B100003A707068327C4FE23A0E706832784FEC6
:101B200003A707008327C4FE23AEE704832784FEB0
:101B300083A707000327C4FE23A0E7068327C4FE6C
:101B400083A707060327C4FE23AEE7046F00C00186
:101B50008327C4FE0327C4FE23A0E7068327C4FE11
:101B60000327C4FE23AEE704832784FE0327C4FEB5
:101B700023A0E7006F00C007832744FE83A7070068
:101B800063860704832744FE83A7070003A707068D
:101B90008327C4FE23A0E706832744FE03A707008C
:101BA0008327C4FE23AEE704832744FE83A70700F0
:101BB0000327C4FE23A0E7068327C4FE83A70706E6
:101BC0000327C4FE23AEE7046F00C0018327C4FED1
:101BD0000327C4FE23A0E7068327C4FE0327C4FE11
:101BE00023AEE704832744FE0327C4FE23A0E700B7
:101BF0008320C101032481011301010267800000D9
